:020000022000DC
:106000000000042071630200596302005B63020018
:106010005D6302005F630200616302000000000034
:1060200000000000000000000000000063630200A8
:1060300065630200000000006763020069630200FC
:1060400001AC02006B630200BDB702006B6302008B
:106050006B6302006B630200D5B402006B63020045
:106060006B6302006B6302006B6302006B630200F0
:106070006B6302006B6302006B6302006B630200E0
:106080006B6302000D8802006B6302006B63020009
:106090004D8802006B630200110903006B6302006C
:1060A0006B6302006B6302006B6302006B630200B0
:1060B0006B6302006B630200000000000000000040
:1060C0006B6302006B6302006B6302006B63020090
:1060D0006B6302006B6302006B6302006B63020080
:1060E0006B6302006B6302006B6302000000000040
:1060F000000000006B630200000000006B63020000
:10610000000000000000000000000000000000008F
:10611000000000000000000000000000000000007F
:10612000000000000000000000000000000000006F
:10613000000000000000000000000000000000005F
:10614000000000000000000000000000000000004F
:10615000000000000000000000000000000000003F
:10616000000000000000000000000000000000002F
:10617000000000000000000000000000000000001F
:10618000000000000000000000000000000000000F
:1061900000000000000000000000000000000000FF
:1061A00000000000000000000000000000000000EF
:1061B00000000000000000000000000000000000DF
:1061C00000000000000000000000000000000000CF
:1061D00000000000000000000000000000000000BF
:1061E00000000000000000000000000000000000AF
:1061F000000000000000000000000000000000009F
:10620000344935480A1A02D0072291438D46334952
:1062100033480A1A06D00722914381F309880222E3
:1062200082F314882F483049304A00F041F8304852
:106230003049314A00F03CF830483149314A00F0E9
:1062400037F831483149324A00F032F831483249A2
:10625000324A00F02DF832483249334A00F028F82B
:1062600032483349334A00F023F833483349002297
:1062700000F029F832483349002200F024F832486F
:106280003249091A0BF01CFB314A90471F4820493C
:10629000884205D00268043003B4904703BCF7E796
:1062A00000208646EC46002000212A4A9047FEE75F
:1062B000884207D0521A05D0037801300B700131A3
:1062C000013AF9D17047884202D002700130FAE7F2
:1062D000704700000000042000E0032000000420BC
:1062E0000000042080320300982A0020842B002024
:1062F000D0630200D0630200D41803008032030090
:10630000982A0020982A0020B8190300B819030021
:10631000B8190300B8190300B8190300B81903002D
:10632000B8190300B8190300803203006C3303006E
:10633000842B0020842B0020842B0020EC3A0020AA
:10634000EC3A0020EC3A0020EC3A0020EC5A002015
:1063500099630200F9DD0200FEE7FEE7FEE7FEE7D3
:10636000FEE7FEE7FEE7FEE7FEE7FEE7704700BF59
:106370001048804710484FF00701884385460F4872
:1063800080470F48016841F470010160BFF34F8FEF
:10639000BFF36F8FFFF734BF0A480B490B4A88429F
:1063A00007D0521A05D0037801300B700131013A41
:1063B000F9D170476D630200000004203DA1020086
:1063C00088ED00E0B8190300982A0020982A0020E0
:1063D00000B585B00190019B002B0AD0074B43F01C
:1063E00001030393019B9B010293039B029898472F
:1063F00000E000BF05B05DF804FB00BFD01903004A
:1064000000B583B00190019B002B0AD04FF47A7045
:10641000FFF7DEFF019B013B0193019B002BF5D1B0
:1064200000E000BF03B05DF804FB08B507F080FE94
:1064300000BF08BD00B589B0039002910192019B95
:10644000002B33D00023079303230693029A079B64
:106450001344019A1946002007F0F4FD0590079AAD
:10646000059B13440793019A059BD31A0193059B3F
:10647000002B13D10F4B1B7883F00103DBB2002BF1
:1064800013D10120FFF7BCFF069B013B0693069B3F
:10649000002B03D1074B00221A7007E0054B0122A5
:1064A0001A70019B002BD1D100E000BF00BF09B0E2
:1064B0005DF804FB842B002000B585B003900291A9
:1064C000054B00934023054A0299039800F012F807
:1064D00000BF05B05DF804FB35640200882B002086
:1064E00082B0019000BF02B0704782B0019000BF3F
:1064F00002B0704700B5A1B00590049103920293D9
:10650000049803F0A1FB039B1593029B16930023B1
:10651000179300238DF8603000231993229B1A9360
:1065200000231F930FA91F9B0822049803F066FC09
:1065300008231F93119B1293BDF84030ADF84C30E7
:10654000BDF84230ADF84E3000238DF851309DF843
:106550003C3003F00303DBB2012B26D10F9BC3F3C6
:1065600095231C939DF83C30C3F3C203DBB28DF836
:106570005030BDF83C30C3F38313DBB21B931B9B3D
:106580009A0009A91F9B049803F038FC1B9B9B00F1
:106590001F9A13441F9312AA09A915AB009313461F
:1065A0001B9A1C9800F078FF2FE09DF83C3003F018
:1065B0000303DBB2022B28D1BDF83E30C3F38913AD
:1065C0009BB21E939DF83C30C3F3C203DBB28DF83F
:1065D00050301E9B082B28BF08231D9307A91F9B23
:1065E0001D9A049803F00AFC1F9A1D9B13441F93E5
:1065F0001E9A1D9BD31A1E9315AB12AA07A81D99AC
:1066000000F0ECFF1E9B002BE3D1049803F02BFB62
:1066100000BF21B05DF804FB82B00190019BDB68F4
:1066200001225A7100BF02B07047000000B583B06C
:106630004FF0FF330193FFF7F8FE0421084800F004
:1066400045FE0190019B002B03DA0649412006F02C
:106650005BFE0348FFF7E0FF00BF03B05DF804FBFB
:10666000A8190300E819030000B583B00190009158
:10667000019B1B681B6800990198984700BF03B0F5
:106680005DF804FB00B583B00190019B1B685B685B
:106690000198984700BF03B05DF804FB00B583B0D4
:1066A0000190019B1B689B680198984700BF03B04D
:1066B0005DF804FB82B001900B468DF80330019B1E
:1066C000DB689DF803201A7100BF02B0704782B0EA
:1066D0000190019BDB681B79184602B0704782B0BD
:1066E0000190019BDB6801225A7100BF02B0704724
:1066F00082B00190019BDB685B79184602B070475D
:1067000000B585B001900091154BFF229A60144BA3
:1067100000221A60124B00225A60114B0022C3F86B
:1067200018240F4B0022C3F814240D4B002283F8C9
:1067300020240C4803F0ECF90390039B002B01D0BC
:10674000039B08E0084803F017FC084A084BD31ADB
:10675000DB0802930023184605B05DF804FB00BF78
:10676000302D00202C190300481A0300A81903003B
:1067700040190300024A034BD31ADB08184670473E
:10678000A81903004019030000B587B001900B461B
:106790008DF803309DF80330002B1FD0FFF7EAFF80
:1067A00004900023059313E0059B9B000E4A1344BD
:1067B0000393039B1B881A46019B1B689A4204D1D2
:1067C000019B059A1A60002309E0059B013305939C
:1067D000059A049B9A42E7D3052300E0002318465C
:1067E00007B05DF804FB00BF982A002000B585B013
:1067F00001900B468DF803309DF8032001AB114644
:106800001846FFF7C1FF0346002B07D1019BDB00B1
:10681000054A13440393039B1B6800E000231846BA
:1068200005B05DF804FB00BF4019030084B001907F
:106830000B468DF80330019BDB00174A134402938B
:106840009DF80330013B032B1CD801A252F823F022
:106850006168020069680200716802007B680200DA
:1068600002238DF80F3011E004238DF80F300DE076
:10687000029B1B798DF80F3008E0029B5B798DF845
:106880000F3003E000238DF80F3000BF9DF80F306C
:10689000184604B0704700BF4019030084B001904F
:1068A000009100238DF80F30019B1B7803F0040347
:1068B000DBB2002B24D0019B1B78C3F30103DBB2B6
:1068C000012B02D0022B0CD017E0009B1B68019A11
:1068D0001288C2F38312D2B213449A1C009B1A602E
:1068E0000BE0009B1B68019A5288C2F3891292B296
:1068F00013449A1C009B1A6000BF01238DF80F30CF
:106900009DF80F30184604B07047000000B58BB0FA
:106910000023ADF826303E4802F005FC3D4802F069
:1069200002FC3D4B5B6804933B4B9B680693049AC7
:10693000069B134002339B00374A134404330893E9
:1069400004AB19460898FFF7A9FF0346002B09D0AE
:10695000049A069B134002339B002F4A13440433CE
:106960000893EDE700BF0023079311E0049B5A1C36
:106970000492069A1340079A920001A90A442649F4
:1069800002339B000B445B681360079B0133079342
:10699000079B012BEAD99DF80430C3F30103DBB256
:1069A000012B10D0022B1CD1BDF80A30ADF82630D7
:1069B000BDF80630C3F389139BB203339A08049BD6
:1069C0001344049313E0BDF80A30ADF82630BDF847
:1069D0000430C3F38313DBB21A46049B13440493BD
:1069E00005E00E494FF4BF7006F08EFC00BF094869
:1069F00002F0A5FB0590059B002B02D0049B064AE4
:106A00005360BDF8263018460BB05DF804FB00BF9C
:106A10004831002044310020302D0020581A030056
:106A200000B585B00021074802F0EEFA0390039B01
:106A30000293029B83F310030193019B184605B058
:106A40005DF804FB4C31002000B589B00390029141
:106A500001920093039B1B0C0793FFF7E1FF069045
:106A6000FFF788FE0246079B934204D3214940F278
:106A7000A31006F049FC069B1904009B5A1C0A9BB4
:106A80001340079A0A431C4902339B000B445A6087
:106A9000009A0A9B134002339B00174A13440433A5
:106AA0000593039B03F00703D9B2059A137861F3AA
:106AB000C5031370019B03F00F03D9B2059A138825
:106AC00061F389131380029BC3F31501059A1368C0
:106AD00061F39F231360059A1378012161F3010389
:106AE0001370059A13786FF38203137000BF09B017
:106AF0005DF804FB581A0300302D002000B58DB05E
:106B00000390029113468DF80730039B02330A93DA
:106B100001238DF8273000238DF81B300DF11B0366
:106B2000184602F0DBF9404B1A68029B1A603E4B94
:106B30009A683D4B59683C4B1B68CB1A1344013390
:106B40000B9314E00121394802F0BDFAFFF7DEFE95
:106B500007900799354802F0B6FA334B9A68324BE2
:106B60005968314B1B68CB1A134401330B930A9AB3
:106B70000B9B9A42E6D89DF82730002B48D0002383
:106B800005939DF80730002B17D09DF81430012293
:106B900062F301038DF814309DF8143043F00403C0
:106BA0008DF81430039B03F00F03DAB2BDF81430F4
:106BB00062F38913ADF8143016E09DF81430022208
:106BC00062F301038DF814309DF8143043F0040390
:106BD0008DF81430039BC3F309039AB2BDF8163045
:106BE00062F38F13ADF816300F4B1A680E4B9B688B
:106BF000134002339B000C4A134404330893059A54
:106C0000089B1A60084B1A680A9B1344064A1360D3
:106C10009DF81B30184602F077F99DF8273018468A
:106C20000DB05DF804FB00BF302D00204C3100207A
:106C300000B58BB005900491039202931F4B9B68A3
:106C4000079306AB012219460298FFF757FF034648
:106C5000002B24D0069B023309930023089311E0F4
:106C6000089B9B00039A1A44099B591C0991079998
:106C70000B401268114902339B000B445A60089B79
:106C800001330893089A029B9A42E9D3069A079B1C
:106C900000931346029A04990598FFF7D5FE074B17
:106CA00093F82034002B05D000BF00F007F903460D
:106CB000002BFAD100BF0BB05DF804FB302D002093
:106CC00000B583B001900091002300220099019843
:106CD000FFF7AEFF00BF03B05DF804FB00B587B05F
:106CE000039002910192019B059305AA0123029949
:106CF0000398FFF79DFF00BF07B05DF804FB00B5E8
:106D000087B00390029101920093019B0493009B32
:106D1000059304AA022302990398FFF789FF00BF95
:106D200007B05DF804FB00B58BB0039002910192AF
:106D30000093019B0593009B06930C9B07930D9B6F
:106D400008930E9B099305AA052302990398FFF760
:106D50006FFF00BF0BB05DF804FB000000B58DB005
:106D6000039002911346ADF806304B4B9B680B9392
:106D7000BDF8063003339B0805A900221846FFF72B
:106D8000BDFE0346002B78D0059B0A93059B02337A
:106D90000593414B9A6805990B9B0B40D31A01331D
:106DA0009B000993BDF80630099A9A420ED3059AC2
:106DB0000B9B134002339B00374A13440433BDF846
:106DC0000620029918460AF03FF917E0059A0B9B36
:106DD000134002339B00304A13440433099A02994A
:106DE00018460AF031F9029A099BD118BDF806201D
:106DF000099BD31A1A4629480AF026F9039B1B0C53
:106E00000893FFF70DFE0790079B19040A9B5A1C75
:106E10000B9B1340089A0A431F4902339B000B4403
:106E20005A600A9A0B9B134002339B001A4A134480
:106E300004330693039B03F00703D9B2069A137831
:106E400061F3C5031370069A13886FF38F131380D1
:106E5000BDF80630C3F3090399B2069A538861F36B
:106E60008F135380069A1378022161F30103137084
:106E7000069A13786FF382031370074B93F820344C
:106E8000002B05D000BF00F019F80346002BFAD103
:106E900000BF0DB05DF804FB302D00203C2D00201C
:106EA000054B5A68044B1B689A420CBF0123002310
:106EB000DBB21846704700BF302D002000B599B0F6
:106EC000FFF7EEFF0346002B01D00023BEE19B4BF2
:106ED0000022C3F81824BFF34F8F00BF974B5B68A5
:106EE0000493964B9B681093049A109B13400233B3
:106EF0009B00924A134404331193002317930023F9
:106F0000169300230F9304AB19461198FFF7C6FCA4
:106F10000346002B19D0894BD3F81834002B14D119
:106F2000864B1A68049B9A4205D8844B1B68834A97
:106F3000536000238AE1049A109B134002339B00A4
:106F40007E4A134404331193DDE70023159311E0C7
:106F5000049B5A1C0492109A1340159A920001A99E
:106F60000A44764902339B000B445B681360159B0F
:106F700001331593159B012BEAD99DF8043003F0DA
:106F80000303DBB2022B40F09C80BDF80630C3F354
:106F900089139BB20D93BDF80630C3F389139BB2DE
:106FA000502B28BF50239BB20C930C9BC3F30903B7
:106FB0009AB2BDF8063062F38F13ADF806300C9B21
:106FC00008330B939DF80430C3F3C203DBB20F9375
:106FD0000B995B4802F0A7FD1790179B002B00F060
:106FE000D180179802F030FE01A9169B082217984D
:106FF00002F0E6FE169B08331693049BDA43109BBF
:10700000134001339B000A930C9A0A9B9A4242D97F
:107010000A9B002B08D0049A109B134002339B005C
:10702000464A1344043300E0464B08930A9B002B66
:1070300002D00A9BDBB201E00C9BDBB28DF81F3063
:107040000A9B002B01D03F4B00E0002306930A9BD4
:10705000002B06D00C9BDAB20A9BDBB2D31ADBB250
:1070600000E000238DF817309DF81F20169B08992B
:10707000179802F0A5FE9DF81F30169A1344169338
:10708000069B002B16D09DF81720169B0699179883
:1070900002F096FE0EE0049A109B134002339B0010
:1070A000264A134404330993169B0C9A099917989E
:1070B00002F086FE0D9B03339A08049B134404934D
:1070C00060E09DF8043003F00303DBB2012B59D1DB
:1070D000BDF80430C3F38313DBB2062B28BF0623AD
:1070E000DAB2BDF8043062F38913ADF80430BDF8AC
:1070F0000430C3F38313DBB202330E939DF80430E4
:10710000C3F3C203DBB20F930E9B9B0019460C48DE
:1071100002F009FD1790179B002B33D0179802F04F
:1071200093FD01A9169B0822179802F049FE169BB1
:1071300008331693002315931BE000BF302D002069
:107140002C1903003C2D0020049B5A1C0492109A19
:10715000134002339B003F4A1344191D169B04221F
:10716000179802F02DFE169B04331693159B0133DE
:107170001593BDF80430C3F38313DBB21A46159B95
:107180009342E1D3179B002B40D0324BD3F81034FD
:107190001493304BD3F81834002B1BD0179802F0FF
:1071A00062FD4DE000238DF84F301498FFF7A0FAF0
:1071B0000346002B02D001238DF84F309DF84F304D
:1071C000002B03D017991498FFF74EFA149BDB6835
:1071D0001B681493149B002BE4D1179802F043FD15
:1071E00000238DF803300DF10303184601F076FEFD
:1071F000184BD3F81834002B02D1049B154A536066
:107200009DF80330184601F07FFE19E0114BD3F8CA
:107210001034129306E01298FFF740FA129BDB68D5
:107220001B681293129B002BF5D10B4A0B4BD31A00
:10723000DB081B0443F0020309491846FFF740FD31
:10724000FFF72EFE034683F00103DBB2184619B0A8
:107250005DF804FB302D002068190300401903007D
:10726000B01A030000B585B00023039323E0164B4A
:10727000D3F81034029301238DF807300FE0029801
:10728000FFF725FA03461A46039B934203D10023D6
:107290008DF8073006E0029BDB681B680293029BB7
:1072A000002BECD19DF80730002B01D0039B07E0A9
:1072B000039B01330393039B092BD8DD4FF0FF336E
:1072C000184605B05DF804FB302D002000B585B0F0
:1072D00001900B468DF80330FFF7C4FF0390039B2A
:1072E000B3F1FF3F01D1039B22E0039BDBB21946C0
:1072F0000198FFF7DFF9104BD3F81034002B08D1B9
:107300000D4A019BC2F81034019BDB6800221A6011
:107310000DE0094BD3F81034DA68019BDB68126882
:107320001A60054BD3F81034DB68019A1A60039B8E
:10733000184605B05DF804FB302D002000B583B081
:107340000D4BD3F8103401930B4B012283F820240A
:1073500009E00198FFF7C3F90198FFF793F9019B42
:10736000DB681B680193019B002BF2D100BF00BFBB
:1073700003B05DF804FB00BF302D002082B0019007
:10738000009100BF02B0704710B584B00390029125
:10739000039BDB88002B0AD0039BDB881A461F4B1C
:1073A000009313461E4A1F49029802F005F8039BFA
:1073B0001B7A052B2ED0039B5B7A002B12D0039BEC
:1073C0009B881A46039B1B7A19461046FFF72EFA34
:1073D00003461A46144B53F822301A4613490298B2
:1073E00001F0EAFF039B1B6819460298FFF7C6FFEE
:1073F000039B1B7A1A460E4B53F82240039B9B8833
:1074000000211846FFF7F2F903462246094902987F
:1074100001F0D2FF00BF04B010BD00BFE41A0300AA
:10742000F41A03002C1B0300B42A0020441B0300A1
:10743000A02A0020481B030000B585B003900291EC
:1074400013468DF80730039B1B7A052B0FD0039B47
:107450005B7A002B06D00D4B1B681A460C4902982C
:1074600001F0AAFF0B49029801F0A6FF07E09DF882
:107470000730002B03D00749029801F09DFF0298C6
:1074800001F078FF00BF05B05DF804FBB42A0020CE
:10749000441B0300541B030030B58BB007900691CA
:1074A000059204930E9B1B7B8DF827300E9B0022C8
:1074B0001A730E990498FFF767FF059B062B7FD878
:1074C00001A252F823F000BFE5740200EF7402003D
:1074D000FF74020013750200317502005975020035
:1074E0008975020007990E9801F066FF69E0069B16
:1074F0001B681A4607990E9801F05EFF61E0069B33
:107500001A68069B04331B6807990E9801F054FF14
:1075100057E0069B1A68069B04331968069B0833DC
:107520001B6800930B4607990E9801F045FF48E051
:10753000069B1968069B04331868069B08331B6872
:10754000069A0C3212680192009303460A46079984
:107550000E9801F031FF34E0069B1868069B043357
:107560001C68069B08331B68069A0C321268069941
:10757000103109680291019200932346024607994F
:107580000E9801F019FF1CE0069B1C68069B043353
:107590001D68069B08331B68069A0C321268069910
:1075A0001031096806981430006803900291019226
:1075B00000932B46224607990E9801F0FDFE00E04D
:1075C00000BF00220E990498FFF736FF0E9B9DF82E
:1075D00027201A7300BF0BB030BD00BF00B587B0C5
:1075E0000390029101920093029B082B60D8009BAC
:1075F0001B7B8DF81330009B00221A7300990198B1
:10760000FFF7C2FE0023059314E0059A029B9A42FD
:1076100009D2039A059B13441B781A462649009801
:1076200001F0CAFE03E02549009801F0C5FE059B64
:1076300001330593059B072BE7D92149009801F0F9
:10764000BBFE0023059326E0059A029B9A421BD2BB
:10765000039A059B13441B788DF812309DF8123065
:107660007E2B0AD89DF81230184609F081FC03469B
:10767000002B02D09DF8123000E02E231A4611494B
:10768000009801F099FE03E00F49009801F094FE84
:10769000059B01330593059B072BD5D90122009942
:1076A0000198FFF7C9FE009B9DF813201A7300E0B4
:1076B00000BF07B05DF804FB581B0300601B03000C
:1076C000641B0300681B03006C1B03002DE9F04FD3
:1076D00097B00D9000238DF85730B8E0624B1A68D0
:1076E0009DF85730DB0013441493149B1B781C4601
:1076F0004FF001024FF00003A4F12001C4F120007B
:1077000003FA04FB02FA01F14BEA010B22FA00F042
:107710004BEA000B02FA04FACDE912AB534BD3E962
:107720000001DDE9122300EA020400940B400193FA
:10773000DDE900120B46134300F08480DDE91223DB
:10774000D1430291DB430393484BD3E90023DDE9A6
:10775000024521461140049129460B400593434BB5
:10776000DDE90412C3E90012149B1B78184603F0EC
:1077700097FE03468DF84730149B1B781C464FF04C
:1077800001024FF00003A4F12001C4F1200003FA2C
:1077900004F902FA01F149EA010922FA00F049EA82
:1077A000000902FA04F8324BD3E9002308EA020187
:1077B000069109EA030307939DF8473000220893D6
:1077C0000992149B1B781946A1F12003C1F12002F4
:1077D000DDE90845284600FA01F7204600FA03F3E0
:1077E0001F43234623FA02F21743234603FA01F606
:1077F000DDE906120B46BA4208BFB34222D19DF81A
:107800004720149B5B78012B0CBF01230023DBB2C4
:107810009A420CBF01230023DBB2DBB200220A93A1
:107820000B92DDE90A34CDE90E34149B5B68002B22
:1078300008D0149B5C68149B1A789DF83830194660
:107840001046A0479DF8573001338DF85730094B4B
:107850001A789DF857309342FFF440AF00BF00BF45
:1078600017B0BDE8F08F00BF5431002088310020F0
:1078700080310020583100202DE9704F90B00B90DE
:107880000B468DF82B304FF001024FF000030B9E9A
:10789000A6F12001C6F1200003FA06F502FA01F173
:1078A0000D4322FA00F0054302FA06F4CDE90E4535
:1078B000384B184601F066F80D900D9B002B65D1F2
:1078C000354BD3E90001DDE90E2300EA0204009400
:1078D0000B400193DDE900120B46134341D10B9895
:1078E00003F0DEFD0346002B0FD02C4BD3E9000143
:1078F000DDE90E2340EA020402940B430393274B75
:10790000DDE90212C3E9001213E0DDE90E236FEA9C
:10791000020A6FEA030B214BD3E900230AEA0201B2
:1079200004910BEA030305931C4BDDE90412C3E940
:107930000012194BD3E90001DDE90E2340EA0204ED
:1079400006940B430793144BDDE90612C3E90012BA
:107950001048134B1B680022194600F0E1FF0D9000
:1079600015E0DDE90E236FEA02086FEA03090A4B0E
:10797000D3E9002308EA0201089109EA0303099305
:10798000054BDDE90812C3E9001200E000BF10B0AA
:10799000BDE8708F603100208831002080310020E8
:1079A0005C31002000B58BB003900B4601928DF83E
:1079B0000B30019B042B01D807235AE003F0EAFCAB
:1079C000034683F00103DBB2002B09D003F090FCE7
:1079D0000990099B0893089B002B01D0089B48E065
:1079E000264A039B1360264A9DF80B301370254AE4
:1079F000019B136024494FF000024FF00003C1E9DE
:107A0000002322494FF000024FF00003C1E9002398
:107A100022E09DF80B30DB00039A1344079305AB7B
:107A200000210A461A800A469A7003238DF8143002
:107A3000079B9B788DF81530079B1B78184605AB84
:107A4000134A194603F0B2FC0990099B0693069B62
:107A5000002B01D0069B0CE09DF80B305A1E8DF8D0
:107A60000B20002BD5D10B4A00210B4800F028FF3A
:107A7000034618460BB05DF804FB00BF54310020EC
:107A8000583100205C3100208031002088310020F6
:107A900079780200CD760200701B030086B0039057
:107AA0000291019201238DF817309DF81730214A79
:107AB000039B13601F4A029B53601E4A019B936005
:107AC000039B44F20102934213D0039B44F202024F
:107AD000934221D1019B174AD360164BDB681B8868
:107AE0001A46144B9A61134BDB685B68114AD361E9
:107AF00012E0019B0F4A13610E4B1B699B680D4AF4
:107B000053610C4B1B691B680A4A9361094B1B6943
:107B10005B68084AD36100BF72B600BF00BF9DF822
:107B20001730DBB2002BFAD162B600BF00BF06B03F
:107B3000704700BF9031002000B583B002900091E3
:107B4000019244F2010071466A4600F003F803B066
:107B500000BD00BF30B58BB007900691059272B69C
:107B600000BFFFF7EBFB00BFFFF7A8F90346002BB0
:107B7000FAD1079B44F2020293422FD0079B44F2B2
:107B80000202934269D8079B44F20102934237D024
:107B9000079B44F2010293425FD8079B012B05D05B
:107BA000079B41F2010293420CD056E0394A3A4B0E
:107BB000D31ADB081B0443F0010338491846FFF7CA
:107BC0007FF857E0334A344BD31ADB081B0443F0E9
:107BD000010333491846FFF773F84BE0059B0993FF
:107BE0002C4A2D4BD31ADB081B0443F00100099BE0
:107BF0005B681A46099B1B882A49FFF780F839E021
:107C0000059B0893234A244BD31ADB081B0443F03B
:107C10000104089B9D68089B9B68184602F026FAA1
:107C200003461846089B5B681946089B1B68069A22
:107C300002920193009103462A461B492046FFF712
:107C400072F8144A144BD31ADB081B0443F00103E7
:107C500016491846FFF734F80CE00E4A0E4BD31ABB
:107C6000DB081B0443F00103069A11491846FFF78D
:107C700035F800BF0F4B1B6803F00103002B00D049
:107C800000BE059A06990798FFF708FF00BF0BB0E2
:107C900030BD00BF6819030040190300741B0300C6
:107CA000941B0300B81B0300D41B0300FC1B030040
:107CB000101C0300F0ED00E084B00190019B9B6874
:107CC0000393019BDA68039BD31A184604B07047EC
:107CD00082B001900B468DF80330019B1A68019B1E
:107CE000DB68019989880B4013449DF803201A70C2
:107CF000019BDB685A1C019BDA6000BF02B0704731
:107D000084B003900B460192ADF80A30039B1A68C9
:107D1000039B9968BDF80A300B44039989880B408E
:107D200013441A78019B1A7000BF04B0704700B565
:107D300083B001900091009A00210198FFF7E0FFC5
:107D4000019B9B685A1C019B9A6000BF03B05DF8C1
:107D500004FB84B0039002911346ADF80630029BF9
:107D6000002B01D10E231DE0BDF80630002B07D0FB
:107D7000BDF806305A1EBDF806301340002B01D066
:107D800009230FE0039B029A1A60BDF80630013BFD
:107D90009AB2039B9A80039B00229A60039B002265
:107DA000DA600023184604B0704700B583B0019034
:107DB0000B468DF803300198FFF77EFF0246019BCA
:107DC0009B889A4207D89DF8033019460198FFF71F
:107DD0007FFF002300E00423184603B05DF804FB96
:107DE00000B583B0019000910198FFF765FF03464D
:107DF000002B05D000990198FFF799FF002300E0C0
:107E00000523184603B05DF804FB000082B003466A
:107E10008DF807309DF8073003F01F0205499DF9E2
:107E200007305B09012000FA02F241F8232000BF6D
:107E300002B0704700E100E082B003468DF80730E1
:107E40009DF8073003F01F0206499DF907305B09D2
:107E5000012000FA02F2203341F8232000BF02B0D3
:107E6000704700BF00E100E082B003468DF80730A4
:107E70009DF8073003F01F0206499DF907305B09A2
:107E8000012000FA02F2403341F8232000BF02B083
:107E9000704700BF00E100E082B003468DF8073074
:107EA0009DF8073003F01F0206499DF907305B0972
:107EB000012000FA02F2603341F8232000BF02B033
:107EC000704700BF00E100E082B0034600918DF8EA
:107ED00007309DF90730002B0CDA009BDAB20C4911
:107EE0009DF8073003F00F03043B5201D2B20B445C
:107EF0001A7609E0009BDAB206499DF90730520173
:107F0000D2B20B4483F8002300BF02B0704700BF19
:107F100000ED00E000E100E000B585B00190019BBC
:107F2000002B0AD0074B43F001030393019B9B01F5
:107F30000293039B0298984700E000BF05B05DF8EC
:107F400004FB00BF301C030000B583B00190064A5B
:107F5000019BC2F8083506211120FFF7B5FF00BFCD
:107F600003B05DF804FB00BF0010014008B50D4BE5
:107F70004FF48032C3F844230A4B4FF48032C3F8E5
:107F800004231120FFF788FF1120FFF73FFF054B67
:107F900001221A602F20FFF7BFFF034B01221A7046
:107FA00000BF08BD00100140CE32002008B51120EE
:107FB000FFF742FF0E4B4FF48032C3F848230C4BBF
:107FC0004FF48032C3F80823094B01225A602F2056
:107FD000FFF7A2FF064B01229A60064B00221A60AF
:107FE0002F20FFF799FF044B00221A7000BF08BD35
:107FF00000100140C0320020CE320020024BD3F8E6
:1080000004351846704700BF0010014082B001904F
:108010000091019A009BD31A23F07F43184602B0C7
:108020007047000082B00190034A019BC2F84035BE
:1080300000BF02B0704700BF0010014086B0019041
:10804000284B1B68002B03D1264A019B136045E097
:10805000019B1A68234B1B681B689A4210D8214B5E
:108060001B681968019B1A681E4B1B688A1A1A60E4
:108070001C4B1A68019BDA611A4A019B13602DE0C0
:10808000019B1B680393174B1B680593154B1B68DB
:10809000049309E0049B1B68039AD31A0393049B7F
:1080A0000593049BDB690493049B002B04D0049B81
:1080B0001B68039A9A42EDD8049B002B05D0049BC1
:1080C0001A68039BD21A049B1A60019B039A1A60D8
:1080D000019B049ADA61059B019ADA6100BF06B040
:1080E000704700BFBC32002000B587B001902A4B1A
:1080F0001B680393284B1B680593059B049308E0BA
:10810000049A019B9A4208D0049B0593049BDB6967
:108110000493049B002BF3D100E000BF049B002BD1
:1081200001D1002333E0059A049B9A4214D11A4BE3
:108130001B68DB69184A1360174B1B68002B0BD1B7
:10814000164B01229A60164B00221A60154B012231
:108150001A702F20FFF7E0FE049B1B680293049B1C
:10816000DA69059BDA61059BDB690493049B002BAC
:1081700005D0049B1A68029B1A44049B1A60064BA4
:108180001B68039A9A4214BF01230023DBB21846EE
:1081900007B05DF804FB00BFBC32002000100140B6
:1081A000C0320020CF32002008B51120FFF75CFE5E
:1081B00000BF08BD08B51420FFF756FE00BF08BD7C
:1081C00000B583B00190019B5B69019A92691046EA
:1081D000984700BF03B05DF804FB000000B585B010
:1081E0002B4B1B68002B4ED000230193FFF706FF9B
:1081F0000246284B1B6819461046FFF707FF0290FE
:10820000234B1B6803931DE0039B1B68029A9A4251
:108210001CD3039B1B68029AD31A0293039B1B680F
:10822000019A13440193039B0093039BDB6903931F
:10823000009B1B7C002B05D0009B00221A74009829
:10824000FFF7BEFF039B002BDED100E000BF124B07
:108250001A78124B1B789A420CD1104B1B780133C1
:10826000DAB20E4B1A700D4B1B78022B02D10B4B5E
:1082700000221A70094B1B781946094A019B42F8E3
:108280002130FFF797FF00BF05B05DF804FB00BF8A
:10829000BC320020C0320020CC320020CD32002081
:1082A000C432002082B00190184B1A78184B1B780A
:1082B0009A4223D0154B1B780133DAB2134B1A7054
:1082C000124B1B78022B02D1104B00221A700F4B5D
:1082D0001B781A460F4B53F82220019B1A60019B12
:1082E0001A680D4B1B6813440B4A13600A4B1B683A
:1082F00023F07F43084A1360012303E0019B00221F
:108300001A600023184602B0704700BFCC3200202C
:10831000CD320020C4320020C032002088B003904B
:10832000029101920023079338E0204B1B680693CB
:10833000069B1B68039A9A4206D2069B1A68039B07
:10834000D21A069B1A602EE0069B1B68039AD31A6A
:108350000393069B1B68079A13440793069B00220E
:108360001A60124B1B680593069BDB690F4A13606A
:10837000069BDB68002B11D0029A079B134423F065
:108380007F42069B5A60069BDA68069B9A60019BB7
:108390001A68069BDA61019B059A1A60034B1B68F9
:1083A000002BC2D100BF00BF08B07047BC32002014
:1083B00000B589B0019000238DF81F30664B1B6813
:1083C0000593AAE0019B002B05D0019B0693069B19
:1083D000DB69019361E0614B1B781A4613465B0031
:1083E0001344DB005D4A1344043304935B4B1B7856
:1083F0000133DAB2594B1A70584B1A78574B9B78A5
:108400009A4202D1554B00221A70049B5B68069376
:10841000049B1B78032B1ED0032B7EDC012B1FD06B
:10842000022B7AD1049B5B681846FFF75DFE03467A
:10843000002B02D001238DF81F30069B00221A74F6
:108440006BE0454B1B680393039B00221A74039B4C
:10845000DB69414A1360404B1B68002BF1D15CE0A3
:1084600000BF069B1B7C002B00D056E0049B9A6843
:10847000069B5A60049BDA68069B9A60049B1A6903
:10848000069BDA60049B5A69069B9A61344B1B7801
:10849000002B02D0069B00225A60069B5A68314B83
:1084A0001B68D31A23F07F432F4A93420ED8069BB2
:1084B0005B682C4A126811461846FFF7A7FD024672
:1084C000069B9B681A44069B1A6017E0254B1A68A6
:1084D000069B5B6819461046FFF798FD0290069BC5
:1084E0009B68029A9A4206D2069B9A68029BD21A0D
:1084F000069B1A6002E0069B00221A60069B00227F
:108500005A60069B00229A60069B01221A74069B01
:108510000022DA610698FFF791FD019B002B7FF4A2
:1085200051AF0E4B1A780D4B5B789A427FF44AAFED
:108530009DF81F30002B04D1074B1B68059A9A4207
:1085400001D0012300E0002303F00103DBB2184651
:1085500009B05DF804FB00BFBC320020B031002040
:10856000CF320020C0320020FEFF7F0010B588B05F
:108570000190274B1B68002B44D0254B1B681B68C0
:108580000793FFF73BFD0690224B1B680593059967
:108590000698FFF73BFD0346033304931E4B1B78FD
:1085A00083F00103DBB2002B01D0FFF7DFFC049A5C
:1085B000079B934238BF1346059A13440593059BC6
:1085C00023F07F4305930598FFF72CFDFFF716FD79
:1085D000039006990398FFF719FD0346DC1C0699E2
:1085E0000598FFF713FD03469C420DD9FFF706FDE2
:1085F00003461846FFF716FD2F20FFF78DFCFFF707
:10860000D3FD01E0FFF7D2FC00BF08B010BD00BFF2
:10861000BC320020C0320020CE32002000B587B02E
:108620000023019300238DF81730194B1B68049326
:10863000184B1B6803936B461846FFF733FE03463F
:108640008DF80B309DF80B30002B08D0009B01AA51
:1086500004991846FFF762FE01238DF81730019B3D
:108660001846FFF7A5FE0346002B02D001238DF824
:1086700017309DF81730002B02D00398FFF776FFD4
:10868000054B00221A7000BF07B05DF804FB00BF65
:10869000C0320020BC320020CF32002082B003461E
:1086A0008DF80730034A9DF80730537000BF02B0C1
:1086B000704700BFB031002084B00190144B5B784C
:1086C00001338DF80F30124B9B789DF80F209A42A2
:1086D00002D100238DF80F300D4B1B789DF80F2031
:1086E0009A4201D100230FE0019B9DF80F201A70E0
:1086F000074B5B781A4613465B001344DB00044AC1
:10870000134404330293029B184604B0704700BF21
:10871000B031002000B589B003900291019200931E
:108720000023079300238DF816300DF11603184629
:1087300000F0D4FB0DF117031846FFF7BDFF0690BC
:10874000069B002B02D10423079318E0069B01220D
:108750001A70069B039A5A60FFF750FC0246069B6C
:108760009A60069B029ADA60069B019A1A61069B40
:10877000009A5A619DF817301846FFF78FFF9DF851
:108780001630184600F0C0FB079B002B01D1FFF705
:1087900011FD079B184609B05DF804FB00B587B0D2
:1087A00001900B468DF803300023059300238DF8CC
:1087B0000E300DF10E03184600F090FB0DF10F0383
:1087C0001846FFF779FF0490049B002B02D1042385
:1087D00005930BE0049B9DF803201A70049B019AFB
:1087E0005A609DF80F301846FFF758FF9DF80E307D
:1087F000184600F089FB059B002B01D1FFF7DAFC3E
:10880000059B184607B05DF804FB000008B50E4B49
:108810000022C3F840210C4B0022C3F844210A4B2C
:108820000022C3F84821084B0022C3F84C21064B14
:108830000022C3F80021044B0022C3F80421FFF7F3
:10884000CDFC00BF08BD00BF0010014008B5FFF718
:10885000E5FE00BF08BD000008B5FFF7A7FB134BFE
:1088600000221A70114B00225A70104B0B229A7082
:108870000F4B00221A600F4B00221A700E4B002281
:108880001A701420FFF708FB06211420FFF71CFBC9
:108890001420FFF7BBFA0020FFF756FBFFF7AEFBF3
:1088A0000346064A13600023184608BDB031002075
:1088B000BC320020CC320020CD320020C03200205B
:1088C00086B003900B4601928DF80B30134B9B78CA
:1088D000002B01D108231EE0019B002B01D10723AF
:1088E00019E0039B002B01D1072314E0039B1B68B5
:1088F0001B7C002B01D008230DE0039B1B68059314
:10890000059B00221A74059B9DF80B205A74059B49
:10891000019A5A610023184606B07047B031002012
:1089200000B587B0039002910192039B0593144B0D
:108930009B78002B01D108231EE0039B002B01D163
:10894000082319E0029B042B01D8072314E0059BA0
:108950005B69002B01D108230EE0059B5B7C012B9A
:1089600001D1029B00E000230493019B049A029929
:108970000598FFF7CFFE0346184607B05DF804FBE5
:10898000B031002000B585B00190019B03930D4BE1
:108990009B78002B01D1082310E0019B002B03D012
:1089A000039B5B69002B01D1082307E0039B002296
:1089B0001A7402210398FFF7F1FE0346184605B02A
:1089C0005DF804FBB031002000B587B00390029140
:1089D00013468DF8073000230593039B1B781A4636
:1089E000114B9B5C002B09D0039B04339DF807209F
:1089F0000299184604F09EF805900FE0039B1B783F
:108A00001A46094B9B5C002B08D1039B0C339DF845
:108A100007200299184603F05BFA0590059B18465B
:108A200007B05DF804FB00BF3C33002000B585B003
:108A3000019000238DF80F30019B1B781A46114BD3
:108A40009B5C002B08D0019B0433184604F01CF9F2
:108A500003468DF80F300EE0019B1B781A46094B38
:108A60009B5C002B07D1019B0C33184603F0B8FA2E
:108A700003468DF80F309DF80F30184605B05DF8AD
:108A800004FB00BF3C33002000B587B00390029187
:108A900013468DF8073000230593039B1B781A4675
:108AA000114B9B5C002B09D0039B04339DF80720DE
:108AB0000299184604F000F905900FE0039B1B781B
:108AC0001A46094B9B5C002B08D1039B0C339DF885
:108AD00007200299184603F0DBFA0590059B18461B
:108AE00007B05DF804FB00BF3C33002084B0019068
:108AF000019B9B680393019BDA68039BD31A18467A
:108B000004B0704700B587B001900091019B1B78BD
:108B1000022B3BD0022B60DC002B48D0012B5CD118
:108B2000019B5B681B7819462E48FFF73EF90590BC
:108B3000059B002B0AD001238DF80C30059B049374
:108B4000294B1B6803AA104698470DE02548FFF7FC
:108B5000CDFF0346002B07D000238DF80C30224BAD
:108B60001B6803AA104698471E48FFF7BFFF03463D
:108B70001C4A9288934205D801221C491C48FFF7E1
:108B800083FF2BE01B4B01221A7027E002238DF894
:108B90000C30019BDB680493012214491448FFF751
:108BA00073FF114B1B6803AA1046984716E0124941
:108BB0001248FFF715F90346002B05D101220E4993
:108BC0000B48FFF701FF09E003238DF80C30064B3B
:108BD0001B6803AA1046984700E000BF00BF07B01B
:108BE0005DF804FBDC320020D0320020D8320020B7
:108BF000D82A0020D9320020D4320020EC320020C4
:108C000030B591B00390029101928DF803303C4A47
:108C1000019B1360029B002B01D107236DE0029B97
:108C20001968029B5B689BB21A463648FFF791F8B9
:108C30000F900F9B0E930E9B002B01D00E9B5CE0C0
:108C4000029B9968029BDB689BB21A462E48FFF78D
:108C500080F80F900F9B0D930D9B002B01D00D9B67
:108C60004BE02A4B04AC1D460FCD0FC495E80F0016
:108C700084E80F00039B5B690A93039B1B7C002B1A
:108C800014BF01230023DBB28DF824309DF803309C
:108C90008DF82C30039B5B7C002B01D00E2300E071
:108CA00000238DF82530039BDB680693039B9B68AC
:108CB0000793039B1B680593039B5B68049304ABBA
:108CC000134A1946134801F0B3FD0F900F9B0C9304
:108CD0000C9B002B01D00C9B0FE00F4B00221A7055
:108CE000039B1B68B3F1FF3F06D001220B490948E3
:108CF000FFF7CAFE034600E00023184611B030BD5E
:108D0000D0320020DC320020EC320020381C03007E
:108D1000058B0200D82A0020D9320020D83200204A
:108D200000B587B00190019B002B03D11449C220EC
:108D300004F0EAFA134B1B788DF8173001991248AA
:108D4000FFF74EF804909DF81730002B12D00D4B12
:108D500000221A7001220D490D48FFF795FE03907D
:108D6000039B0293029B002B04D0054ACE2102985C
:108D7000FEF7E2FE049B184607B05DF804FB00BF57
:108D8000581C0300D9320020DC320020D8320020E9
:108D9000D82A002000B585B003468DF807309DF82D
:108DA000073019461048FFF700F80390039B002B8B
:108DB00015D10E48FFF73AFE034683F00103DBB2FC
:108DC000002B0CD00A490848FFF70AF80346002B8D
:108DD00005D1012206490548FFF7F6FD0390039BE4
:108DE000184605B05DF804FBEC320020D82A0020BC
:108DF000D432002082B0EFF310830093009B0193E4
:108E000072B600BF019B184602B0704762B600BF41
:108E100000BF704700B585B00190FFF7EBFF0390EE
:108E2000164B9B68002B1BD1144B01229A60144BEC
:108E3000D3F88020134B1340104A1360104B114A93
:108E4000C3F880200E4BD3F884300C4A53600C4B8F
:108E50004FF0FF32C3F88420019B00221A7002E019
:108E6000019B01221A70039B002B01D1FFF7CEFF5B
:108E70000023184605B05DF804FB00BFFC3200205B
:108E800000E100E0FC06FFBD00B585B003468DF8AB
:108E90000730104B9B68002B16D09DF80730002B35
:108EA00012D1FFF7A7FF03900B4A0A4B1B68136010
:108EB000094A084B5B685360064B00229A60039B8B
:108EC000002B01D1FFF7A2FF0023184605B05DF883
:108ED00004FB00BFFC32002000E100E000B583B0DD
:108EE000019000F02BF80346012B03D005494320E5
:108EF00004F00AFA0198FFF78DFF00BF03B05DF898
:108F000004FB00BFAC1C030000B583B003468DF822
:108F1000073000F013F80346012B03D00649512017
:108F200004F0F2F99DF807301846FFF7ADFF00BFD7
:108F300003B05DF804FB00BFAC1C030084B0EFF38A
:108F400005830193019BC3F308030393039B002B49
:108F50000DD1EFF314830093009B0293029B03F067
:108F60000103002B0CBF01230023DBB200E001232F
:108F7000184604B0704700B585B001900091009B81
:108F80005B099B00019A1A44009B03F01F03012117
:108F900001FA03F31946104600F04DF8039000BFA4
:108FA00005B05DF804FB00B585B001900091009B11
:108FB0005B099B00019A1A44009B03F01F030121E7
:108FC00001FA03F3DB431946104600F064F80390FE
:108FD00000BF05B05DF804FB82B001900091009BDA
:108FE0005B099B00019A13441A68009B03F01F035E
:108FF00022FA03F303F00103002B14BF0123002323
:10900000DBB2184602B0704710B487B001900091EF
:10901000019B009A53E8004F104643E8000191F08D
:10902000000FF7D1059404900391059B184607B0F3
:109030005DF8044B704710B487B001900091019B1C
:10904000009A53E8004F44EA020043E8000191F01F
:10905000000FF6D1059404900391049B184607B0C5
:109060005DF8044B704710B487B001900091019BEC
:10907000009A53E8004F04EA020043E8000191F02F
:10908000000FF6D1059404900391059B184607B094
:109090005DF8044B704710B487B001900091019BBC
:1090A000009A53E8004F04EA020043E8000191F0FF
:1090B000000FF6D1059404900391049B184607B065
:1090C0005DF8044B704710B487B001900091019B8C
:1090D000009A53E8004F04EB020043E8000191F0CE
:1090E000000FF6D1059404900391049B184607B035
:1090F0005DF8044B704710B487B001900091019B5C
:10910000009A53E8004FA4EB020043E8000191F0FD
:10911000000FF6D1059404900391049B184607B004
:109120005DF8044B704700B583B0019001210198B0
:10913000FFF781FF0346184603B05DF804FB00B556
:1091400083B0019000210198FFF78DFF0346184678
:1091500003B05DF804FB000000B583B001900B463E
:109160008DF80330019B002B03D10849E82004F05F
:10917000CBF8019BDA689DF803300199098A01FB5D
:1091800003F31344184603B05DF804FB041D030009
:1091900000B583B001900091019B002B03D10849D9
:1091A000F52004F0B1F8009B019AD2689B1A019A4D
:1091B000128AB3FBF2F3DBB2184603B05DF804FB8E
:1091C000041D030000B585B00190019B002B01D167
:1091D0000E234CE0019B1B68002B03D12649FF2086
:1091E00004F092F8019B5B68002B04D122494FF4F4
:1091F000807004F089F8019B9B68002B04D11E4904
:1092000040F2011004F080F8019BDB68002B04D1D0
:1092100019494FF4817004F077F8019B1B8A002BE9
:1092200004D1154940F2031004F06EF8019B9A68CE
:10923000019B5B68D31A8DF80F30019B1B68019A64
:1092400052681A6007E0019B1A681368591C116084
:109250009DF80F201A709DF80F305A1E8DF80F20C0
:10926000002BF0D1019B1B6800221A7100231846C5
:1092700005B05DF804FB00BF041D030000B585B018
:109280000190019B002B04D11F494FF4927004F010
:109290003BF80023039300238DF80A300DF10A03F5
:1092A0001846FFF71BFE019B1B681A68019B5B6851
:1092B0009A421FD9019B1B681A68013A1A601B6801
:1092C0001B7819460198FFF747FF0390019B9A68A6
:1092D000019B1B681B68D31A8DF80B30019B1B6820
:1092E0001B799DF80B209A4204D9019B1B689DF8BD
:1092F0000B201A719DF80A301846FFF705FE039BF4
:10930000184605B05DF804FB041D030010B584B0D9
:1093100001900091019B002B04D1154940F24710A8
:1093200003F0F2FF009B002B04D111494FF4A4700D
:1093300003F0EAFF009B039300238DF80B300DF13F
:109340000B031846FFF7CAFD019B1B681C68621CD3
:109350001A6003990198FFF71BFF034623709DF8DD
:109360000B301846FFF7D0FD00BF04B010BD00BFA2
:10937000041D030000B583B00190019B002B03D1B5
:109380000C49312003F0C0FF019B9B68002B0CD0DF
:10939000019B5B69019A1069019A1168019A9268B0
:1093A0009847019B00229A6000E000BF03B05DF87F
:1093B00004FB00BF541D03000EB400B584B001903F
:1093C000019B002B03D11849422003F09DFF019B14
:1093D0005B69002B03D11449432003F095FF019BE7
:1093E0001B68002B03D11049442003F08DFF019B23
:1093F0005B68002B03D10C49452003F085FF059BDA
:10940000002B0AD00023039306AB039303AB1A4649
:109410000599019800F0B8F900E000BF04B05DF8CC
:1094200004EB03B0704700BF541D030000B583B0C8
:1094300001900B468DF803309DF803300A2B03D1C1
:109440000D210198FFF7F2FF019B1A68019B9B68B1
:10945000581C0199886013449DF803201A70019BE1
:109460009A68019B5B689A4202D30198FFF782FFDA
:1094700000BF03B05DF804FB00B587B00390029114
:109480000192009300230593009B03F00103002B3E
:1094900024D00BE0029B01330293059B013305931B
:1094A0009DF8133019460398FFF7C0FF029B1B7805
:1094B0008DF813309DF81330002BEBD106E0019BA3
:1094C000013B019320210398FFF7B0FF019A059B10
:1094D0009A422ED9019B002BF1D12AE0029B002B4E
:1094E0000BD0029807F080FD059006E0019B013B40
:1094F000019320210398FFF799FF019A059B9A4257
:109500000FD9019B002BF1D10BE0029B0133029399
:10951000059B013305939DF8133019460398FFF717
:1095200085FF029B1B788DF813309DF81330002BBC
:10953000EBD100BF07B05DF804FB000000B589B0B7
:109540000390029101920093029B079301230693DB
:1095500007E0079A019BB2FBF3F30793069B0133E5
:109560000693079A019B9A42F3D2009A069B9A426D
:1095700001D9009B06930B9B03F00103002B22D122
:109580000A9B002B1FD00B9B03F00203002B06D07D
:10959000009B002B03D130238DF8173002E02023ED
:1095A0008DF8173008E00A9B013B0A939DF81730AD
:1095B00019460398FFF73AFF0A9B002B03D0069A3F
:1095C0000A9B9A42EFD301230793009B012B03D9F7
:1095D000009B013B009309E0029A079BB2FBF3F367
:1095E0000493049A019B9A4200D205E0079B019ADA
:1095F00002FB03F30793E8E7029A079BB2FBF3F33E
:109600000493049B079A02FB03F3029AD31A029372
:10961000154A049B13441B7819460398FFF706FF6D
:10962000079A019BB2FBF3F30793079B002BE3D14F
:109630000B9B03F00103002B11D00A9B002B0ED0D3
:1096400006E00A9B013B0A9320210398FFF7EEFEF8
:109650000A9B002B03D0069A0A9B9A42F1D300BFC3
:1096600009B05DF804FB00BFEC1D030000B589B034
:109670000590049103920293049B002BB8BF5B42B8
:1096800006930123079307E0039B069A92FBF3F3EB
:109690000693079B01330793039B069A9A42F3DADA
:1096A000029A079B9A4201D9029B07930A9B002BBF
:1096B0000AD0049B002B04DB0B9B03F00403002B5C
:1096C00002D00A9B013B0A930B9B03F00203002B81
:1096D00002D0029B002B16D00B9B03F00103002B42
:1096E00011D10A9B002B0ED006E00A9B013B0A9386
:1096F00020210598FFF79AFE0A9B002B03D0079ABA
:109700000A9B9A42F1D3049B002B07DA049B5B422D
:1097100004932D210598FFF789FE08E00B9B03F0C9
:109720000403002B03D02B210598FFF77FFE0B9B32
:1097300003F00203002B19D00B9B03F00103002B55
:1097400014D1029B002B11D10A9B002B0ED006E0F6
:109750000A9B013B0A9330210598FFF767FE0A9B9D
:10976000002B03D0079A0A9B9A42F1D304990B9BD2
:1097700001930A9B0093029B039A0598FFF7DEFE74
:1097800000BF09B05DF804FB00B58FB005900491EF
:109790000392059B002B04D1AD494FF4A27003F056
:1097A000B3FD059B5B69002B04D1A9494FF4A3705D
:1097B00003F0AAFD059B1B68002B04D1A44940F2CD
:1097C000471003F0A1FD059B5B68002B04D1A04965
:1097D0004FF4A47003F098FD049B002B00F09381DC
:1097E000049B1B788DF83730049B013304939DF85C
:1097F0003730002B00F07E819DF83730252B40F06C
:109800006D8100230A9301230C93049B1B788DF830
:1098100037309DF83730302B0DD0302B1BDC2B2B05
:1098200011D02D2B17D10A9B43F001030A93049BFF
:109830000133049312E00A9B43F002030A93049B52
:10984000013304930AE00A9B43F004030A93049B48
:109850000133049302E000230C9300BF0C9B002B08
:10986000D3D1002309939DF837302A2B0CD1039BC9
:109870001B68191D039A11601B68099A1344099308
:10988000049B013304931AE0049B1B788DF8373056
:109890009DF837302F2B12D99DF83730392B0ED841
:1098A000049B01330493099A13469B0013445B0005
:1098B0001A469DF837301344303B0993D3E7002311
:1098C0000B93049B1B788DF837309DF837302E2B87
:1098D0001DD1049B01330493049B1B788DF8373012
:1098E0009DF837302F2B12D99DF83730392B0ED8F1
:1098F000049B013304930B9A13469B0013445B00B3
:109900001A469DF837301344303B0B93E4E7049B31
:109910001B788DF837309DF837306C2B03D09DF8CD
:109920003730682B07D1049B01330493049B1B78C9
:109930008DF83730EFE79DF83730252B00F0C480E5
:10994000252BC0F2C680782B00F3C380582BC0F2C1
:10995000C080583B202B00F2BC8001A252F823F0BB
:10996000559A0200D39A0200D39A0200D39A0200B9
:10997000D39A0200D39A0200D39A0200D39A02002B
:10998000D39A0200D39A0200D39A0200E59902000A
:10999000079A0200D39A0200D39A0200D39A0200D7
:1099A000D39A0200079A0200D39A0200D39A0200C7
:1099B000D39A0200D39A0200D39A0200D39A0200EB
:1099C000959A0200D39A0200D39A0200799A020073
:1099D000D39A02002B9A0200D39A0200D39A020073
:1099E000559A0200039B1B68191D039A11601B689E
:1099F0000C930C9B8DF81F309DF81F30194605986D
:109A0000FFF714FD66E0039B1B68191D039A1160A4
:109A10001B680C930A9B0193099B00930B9B0A22E2
:109A20000C990598FFF722FE54E0039B1B68191D53
:109A3000039A11601B680C930C990A9B0193099B74
:109A400000930B9B0A220598FFF778FD42E000BFC8
:109A50009C1D0300039B1B68191D039A11601B6862
:109A60000C930C990A9B0193099B00930B9B10226A
:109A70000598FFF763FD2DE0039B1B68191D039AF2
:109A800011601B6808930A9B099A08990598FFF7CB
:109A9000F3FC1FE0039B1B68191D039A11601B68F0
:109AA0000C9330210598FFF7C1FC78210598FFF74A
:109AB000BDFC0C9900230193082300930823102276
:109AC0000598FFF73BFD05E025210598FFF7AEFC63
:109AD00000E000BF049B0133049305E09DF837309C
:109AE00019460598FFF7A2FC049B1B78002B7FF416
:109AF00077AE00E000BF059B1B7B002B04D00598D0
:109B0000FFF738FC00E000BF0FB05DF804FB00BFBA
:109B100000B583B001900198FFF754FB0346184647
:109B200003B05DF804FB00B58BB001900091019B80
:109B30001B8A043B0793009A079B1344DA1C079B7C
:109B4000B2FBF3F38DF81B300198FFF797FB0590FC
:109B5000059B002B01D1002338E0059B00221A71E0
:109B6000059B01225A71079B9AB2059BDA80059BDF
:109B700009939DF81B30013B0493099B019A1A60DD
:109B8000002308931DE00198FFF778FB0390039BE7
:109B9000002B0ED0059B5B790133DAB2059B5A711D
:109BA000099B039A1A60039B019A1A60039B09930D
:109BB00004E0059800F00EF8002307E0089B01334D
:109BC0000893089A049B9A42DDD3059B18460BB074
:109BD0005DF804FB00B58BB00190019B0793079BD8
:109BE0005B798DF81B30019B08939DF81B30013B7E
:109BF00005930023099305E0089B1B680893099BC4
:109C000001330993099A059B9A42F5D3089B1B6877
:109C10000493019B0893002309930BE0089B1B68A6
:109C2000039308990498FFF771FB039B0893099B22
:109C3000013309939DF81B30099A9A42EED300BF75
:109C400000BF0BB05DF804FB00B585B00190019B2F
:109C50000393039B043301211846FFF734FA00BF36
:109C600005B05DF804FB00B587B00190019B05933A
:109C7000059B043301211846FFF73DFA0346039381
:109C800003AB0493049B1B78002B02D10198FFF7D0
:109C9000A1FF00BF07B05DF804FB000000B591B064
:109CA0000390029101920093039B002B03D143493F
:109CB000B62003F029FB039B0993039B0F93099B99
:109CC000DB881A46099B5B7902FB03F3043B08938C
:109CD000009A089B9A4203D33849C42003F014FB2E
:109CE000099BDB880793009B1A1D079BB2FBF3F3CC
:109CF0000E93009B0433079AB3FBF2F2079901FB22
:109D000002F29B1A0D93019B1A68009B1344089A58
:109D10009A4203D2089A009BD31A01E0019B1B6868
:109D20000C93019B0C9A1A6005E00F9B1B680F9324
:109D30000E9B013B0E930E9B002BF6D100230B9341
:109D4000079A0D9BD31A0A930A9A0C9B934228BF39
:109D500013460A932AE0029A0B9B134406930F9A28
:109D60000D9B1344043305939DF84830002B05D018
:109D70000A9A0599069807F067F904E00A9A069985
:109D8000059807F061F900230D930F9B1B680F9353
:109D90000C9A0A9BD31A0C930B9A0A9B13440B93AD
:109DA000079A0C9B934228BF13460A930C9B002BE7
:109DB000D1D100BF00BF11B05DF804FBFC1D030052
:109DC00000B589B00590049103920293039B079319
:109DD00007AA00230093029B04990598FFF75EFFF2
:109DE000079B039A9A4203D00349F62003F08CFAAA
:109DF00000BF09B05DF804FBFC1D030000B589B08D
:109E00000590049103920293039B079307AA0123F1
:109E10000093029B04990598FFF740FF079B039A64
:109E20009A4204D004494FF4807003F06DFA00BFE9
:109E300009B05DF804FB00BFFC1D030082B00346BF
:109E40008DF807309DF8073003F01F0206499DF991
:109E500007305B09012000FA02F2603341F8232049
:109E600000BF02B0704700BF00E100E000B583B062
:109E70000190019B002B03D10649722003F044FAA4
:109E8000019B00221A60BFF35F8F00BF00BF03B0C9
:109E90005DF804FBA01E030041DF704700BF1846B9
:109EA00000B585B000238DF803300DF1030318468B
:109EB000FFF714F8F1EE103A0193019B0393039B13
:109EC00023F09F030293029BE1EE103A00BFBFF321
:109ED0005F8F00BF2620FFF7B1FF9DF803301846C3
:109EE000FFF712F8039B03F00703002B03D004498C
:109EF0007D2003F009FA00BF05B05DF804FB00BF48
:109F0000E41E030008B5064B00221A700548FFF74F
:109F1000ADFF0549054800F04DF80023184608BD7F
:109F20000C33002008330020381F030010330020BA
:109F300000B583B0FFF7B4FF06F0BCFC0346002B6E
:109F40000ED0FFF7A9FF0190019B002B0ED0019BC3
:109F5000022B0BD007494FF4B07003F0D5F905E0A0
:109F600020BF00BF40BF00BF20BF00BF00BF03B085
:109F70005DF804FBE41E030082B00190019B9B6826
:109F800000229A60019B9B6800221A61019B9B68DA
:109F900000225A61019B9B680022DA60019B9B684A
:109FA00000225A60019B9B6800221A6000BF02B029
:109FB0007047000000B583B001900091019B002B19
:109FC00003D11049502003F09FF9009B002B03D1CF
:109FD0000C49512003F098F9019B009A1A60019BEB
:109FE0001B681A68019B5A60019B5A68019B1B6899
:109FF0005B689A4202D1019B00225A6000BF03B005
:10A000005DF804FB441F030000B583B00190019B81
:10A01000002B03D11449632003F076F9019B1B68E0
:10A02000002B03D11049642003F06EF9019B5B689B
:10A03000002B14D0019B5B681A46019B1B689B6830
:10A0400013441A46019B5A60019B5A68019B1B6886
:10A050005B689A4204D1019B00225A6000E000BF75
:10A0600003B05DF804FB00BF441F030000B585B0DA
:10A070000190019800F00EF80390039B002B01D093
:10A08000039B00E0024B184605B05DF804FB00BFDF
:10A09000B01F030086B00190164B0593164B049336
:10A0A0001FE0049A059BD31ADB10DA0F13445B10F0
:10A0B000DB00059A13440393039B1B680293029AE7
:10A0C000019B9A4202D9039B04930AE0029A019BE6
:10A0D0009A4203D2039B0833059302E0039B5B681B
:10A0E00004E0059A049B9A42DBD30023184606B08D
:10A0F000704700BFB0230300D8240300BFF34F8F85
:10A1000000BF074BDB6803F4E0620549054B1343CE
:10A11000CB60BFF34F8F00BF00BF00BFFCE700BFA5
:10A1200000ED00E00400FA05024B034A1A6000BF8C
:10A13000704700BFEC2A00200090D00308B500F063
:10A1400027F90346002B0ED04FF080430022C3F8BE
:10A150000C214FF080430022C3F810214FF08043C0
:10A160000022C3F8382500F037F90346002B76D0DB
:10A170004FF080537D4AD3F80434C2F820354FF0B5
:10A1800080537A4AD3F80834C2F824354FF080530C
:10A19000764AD3F80C34C2F828354FF08053734A0E
:10A1A000D3F81034C2F82C354FF080536F4AD3F8EF
:10A1B0001434C2F830354FF080536C4AD3F8183459
:10A1C000C2F834354FF08053684AD3F81C34C2F8D3
:10A1D00040354FF08053654AD3F82034C2F84435F7
:10A1E0004FF08053614AD3F82434C2F848354FF019
:10A1F00080535E4AD3F82834C2F84C354FF0805370
:10A200005A4AD3F82C34C2F850354FF08053574A8D
:10A21000D3F83034C2F854354FF08053534AD3F852
:10A220003434C2F860354FF08053504AD3F8383494
:10A23000C2F864354FF080534C4AD3F83C34C2F82E
:10A2400068354FF08053494AD3F84034C2F86C3532
:10A250004FF08053454AD3F84434C2F8703500F0CB
:10A26000DFF80346002B02D0414B424A1A6000F04F
:10A27000E9F80346002B03D03F4BFB22C3F8182517
:10A2800000F0F2F80346002B0AD03C4B1B6823F089
:10A290000F023B4B1B6803F00F03384913430B605D
:10A2A00000F0F4F80346002B03D0364B4FF4007255
:10A2B0001A6000F0FDF80346002B0DD04FF08043EC
:10A2C000D3F8003403F00103002B05D04FF0804396
:10A2D0006FF00102C3F800242B4BD3F888302A4AD0
:10A2E00043F47003C2F88830BFF34F8F00BFBFF351
:10A2F0006F8F00BF4FF01023D3F80032002B05DB27
:10A300004FF01023D3F80432002B2BDA1F4B01221D
:10A31000C3F8042500BF1D4BD3F80034002BFAD03E
:10A320004FF010231222C3F8002200BF174BD3F8BE
:10A330000034002BFAD04FF010231222C3F804226D
:10A3400000BF124BD3F80034002BFAD00F4B002281
:10A35000C3F8042500BF0D4BD3F80034002BFAD00E
:10A36000FFF7CCFEFFF7E0FE00BF08BD00C00040D5
:10A370008C5600404881030000F00040E40E00408D
:10A38000580200104096024000ED00E000E001405D
:10A390000F4B1B68082B17D10E4B1B68002B01D1EC
:10A3A000012312E00B4B1B68012B01D101230CE0B0
:10A3B000084B1B68022B01D1012306E0054B1B68EB
:10A3C000032B01D1012300E001231846704700BF91
:10A3D00030010010340100100F4B1B68082B17D1FF
:10A3E0000E4B1B68002B01D1012312E00B4B1B68A5
:10A3F000012B01D101230CE0084B1B68022B01D17A
:10A40000012306E0054B1B68032B01D1012300E06B
:10A4100001231846704700BF3001001034010010BE
:10A42000064B1B68082B05D1054B1B68002B01D17F
:10A43000012300E000231846704700BF30010010E0
:10A4400034010010064B1B68082B05D1054B1B6817
:10A45000002B01D1012300E000231846704700BF04
:10A460003001001034010010064B1B68082B05D189
:10A47000054B1B68002B01D1012300E00023184687
:10A48000704700BF3001001034010010064B1B68FC
:10A49000082B05D1054B1B68002B01D1012300E0DF
:10A4A00000231846704700BF30010010340100102F
:10A4B0000F4B1B68082B17D10E4B1B68002B01D1CB
:10A4C000012312E00B4B1B68012B01D101230CE08F
:10A4D000084B1B68022B01D1012306E0054B1B68CA
:10A4E000032B01D1012300E001231846704700BF70
:10A4F000300100103401001082B003468DF807309F
:10A500009DF8073003F01F0206499DF907305B09EB
:10A51000012000FA02F2203341F8232000BF02B0EC
:10A52000704700BF00E100E008B506F0C3F903463C
:10A5300083F00103DBB2002B03D10549792002F03F
:10A54000E3FE00F043FB034B00229A7000BF08BDFE
:10A55000E02403001833002000B583B000230193EA
:10A56000144B1B78002B02D0852301931CE0114B68
:10A5700000229A600F4B00225A600E4B00221A6193
:10A580000C4B0022DA600C4800F0E6FA019006F06D
:10A5900091F9034683F00103DBB2002B01D000F0F8
:10A5A00001FB044B01221A70019B184603B05DF8B1
:10A5B00004FB00BF1833002091A6020084B0019074
:10A5C000019B1B680393039B002B03D0039B1A681A
:10A5D000019B1A60039B184604B0704700B583B016
:10A5E000164B1B78002B04D115494FF4857002F0EF
:10A5F0008BFE124BDB68002B04D1114940F20B108B
:10A6000002F082FE00238DF807300DF10703184693
:10A61000FEF764FC094BDB68013B084AD360074B3B
:10A62000DB68002B01D1FFF77FFF9DF8073018464C
:10A63000FEF76AFC00BF03B05DF804FB183300208E
:10A64000E024030000B585B003468DF807309DF87F
:10A650000730002B02D10C4B039301E00B4B03930B
:10A660000398FFF7ABFF0290029B002B06D0029BE2
:10A670005B689DF8072010469847F1E700BF00BFD0
:10A6800005B05DF804FB00BF203300202833002014
:10A6900000B583B003468DF807309DF80730002BD6
:10A6A00005D10A4B01225A700020FFF7CBFF9DF81D
:10A6B0000730012B05D1054B01229A700120FFF7CD
:10A6C000C1FF00BF03B05DF804FB00BF18330020DA
:10A6D00000B583B001900091019B002B05D1054B83
:10A6E00001225A700020FFF7ADFF00BF03B05DF8F4
:10A6F00004FB00BF1833002000B585B0034600916D
:10A700008DF807309DF80730032B29D0032B35DC5B
:10A71000002B02D0012B04D030E00020FFF7ECFE2C
:10A720002DE000238DF80F300DF10F031846FEF7D2
:10A73000D5FB154B1B7883F00103DBB2002B01D056
:10A74000FFF70AFF104BDB6801330F4AD3600E4B53
:10A7500001229A709DF80F301846FEF7D5FB0EE0E7
:10A76000094B1B78002B04D1084940F2452002F028
:10A77000CBFD00F017FAFFF731FF00E000BF00BF8C
:10A7800005B05DF804FB00BF18330020E02403008F
:10A7900000B589B001900091009B0793019B1B7845
:10A7A0008DF80C30019B5B680493019B9B68DBB2C6
:10A7B0008DF81430019BDB680693074A079B52F81B
:10A7C00023300649079A51F8221003AA10469847E9
:10A7D00000BF09B05DF804FB2C33002034330020A7
:10A7E00000B589B001900091009B0793019B1B78F5
:10A7F0008DF80C30019B5B680493019B9B68DBB276
:10A800008DF81430019BDB680693074A079B52F8CA
:10A8100023300649079A51F8221003AA1046984798
:10A8200000BF09B05DF804FB2C3300203433002056
:10A8300030B58FB0039002910192039B1B780C936B
:10A840002C490C9B019A41F82320029B1A692A4942
:10A850000C9B41F823200C9B012B07D1029B5B7FB3
:10A86000002B03D12549762002F04EFD029B5B7F31
:10A870001946234A0C9B13440A461A70029B04ACE7
:10A880001D460FCD0FC495E80F0084E80F000C9B08
:10A89000089300230D93039B1B781A46184B9B5C6F
:10A8A000002B0DD0039B181D019B002B01D0154AD6
:10A8B00000E0002204AB194602F0D6F80D9014E037
:10A8C000039B1B781A460E4B9B5C002B0DD1039B00
:10A8D00003F10C00019B002B01D00B4A00E0002289
:10A8E00004AB194601F042FA0D900D9B18460FB0CB
:10A8F00030BD00BF2C33002034330020302503004E
:10A900003C33002091A70200E1A7020082B0034679
:10A910008DF807309DF8073003F01F0205499DF9B7
:10A9200007305B09012000FA02F241F8232000BF42
:10A9300002B0704700E100E082B0034600918DF85C
:10A9400007309DF90730002B0CDA009BDAB20C4976
:10A950009DF8073003F00F03043B5201D2B20B44C1
:10A960001A7609E0009BDAB206499DF907305201D8
:10A97000D2B20B4483F8002300BF02B0704700BF7F
:10A9800000ED00E000E100E082B00190019B1B0BB4
:10A990005BB2184602B0704700B583B003460A4662
:10A9A0008DF8073013468DF806309DF80630012BE0
:10A9B00003D99DF80630032B0BD99DF80630042BE4
:10A9C00003D99DF80630072B03D908496B2002F004
:10A9D0009BFC9DF806209DF9073011461846FFF7AD
:10A9E000ABFF00BF03B05DF804FB00BF8025030090
:10A9F00000B583B003468DF807309DF9073018463F
:10AA0000FFF784FF00BF03B05DF804FB82B003468C
:10AA10008DF807300F4A9DF90730002B00DA1F33FD
:10AA20005B115BB252F823209DF90730594203F0C5
:10AA30001F0301F01F0158BF4B425BB222FA03F320
:10AA400003F00103002B14BF01230023DBB21846DF
:10AA500002B0704700E100E082B001904FF0804208
:10AA6000019BC2F8083300BF02B0704782B00346B2
:10AA70008DF807309DF8073003F1804301221A60FA
:10AA800000BF02B0704784B00346ADF80630BDF891
:10AA9000063003F1804300221A60BDF8063003F14E
:10AAA00080431B680393039B00BF04B0704782B0D0
:10AAB0000346ADF80630BDF8063003F180431B684D
:10AAC000002B14BF01230023DBB2184602B07047ED
:10AAD00082B001904FF08042019BC2F8183500BF50
:10AAE00002B070474FF08043D3F818341B0C03F0CA
:10AAF0000103002B14BF01230023DBB2184670476B
:10AB000000B583B006238DF807304FF08040FFF783
:10AB10003BFF03461846FFF779FF034683F0010326
:10AB2000DBB2002B13D04FF08040FFF72DFF034620
:10AB30001A469DF8073019461046FFF72DFF4FF0D3
:10AB40008040FFF721FF03461846FFF751FF00BF83
:10AB500003B05DF804FB000000B585B00190019BD7
:10AB6000002B03D10D49A02002F0CEFB002303935C
:10AB70000B4B1B79002B02D08523039308E0084A76
:10AB8000019B1360064B01221A71054B00225A717A
:10AB9000039B184605B05DF804FB00BFB825030011
:10ABA0004033002008B5074B1B79002B03D1064921
:10ABB000B92002F0A9FBFFF7A3FF0120FFF788FFF0
:10ABC00000BF08BD40330020B825030008B50A4B7C
:10ABD0001B79002B03D10949F32002F095FB0C20CF
:10ABE000FFF744FF00BFFFF77DFF0346002BFAD1BC
:10ABF00000BF00BF08BD00BF40330020B8250300E0
:10AC000008B54FF48070FFF752FF0346002B14D0B5
:10AC10004FF48070FFF737FF0120FFF71DFF114B46
:10AC20005B7983F00103DBB2002B06D00D4B0122D0
:10AC30005A710C4B1B68002098474FF48270FFF745
:10AC400036FF0346002B0AD04FF48270FFF71BFF3C
:10AC50000220FFF701FF034B1B680120984700BF4C
:10AC600008BD00BF4033002082B003468DF8073096
:10AC70009DF8073003F01F0205499DF907305B0975
:10AC8000012000FA02F241F8232000BF02B0704711
:10AC900000E100E082B0034600918DF807309DF995
:10ACA0000730002B0CDA009BDAB20C499DF8073014
:10ACB00003F00F03043B5201D2B20B441A7609E0B1
:10ACC000009BDAB206499DF907305201D2B20B441B
:10ACD00083F8002300BF02B0704700BF00ED00E022
:10ACE00000E100E000B583B003460A468DF8073066
:10ACF00013468DF806309DF80630012B03D99DF8D8
:10AD00000630032B0BD99DF80630042B03D99DF890
:10AD10000630072B03D908496B2002F0F5FA9DF89D
:10AD200006209DF9073011461846FFF7B3FF00BF14
:10AD300003B05DF804FB00BF0826030000B583B034
:10AD400003468DF807309DF907301846FFF78CFF52
:10AD500000BF03B05DF804FB00B583B00346ADF857
:10AD60000630BDF80630184600F026F803461B688A
:10AD7000012B0CBF01230023DBB2184603B05DF8A2
:10AD800004FB00B585B00346ADF80630BDF80630CB
:10AD9000184600F011F803461A4600231360BDF868
:10ADA0000630184600F008F803461B680393039B1F
:10ADB00000BF05B05DF804FB82B00346ADF8063075
:10ADC000BDF8063003F1804303F5C043184602B0D6
:10ADD0007047000082B00190034A019BC2F804331F
:10ADE00000BF02B0704700BF0060004082B0019019
:10ADF000034BD3F80423019B1340184602B070475D
:10AE00000060004084B00390029113468DF8073033
:10AE1000144A039B03F5A27352F82330114923F41B
:10AE20004F3323F44073039A02F5A27241F82230A3
:10AE30000C4A039B03F5A27352F82320029B1B02CA
:10AE400003F47C519DF807301B0403F440330B439B
:10AE500004491A43039B03F5A27341F8232000BF62
:10AE600004B070470060004082B00190054A019B29
:10AE700003F5A27352F823301B0A03F03F03184670
:10AE800002B070470060004082B00190064A019B0A
:10AE900003F5A27352F823301B0C03F00303DBB25B
:10AEA000184602B0704700BF0060004000B583B094
:10AEB0000190019B1B682F2B04D90B494FF4F370B1
:10AEC00002F022FA019B1B681F2B02D84FF0A0430F
:10AED00006E0019B1B6803F01F02019B1A60034BF5
:10AEE000184603B05DF804FB382603000003005049
:10AEF00000B585B00190084611461A4603468DF804
:10AF000003300B468DF8023013468DF8013001AB4B
:10AF10001846FFF7CBFF03909DF803209DF8023001
:10AF20005B001A439DF801309B001A439DF81830CE
:10AF30001B0242EA03019DF81C301B04019A1943CD
:10AF4000039B02F5E07243F8221000BF05B05DF8E4
:10AF500004FB00B585B003900B468DF80B309DF8CF
:10AF60000B3000220192002200920022002103985F
:10AF7000FFF7BEFF00BF05B05DF804FB00B585B06C
:10AF8000019001AB1846FFF791FF0390019A039BD4
:10AF900002F5E07253F8223023F002030293019A83
:10AFA000039B02F5E072029943F8221000BF05B03E
:10AFB0005DF804FB00B585B001900B468DF80330B9
:10AFC00001AB1846FFF772FF0390019A039B02F54D
:10AFD000E07253F82230019A23F44031039B02F5CA
:10AFE000E07243F82210019A039B02F5E07253F8D5
:10AFF00022309DF8032012041146019A1943039B45
:10B0000002F5E07243F8221000BF05B05DF804FBC2
:10B0100000B585B0019001AB1846FFF747FF0390DC
:10B02000039800F020F80246019B22FA03F303F094
:10B030000103184605B05DF804FB00B585B001902A
:10B0400001AB1846FFF732FF0390019A039B02F50C
:10B05000E07253F822301B0C03F00303DBB21846F6
:10B0600005B05DF804FB82B00190019BD3F8103568
:10B07000184602B07047000000B589B003900291F5
:10B080000192184A05AB92E8030083E80300039A93
:10B09000029B1344022B04D9134940F2163002F0EC
:10B0A00033F9039B079311E0079B9B0020336B440C
:10B0B00053F80C3C1846FFF7D6FF0246019B1A6076
:10B0C000019B04330193079B01330793039A029B6F
:10B0D0001344079A9A42E7D300BF00BF09B05DF856
:10B0E00004FB00BF682603003826030084B00190EB
:10B0F0000091009B0393019BDB080293019B03F0EB
:10B10000070301930122019B02FA03F30399029AB8
:10B110000A4412781340184604B0704784B0019076
:10B120000091009B0393019BDB080293019B03F0BA
:10B1300007030193039A029B13441B785AB201211F
:10B14000019B01FA03F35BB2134359B2039A029BCA
:10B150001344CAB21A7000BF04B0704782B00190A5
:10B16000064A019B1344303393F90030DB43DBB2D2
:10B17000DB09DBB2184602B0704700BF483300203D
:10B1800084B00390029101928DF80330029B59B272
:10B190000E4A039B134430330A461A700B49029B34
:10B1A000019A41F823209DF8033083F00103DBB2BC
:10B1B000002B08D0029B083B039A51B2034A134468
:10B1C0000A4683F8602000BF04B07047483300206F
:10B1D00082B00190044A019B13443033FF221A705D
:10B1E00000BF02B0704700BF4833002000B583B0F5
:10B1F000019004490198FFF791FF00BF03B05DF88B
:10B2000004FB00BFAC33002082B00190044A019BD4
:10B210001344303393F90030184602B0704700BF32
:10B220004833002082B00190034A019B52F823303A
:10B23000184602B0704700BF4833002000B589B0FF
:10B240000390029113468DF80730FF238DF81F30CD
:10B250009DF80730002B01D0002300E00823059360
:10B260009DF80730002B01D0082300E00C23049345
:10B27000059B069314E00F4A069B52F82330B3F166
:10B28000FF3F0AD19DF80730029A06990398FFF70D
:10B2900077FF069B8DF81F3006E0069B013306936F
:10B2A000069A049B9A42E6D39DF91F30184609B0CE
:10B2B0005DF804FB4833002082B003468DF8073068
:10B2C0009DF80730094A4FF0FF3142F823109DF8EE
:10B2D0000730072B07D99DF80730083B034A134472
:10B2E000FF2283F8602000BF02B07047483300207F
:10B2F00000B583B0254B93F86A30002B03D00823A8
:10B300000193019B3EE000238DF8033009E09DF896
:10B3100003301846FFF75CFF9DF8033001338DF8CA
:10B3200003309DF803302F2BF1D900238DF8033023
:10B3300009E09DF803301846FFF7BEFF9DF8033083
:10B3400001338DF803309DF803300B2BF1D9062221
:10B3500000210F4805F0AEFE06210620FFF7C2FCD3
:10B360000620FFF7EBFC4FF4BE70FFF70AFD4FF02D
:10B370000040FFF72FFD054B012283F86A200023D0
:10B380000193019B184603B05DF804FB483300208D
:10B39000AC330020044B93F86A30002B14BF012318
:10B3A0000023DBB2184670474833002000B587B051
:10B3B000039002910192039B2F2B04D9364940F24E
:10B3C000072001F0A1FF002305930398FFF7C6FEB5
:10B3D0000346002B02D00823059357E0029B9B787D
:10B3E000C3F34003DBB21A4601990398FFF726FF27
:10B3F00003468DF813309DF91330B3F1FF3F43D06E
:10B40000029B9B78C3F38003DBB283F00103DBB2C2
:10B41000002B13D0029B9B7803F00103DBB2002BBF
:10B4200003D00398FFF7AAFD05E0029B5B7819465D
:10B430000398FFF78EFD0398FFF7D8FE029B9B78D9
:10B4400003F00203DBB2002B08D09DF91300029B2E
:10B450001B781A460399FFF7D5FC17E09DF91330C6
:10B46000083B0E4A134493F96010029B1B789B0122
:10B470005AB29DF91330083B0A4351B2074A1344AC
:10B480000A4683F8602001E004230593059B1846D3
:10B4900007B05DF804FB00BF7826030048330020A6
:10B4A00000B583B00190019B2F2B04D908494FF4BC
:10B4B000227001F029FF0198FFF7AAFD0346002B37
:10B4C00014BF01230023DBB2184603B05DF804FB70
:10B4D0007826030000B599B00023149306AB002230
:10B4E0001A605A604FF48073ADF84A300123169306
:10B4F0000023139321E0BDF84A301846FFF72CFCD7
:10B500000346002B0ED01698FFF770FC0346002B65
:10B5100008D0BDF84A301846FFF733FC149A169B42
:10B5200013431493169B5B001693BDF84A30043303
:10B53000ADF84A30139B01331393139B072BDAD9D1
:10B540004FF4BE70FFF708FC0346002B0DD04FF4FC
:10B55000BE70FFF716FC149B43F00043149306AB38
:10B560001A4602210020FFF787FD149BDBB2002B57
:10B5700029D0012316930023139321E0169A149BDC
:10B580001340002B16D01398FFF76EFC1190139800
:10B59000FFF77AFC03468DF843301398FFF742FE1D
:10B5A0000F900F9B002B05D09DF843200F9B114659
:10B5B00011989847169B5B001693139B01331393C6
:10B5C000139B072BDAD9149B002B80F2F080002309
:10B5D0008DF85F3004AB00221A605A600023159387
:10B5E0000AE0159B9B0060336B444FF0FF3243F839
:10B5F000582C159B01331593159B012BF1D9002372
:10B600008DF85F300023139378E06B4A139B13444B
:10B61000603393F900308DF83B309DF83B3023F0D8
:10B62000C0030D93644A139B1344603393F90030B5
:10B63000B3F1FF3F5FD002AB19460D98FFF756FDFF
:10B640000346002B57D09DF83B309B098DF83330D3
:10B650000D98FFF7D9FD03461846FFF7E3FD0B9061
:10B660000B9B002B03D19DF83330032B43D19DF866
:10B670003330032B04D104AB19460D98FFF74EFD70
:10B680000D98FFF7DAFC03468DF82B3006AB194610
:10B690000D98FFF72BFD0990099B002B03D09DF817
:10B6A0002B30022B06D0099B002B24D19DF82B3088
:10B6B000032B20D19DF83330032B13D19DF82B3071
:10B6C000022B01D1032300E002238DF823309DF8E3
:10B6D000233019460D98FFF76DFC9DF85F3001335C
:10B6E0008DF85F300B9B002B05D09DF833200B9B12
:10B6F00011460D989847139B01331393139B032B0B
:10B7000083D99DF85F30002B4CD001238DF85E303B
:10B710006B461A4602210020FFF7AEFC002315936A
:10B7200014E0159B9B0060336B4453F8602C159B11
:10B730009B0060336B4453F8483C9A4203D000238B
:10B740008DF85E3005E0159B01331593159B012B99
:10B75000E7D99DF85E30002B03D000238DF85F30D1
:10B7600020E0002315931AE0159B9B0060336B4487
:10B7700053F8602C159B9B0060336B4443F8482CB6
:10B78000159B9B0060336B4453F8502C159B9B001A
:10B7900060336B4443F8582C159B01331593159B6C
:10B7A000012BE1D99DF85F30002B7FF428AF00BF5B
:10B7B00019B05DF804FB00BF4833002008B5064B04
:10B7C0001B68002B03D10549512001F09DFD024B60
:10B7D0001B68984700BF08BDB4330020CC26030087
:10B7E00082B00190019B044A934201D1034B00E0D7
:10B7F0000023184602B0704700200040B4330020F8
:10B8000000B587B001900091019B002B03D11C492A
:10B81000772001F079FD0198FFF7E2FF0590059B85
:10B82000002B25D000238DF8133000238DF80B302A
:10B830000DF10B031846FDF751FB059B1B79002BFF
:10B8400003D001238DF8133005E0059B009A1A60A0
:10B85000059B01221A719DF80B301846FDF754FB29
:10B860009DF81330002B03D011230393039B02E0B8
:10B8700000230393039B184607B05DF804FB00BF49
:10B88000CC26030082B003468DF807309DF80730C0
:10B8900003F01F0205499DF907305B09012000FAFA
:10B8A00002F241F8232000BF02B0704700E100E03F
:10B8B00082B0034600918DF807309DF90730002BC8
:10B8C0000CDA009BDAB20C499DF8073003F00F0345
:10B8D000043B5201D2B20B441A7609E0009BDAB263
:10B8E00006499DF907305201D2B20B4483F8002378
:10B8F00000BF02B0704700BF00ED00E000E100E0D3
:10B9000082B00190019B1B0B5BB2184602B07047DE
:10B9100000B583B003460A468DF8073013468DF80C
:10B9200006309DF80630012B03D99DF80630032B15
:10B930000BD99DF80630042B03D99DF80630072B50
:10B9400003D908496B2001F0DFFC9DF806209DF922
:10B95000073011461846FFF7ABFF00BF03B05DF894
:10B9600004FB00BF1C27030000B583B003468DF81D
:10B9700007309DF907301846FFF784FF00BF03B07A
:10B980005DF804FB84B001900B46ADF80230BDF8C1
:10B990000230019A134400221A60BDF80230019A65
:10B9A00013441B680393039B00BF04B0704782B02D
:10B9B00001900B46ADF80230BDF80230019A1344F5
:10B9C0001B68002B14BF01230023DBB2184602B012
:10B9D000704782B001900091019B009AC3F8042344
:10B9E00000BF02B0704782B001900091019BD3F874
:10B9F0000423009B1340002B14BF01230023DBB260
:10BA0000184602B0704782B001900091019B009AE5
:10BA1000C3F8082300BF02B0704784B00190019BB7
:10BA2000D3F880340393019B039AC3F88024039BCB
:10BA3000184604B0704782B00190019B0422C3F8FD
:10BA4000002500BF02B0704784B0039002910192BC
:10BA5000039B019AC3F81425039B029AC3F80C2593
:10BA600000BF04B0704784B0039002910192039B21
:10BA7000029AC3F80825039B019AC3F8102500BF5A
:10BA800004B0704782B00190019BD3F81835DBB247
:10BA9000184602B0704782B001900B468DF8033013
:10BAA0009DF80320019BC3F81C2500BF02B070471E
:10BAB00082B001900B468DF803309DF80330019A57
:10BAC000134401221A6000BF02B0704782B0019097
:10BAD0000B468DF8033013468DF802309DF8032095
:10BAE0009DF802301343DBB21A46019BC3F86C2564
:10BAF00000BF02B0704782B001900091019B009A94
:10BB0000C3F8242500BF02B07047000000B583B021
:10BB10000190019B1B682F2B04D90B494FF4F37044
:10BB200001F0F2FB019B1B681F2B02D84FF0A043D2
:10BB300006E0019B1B6803F01F02019B1A60034B88
:10BB4000184603B05DF804FB4C27030000030050C7
:10BB500000B585B00190084611461A4603468DF897
:10BB600003300B468DF8023013468DF8013001ABDF
:10BB70001846FFF7CBFF03909DF803209DF8023095
:10BB80005B001A439DF801309B001A439DF8183062
:10BB90001B0242EA03019DF81C301B04019A194361
:10BBA000039B02F5E07243F8221000BF05B05DF878
:10BBB00004FB00B585B0039000230193002300939C
:10BBC0000023012201210398FFF7C2FF00BF05B047
:10BBD0005DF804FB00B585B003900B468DF80B3083
:10BBE0009DF80B30002201920022009200220021D9
:10BBF0000398FFF7ADFF00BF05B05DF804FB00B58B
:10BC000085B0019001AB1846FFF780FF0390019BC0
:10BC1000012202FA03F31946039800F004F800BF6A
:10BC200005B05DF804FB82B001900091019B009A81
:10BC3000C3F8082500BF02B0704700B583B001907B
:10BC40000091009B1B68B3F1FF3F09D0009B1B686C
:10BC50001846FFF7D4FF009B1B681846FFF7A9FFA3
:10BC6000009B5B68B3F1FF3F05D0009B5B68002140
:10BC70001846FFF7AFFF019B1A68009B9B691946A6
:10BC80001046FFF738FF019B1868009B597D009B09
:10BC90001B7D1A46FFF71AFF019B1868009B196865
:10BCA000009B5B681A46FFF7CFFE009B1B7D012BB4
:10BCB00022D1009B9B68B3F1FF3F05D0009B9B689E
:10BCC00000211846FFF786FF009BDB68B3F1FF3FBA
:10BCD00009D0009BDB681846FFF791FF009BDB68EB
:10BCE0001846FFF766FF019B1868009BD968009B08
:10BCF0009B681A46FFF7B7FE00BF03B05DF804FB70
:10BD000000B583B001900B468DF80330019B1B6892
:10BD10004FF48E711846FFF735FE019B1B684FF4F8
:10BD2000A2711846FFF72EFE019B1B680E491846AC
:10BD3000FFF74FFE019B1B681846FFF7E1FD034626
:10BD40001A469DF8033019461046FFF7E1FD019BA6
:10BD50001B681846FFF7D4FD03461846FFF704FE9C
:10BD600000BF03B05DF804FB8000020000B587B09F
:10BD7000039002910192029B002B03D12D49AA202E
:10BD800001F0C2FA039B1B791A462C2302FB03F332
:10BD9000294A1344049300230593049B93F82A3003
:10BDA000002B03D008230593059B3EE0039B1A68F4
:10BDB000039B1B791946214B53F821301946104635
:10BDC000FFF71EFD0346002B03D011230593059BAF
:10BDD0002BE002990398FFF730FF049B019A5A6009
:10BDE000029B1A69049B1A60049B5B68002B05D0B8
:10BDF000029B1B7F19460398FFF782FF039B1B687A
:10BE00001846FFF718FE049B00229A61049B00224B
:10BE1000DA61049B002283F82920049B00225A61E6
:10BE2000049B012283F82A20059B184607B05DF881
:10BE300004FB00BF84270300BC330020D02703008D
:10BE400000B585B0019000914FF48E710198FFF715
:10BE500099FD009B9A68009B1B6A13441B788DF820
:10BE60000F30009B1B6A5A1C009B1A629DF80F3012
:10BE700019460198FFF70FFE00BF05B05DF804FBFF
:10BE800000B583B00190009116E0009B93F8283034
:10BE9000DBB2002B01D0002315E04FF48E71019826
:10BEA000FFF785FD034683F00103DBB2002BECD1E5
:10BEB00000990198FFF7C4FF009B1A6A009B5B6919
:10BEC0009A42EAD30123184603B05DF804FB000050
:10BED00000B587B0039002910192039B1B791A462B
:10BEE0002C2302FB03F33C4A13440493049B93F872
:10BEF0002A30012B04D0394940F2151001F004FA20
:10BF0000029B002B04D135494FF48B7001F0FCF9F2
:10BF1000019B002B04D1314940F2171001F0F4F9D4
:10BF2000039800F05DF80346002B03D0112305931E
:10BF3000059B4CE0049B019A5A61049B029A9A600B
:10BF4000049B00221A62049B002283F8282000230D
:10BF50000593039B1B684FF48E711846FFF712FD83
:10BF6000039B1B6808211846FFF7A2FD039B1B6873
:10BF700004991846FFF764FF049B5B68002B25D1EA
:10BF8000039B1B6804991846FFF77AFF034683F06A
:10BF90000103DBB2002B02D00F23059313E000BF97
:10BFA000039B1B684FF48E711846FFF700FD034694
:10BFB00083F00103DBB2002BF2D1039B1B680C2141
:10BFC0001846FFF775FD049B00225A61059B184631
:10BFD00007B05DF804FB00BFBC33002084270300DA
:10BFE00082B00190019B1B791946074A2C2301FB63
:10BFF00003F3134414331B68002B14BF01230023E5
:10C00000DBB2184602B07047BC33002000B583B0E5
:10C010000190019B1B684FF492711846FFF7B2FC28
:10C02000019B1B684FF484711846FFF7ABFC019B22
:10C030001B6800211846FFF73BFD00BF03B05DF809
:10C0400004FB10B582B001900091009B9B69002B0E
:10C0500008D14FF484710198FFF794FC0198FFF721
:10C0600011FD13E04FF484710198FFF78BFC009BE6
:10C07000DA68009B5B6AD4180198FFF703FD03465A
:10C080002370009B5B6A5A1C009B5A6202B010BD71
:10C0900000B589B0039002910192039B1B791A4667
:10C0A0002C2302FB03F37F4A13440593039B1B7964
:10C0B00019467C4A2C2301FB03F313442A331B78D3
:10C0C000012B04D0784940F2691001F01DF9029B60
:10C0D000002B04D174494FF4B57001F015F9019BA0
:10C0E000002B04D1704940F26B1001F00DF90023D0
:10C0F0008DF81C30059B5B68002B06D0039B1B68EA
:10C100004FF401711846FFF77EFC059B9B69002BDD
:10C1100015D0059BDB69002B0ED0059B5B68002BBF
:10C1200006D0039B1B684FF401711846FFF751FCC2
:10C1300011230693069BB0E001238DF81C309DF877
:10C140001C3083F00103DBB2002B0CD0059B019A5D
:10C150009A61059B029ADA60059B00225A62059B50
:10C160000022DA6105E0059B029A1A61059B019A9B
:10C17000DA61059B93F8293083F00103DBB2002BD1
:10C1800009D09DF81C3083F00103DBB2002B02D0F4
:10C190000398FFF73BFF059B5B68002B73D1039B64
:10C1A0001B684FF4A2711846FFF7ECFB039B1B685A
:10C1B0004FF492711846FFF7FAFB03468DF81F30D3
:10C1C000039B1B684FF484711846FFF7F0FB03468E
:10C1D0008DF81E30039B1B684FF4A2711846FFF7C1
:10C1E000E6FB03468DF81D309DF81E3083F00103F9
:10C1F000DBB2002B0DD09DF81D3083F00103DBB2C4
:10C20000002B06D09DF81F3083F00103DBB2002B1A
:10C21000CCD19DF81F30002B0FD19DF81D30002B85
:10C220000BD1039B1B6805991846FFF70AFF059B76
:10C230009A69059B5B6A9A42B8D8059B00229A616D
:10C240009DF81F30002B03D003230693069B24E0A8
:10C250009DF81D30002B03D00F230693069B1CE096
:10C26000059B93F82930002B06D0039B1B68002107
:10C270001846FFF71DFC0DE0039B1B6804211846C0
:10C28000FFF716FC06E0039B1B684FF4017118468C
:10C29000FFF79FFB00230693069B184609B05DF845
:10C2A00004FB00BFBC3300208427030000B589B025
:10C2B00003900291019201238DF81030029B0693A6
:10C2C000019B0593039B5B68039A116804AA1046BF
:10C2D000984700BF09B05DF804FB00B587B0019036
:10C2E000009100238DF80830009B0493019B9B680C
:10C2F0000393019B00225A61019B5B68019A1168BC
:10C3000002AA1046984700BF07B05DF804FB00B5CD
:10C3100089B0019000914FF400710198FFF763FB21
:10C320000346002B39D04FF492710198FFF73FFB81
:10C330000346002B31D04FF492710198FFF722FB96
:10C340004FF401710198FFF75EFB009B93F82930D1
:10C3500083F00103DBB2002B03D004210198FFF727
:10C36000A7FB02238DF808300198FFF756FB034620
:10C370000593009B9B690493009BDB680393009BE0
:10C3800000229A61009B0022DA61009B5B68009AA0
:10C39000116802AA1046984752E004210198FFF75D
:10C3A00022FB0346002B4BD04FF484710198FFF71A
:10C3B000FEFA0346002B43D000990198FFF741FE97
:10C3C000009B9A69009B5B6A9A4239D1009BDB69AA
:10C3D000002B19D0009BDB680793009B5B6A0693D8
:10C3E000009BDA69009B9A61009B1A69009BDA60E6
:10C3F000009B0022DA61009B00225A62079A06998C
:10C400000098FFF753FF1BE0009B93F8293083F05F
:10C410000103DBB2002B03D004210198FFF748FB96
:10C420004FF401710198FFF7EEFA009B00229A6128
:10C43000009B596A009BDB681A460098FFF736FF9D
:10C440004FF48E710198FFF7B2FA0346002B22D009
:10C45000009B1A6A009B5B699A420DD2009B93F87D
:10C460002830DBB283F00103DBB2002B04D000994B
:10C470000198FFF7E5FC0EE04FF48E710198FFF78D
:10C4800081FA009B5B69002B05D0009B5B69194614
:10C490000098FFF722FF4FF4A2710198FFF787FA87
:10C4A0000346002B1CD04FF4A2710198FFF76AFAE3
:10C4B000009B93F82930002B03D000210198FFF74F
:10C4C000F7FA009B9B69002B0AD0009B00229A611F
:10C4D000009B596A009BDB681A460098FFF7E6FE4E
:10C4E00000BF09B05DF804FB08B503490348FFF736
:10C4F0000EFF00BF08BD00BFBC330020002000407D
:10C5000082B003468DF807309DF8073003F01F0214
:10C5100005499DF907305B09012000FA02F241F854
:10C52000232000BF02B0704700E100E082B0034664
:10C5300000918DF807309DF90730002B0CDA009B35
:10C54000DAB20C499DF8073003F00F03043B5201A7
:10C55000D2B20B441A7609E0009BDAB206499DF983
:10C5600007305201D2B20B4483F8002300BF02B05F
:10C57000704700BF00ED00E000E100E082B00190F4
:10C58000019B03F06043B3F1005F0CBF0123002364
:10C59000DBB2184602B0704782B00190019B1B0BC2
:10C5A0005BB2184602B0704700B583B003460A4636
:10C5B0008DF8073013468DF806309DF80630012BB4
:10C5C00003D99DF80630032B0BD99DF80630042BB8
:10C5D00003D99DF80630072B03D908496B2000F0DA
:10C5E00093FE9DF806209DF9073011461846FFF787
:10C5F0009DFF00BF03B05DF804FB00BFD42703001C
:10C6000000B583B003468DF807309DF90730184612
:10C61000FFF776FF00BF03B05DF804FB84B0019024
:10C620000B46ADF80230BDF80230019A13440022E7
:10C630001A60BDF80230019A13441B680393039BF0
:10C6400000BF04B0704782B001900B46ADF80230D5
:10C65000BDF80230019A13441B68002B14BF01235C
:10C660000023DBB2184602B0704782B001900091FF
:10C67000019BD3F80022009B1A43019BC3F80022C0
:10C6800000BF02B0704782B001900091019BD3F8C7
:10C690000022009BDB431A40019BC3F8002200BF2D
:10C6A00002B0704782B001900091019B009AC3F8DC
:10C6B000042300BF02B0704782B001900091019B3B
:10C6C000009AC3F8082300BF02B0704784B00190FD
:10C6D000019BD3F880340393019B039AC3F8802411
:10C6E000039B184604B0704782B00190019B08225A
:10C6F000C3F8002500BF02B0704784B003900291D8
:10C700000192039B029AC3F80C25039B019AC3F87C
:10C71000142500BF04B0704784B0039002910192C9
:10C72000039B029AC3F80825039B019AC3F81025BE
:10C7300000BF04B0704782B001900B468DF8033003
:10C740009DF80330019A134401221A6000BF02B021
:10C75000704782B001900B468DF8033013468DF878
:10C7600002309DF803209DF802301343DBB21A46D5
:10C77000019BC3F86C2500BF02B0704782B00190E6
:10C780000091019B009AC3F8242500BF02B07047B6
:10C7900084B0039002910192029A039BC3F844254E
:10C7A000039B019AC3F8482500BF04B0704782B0CC
:10C7B0000190019BD3F84C35184602B0704784B005
:10C7C000039002910192029A039BC3F83425039BC4
:10C7D000019AC3F8382500BF04B0704782B00190B9
:10C7E000019BD3F83C35184602B0704700B583B0C2
:10C7F0000190019B1B682F2B04D90B494FF4F37058
:10C8000000F082FD019B1B681F2B02D84FF0A04354
:10C8100006E0019B1B6803F01F02019B1A60034B9B
:10C82000184603B05DF804FB042803000003005021
:10C8300000B585B00190084611461A4603468DF8AA
:10C8400003300B468DF8023013468DF8013001ABF2
:10C850001846FFF7CBFF03909DF803209DF80230A8
:10C860005B001A439DF801309B001A439DF8183075
:10C870001B0242EA03019DF81C301B04019A194374
:10C88000039B02F5E07243F8221000BF05B05DF88B
:10C8900004FB00B585B003900023019300230093AF
:10C8A0000023012201210398FFF7C2FF00BF05B05A
:10C8B0005DF804FB00B585B003900B468DF80B3096
:10C8C0009DF80B30002201920022009200220021EC
:10C8D0000398FFF7ADFF00BF05B05DF804FB00B59E
:10C8E00085B0019001AB1846FFF780FF0390019BD4
:10C8F000012202FA03F31946039800F004F800BF7E
:10C9000005B05DF804FB82B001900091019B009A94
:10C91000C3F8082500BF02B0704700B583B001908E
:10C920000091009B1B68B3F1FF3F09D0009B1B687F
:10C930001846FFF7D4FF009B1B681846FFF7A9FFB6
:10C94000009B5B68B3F1FF3F05D0009B5B68002153
:10C950001846FFF7AFFF019B1A68009B9B691946B9
:10C960001046FFF70BFF019B1868009B597D009B49
:10C970001B7D1A46FFF7EDFE019B1868009B1968A6
:10C98000009B5B681A46FFF7B8FE009B1B7D012BDE
:10C9900022D1009B9B68B3F1FF3F05D0009B9B68B1
:10C9A00000211846FFF786FF009BDB68B3F1FF3FCD
:10C9B00009D0009BDB681846FFF791FF009BDB68FE
:10C9C0001846FFF766FF019B1868009BD968009B1B
:10C9D0009B681A46FFF7A0FE00BF03B05DF804FB9A
:10C9E00000B583B001900B468DF80330019B1B68A6
:10C9F0004FF488711846FFF711FE019B1B684FF436
:10CA000090711846FFF70AFE019B1B684FF4927164
:10CA10001846FFF703FE019B1B684FF4A2711846EE
:10CA2000FFF7FCFD019B1B680E491846FFF73AFE15
:10CA3000019B1B681846FFF7AFFD03461A469DF899
:10CA4000033019461046FFF7AFFD019B1B681846DF
:10CA5000FFF7A2FD03461846FFF7D2FD00BF03B063
:10CA60005DF804FB1003020000B587B0039002914B
:10CA70000192029B002B03D12B49CD2000F044FCF6
:10CA8000039B1B791A461346DB0013449B00274A7D
:10CA90001344049300230593049B93F82030002B48
:10CAA00003D008230593059B3AE0039B1A68039B78
:10CAB0001B7919461E4B53F8213019461046FEF7D4
:10CAC0009FFE0346002B03D011230593059B27E00F
:10CAD00002990398FFF721FF049B019A5A60029B79
:10CAE0001A69049B1A60049B5B68002B05D0029BAB
:10CAF0001B7F19460398FFF773FF039B1B681846BB
:10CB0000FFF7F2FD049B00229A61049B0022DA6188
:10CB1000049B00225A61049B012283F82020059B7C
:10CB2000184607B05DF804FB3C280300E8330020FA
:10CB30008C28030000B589B0039002910192039BF9
:10CB40001B791A461346DB0013449B004C4A1344DE
:10CB50000493049B93F82030012B04D049494FF4EF
:10CB6000927000F0D1FB029B002B04D1454940F2AA
:10CB7000251000F0C9FB019B002B04D141494FF463
:10CB8000937000F0C1FB039B1B79002B03D1019B29
:10CB9000B3F5803F04D33B4940F2271000F0B4FBCB
:10CBA0000298FFF7EBFC034683F00103DBB2002B96
:10CBB00003D010230693069B5EE0039800F064F810
:10CBC0000346002B03D011230693069B54E0049BDD
:10CBD000019A5A61049B029A9A6000230693039B70
:10CBE0001B684FF490711846FFF718FD039B1B68F4
:10CBF0004FF4AC711846FFF711FD039B1868049BB6
:10CC00009968049B5B691A46FFF7C2FD039B1B688A
:10CC100008211846FFF78FFD049B5B68002B2AD183
:10CC2000039B1B684FF490711846FFF70CFD0346F9
:10CC30008DF81730039B1B684FF4AC711846FFF753
:10CC400002FD03468DF81F309DF8173083F0010375
:10CC5000DBB2002B06D09DF81F3083F00103DBB25E
:10CC6000002BDDD19DF81F30002B01D00F23069340
:10CC7000049B00225A61069B184609B05DF804FB2C
:10CC8000E83300203C28030082B00190019B1B790F
:10CC90001946084A0B46DB000B449B00134414332F
:10CCA0001B68002B14BF01230023DBB2184602B01F
:10CCB000704700BFE833002000B589B003900291AF
:10CCC0000192039B1B791A461346DB0013449B0019
:10CCD000864A13440593039B1B791946834A0B46E6
:10CCE000DB000B449B00134420331B78012B04D042
:10CCF0007F494FF4B77000F007FB029B002B04D173
:10CD00007B4940F26F1000F0FFFA019B002B04D129
:10CD100077494FF4B87000F0F7FA039B1B79002BAA
:10CD200003D1019BB3F5803F04D3714940F27110E8
:10CD300000F0EAFA0298FFF721FC034683F00103B2
:10CD4000DBB2002B03D010230693069BCAE000231E
:10CD50008DF81F30059B5B68002B06D0039B1B687A
:10CD60004FF404711846FFF7A7FC059B9B69002B45
:10CD700015D0059BDB69002B0ED0059B5B68002B53
:10CD800006D0039B1B684FF404711846FFF78AFC1A
:10CD900011230693069BA5E001238DF81F309DF813
:10CDA0001F3083F00103DBB2002B09D0059B019AF1
:10CDB0009A61059B029ADA60059B0022DA6105E020
:10CDC000059B029A1A61059B019ADA61002306937A
:10CDD000039B1B684FF488711846FFF71FFC039BE9
:10CDE0001B684FF4A2711846FFF718FC039B1B68E1
:10CDF000019A02991846FFF7E2FC9DF81F3083F074
:10CE00000103DBB2002B06D0039B1B6800211846F0
:10CE1000FFF791FC05E0039B1B6820211846FFF7F4
:10CE200024FC039B1B791946304A0B46DB000B445C
:10CE30009B00134404331B68002B4BD1039B1B68DE
:10CE40004FF488711846FFF7FEFB03468DF8133048
:10CE5000039B1B684FF4A2711846FFF7F4FB0346CF
:10CE60008DF81230039B1B684FF492711846FFF740
:10CE7000EAFB03468DF811309DF8133083F001036F
:10CE8000DBB2002B0DD09DF8123083F00103DBB232
:10CE9000002B06D09DF8113083F00103DBB2002B8C
:10CEA000CCD1039B1B791946104A0B46DB000B447F
:10CEB0009B001344183300221A609DF81130002B98
:10CEC00001D0032306939DF81230002B09D00F23C5
:10CED000069306E0039B1B684FF404711846FFF7A6
:10CEE000E1FB069B184609B05DF804FBE83300201F
:10CEF0003C28030000B589B0039002910192012300
:10CF00008DF81030029B0693019B0593039B5B6891
:10CF1000039A116804AA1046984700BF09B05DF84B
:10CF200004FB00B587B00190009100238DF8083014
:10CF3000009B0493019B9B680393019B00225A6111
:10CF4000019B5B68019A116802AA1046984700BFCE
:10CF500007B05DF804FB00B589B0019000914FF473
:10CF600092710198FFF76FFB0346002B22D04FF41C
:10CF700092710198FFF752FB02238DF80830019857
:10CF8000FFF7A4FB034605930198FFF727FC034630
:10CF90000493009BDB680393009B00229A61009B33
:10CFA0000022DA61009B5B68009A116802AA1046B1
:10CFB00098473BE04FF488710198FFF744FB034624
:10CFC000002B33D04FF488710198FFF727FB0198AD
:10CFD000FFF704FC0790009B9B69079A9A4225D1B2
:10CFE000009BDB69002B17D0009BDB680693202198
:10CFF0000198FFF748FB009BDA69009B9A61009B50
:10D000001A69009BDA60009B0022DA61069A079990
:10D010000098FFF76FFF09E0009B00229A61009BD8
:10D02000DB681A4607990098FFF764FF4FF4A27176
:10D030000198FFF708FB0346002B18D04FF4A271AC
:10D040000198FFF7EBFA009B9B69002B0FD0009B28
:10D0500000229A61009B0022DA610198FFF7BEFB73
:10D060000146009BDB681A460098FFF743FF4FF428
:10D0700090710198FFF7E7FA0346002B10D04FF4A8
:10D0800090710198FFF7CAFA009B5B69002B07D0EB
:10D090000198FFF78CFB034619460098FFF741FF04
:10D0A00000BF09B05DF804FB08B503490348FFF76A
:10D0B00052FF00BF08BD00BFE83300200020004041
:10D0C00084B001900B468DF8033013468DF8023082
:10D0D00000230393019B032B3CD89DF80230012BC6
:10D0E0000BD19DF80330012B04D1019BDBB20E3331
:10D0F000DBB200E000238DF802309DF80330022BF4
:10D100000FD0022B23DC002B16D0012B1FD114498A
:10D11000019A13465B0013440B449DF802201A70D9
:10D120001AE00F49019A13465B0013440B44013384
:10D130009DF802201A700FE00949019A13465B001E
:10D1400013440B4402339DF802201A7004E00723B5
:10D15000039301E007230393039B184604B0704731
:10D160000C34002000B583B0012200210020FFF71D
:10D17000A7FF0190019B002B04D0019B072B01D03E
:10D18000019B1CE0072202210120FFF799FF01907B
:10D19000019B002B04D0019B072B01D0019B0EE0CB
:10D1A000042202210020FFF78BFF0190019B002B3E
:10D1B00004D0019B072B01D0019B00E000231846FF
:10D1C00003B05DF804FB00B583B00122022100200A
:10D1D000FFF776FF0190019B002B04D0019B072BEA
:10D1E00001D0019B1CE0072202210120FFF768FF0C
:10D1F0000190019B002B04D0019B072B01D0019BC8
:10D200000EE00A2200210020FFF75AFF0190019B47
:10D21000002B04D0019B072B01D0019B00E00023D1
:10D22000184603B05DF804FB00B585B0019000918D
:10D23000019B1B88102B02D0112B18D02FE01A4B0A
:10D240001B68002B0DD1FFF78DFF0390039B002B74
:10D2500007D0164B1B68002B03D0144B1B68039898
:10D260009847114B1B6801330F4A136017E00E4BB0
:10D270001B68013B0C4A13600B4B1B68002B0DD144
:10D28000FFF7A1FF0390039B002B07D0074B1B6800
:10D29000002B03D0054B1B680398984700BF00BFC5
:10D2A00005B05DF804FB00BF1C34002018340020DA
:10D2B00072DF704700BF184673DF704700BF184623
:10D2C00076DF704700BF184677DF704700BF18460B
:10D2D0007ADF704700BF18467CDF704700BF1846F2
:10D2E0007FDF704700BF18468FDF704700BF1846CA
:10D2F000B1DF704700BF184632DF704700BF1846E5
:10D300003FDF704700BF184600B583B00346009169
:10D31000ADF80630BDF80630009A19460348FAF712
:10D320000BFC00BF03B05DF804FB00BFEFBEADDE39
:10D3300000B583B0FBF790FA0190019B0093009B2E
:10D34000002B04D0044AEE210098FAF7F5FB00BF49
:10D3500003B05DF804FB00BF9028030000B587B060
:10D360009DF80030012262F303038DF800309DF830
:10D370000030012262F307138DF800306B4609225A
:10D380001B491846FFF7A8FF0590059B0493049BD3
:10D39000002B05D0174A40F201110498FAF7CCFB94
:10D3A00001AB08220021184603F084FE0623ADF8E5
:10D3B00004300623ADF806300023ADF808304FF4F2
:10D3C000C873ADF80A3001AB1846FFF781FF05902E
:10D3D000059B0393039B002B05D0064A40F20B11DB
:10D3E0000398FAF7A9FB00BF07B05DF804FB00BF84
:10D3F000E42803009028030000B583B00190054A9B
:10D400004FF48C710198FAF797FB00BF03B05DF8F9
:10D4100004FB00BF9028030000B587B00190019B7A
:10D420001B78002B44D1002305932BE0019B1A6944
:10D43000059B13441B781846FBF7ACFC0490049B37
:10D44000002B19D0049B112B16D01B4A1B4BD31A4F
:10D45000DB081B0443F00103049A19491846F9F745
:10D460003DFC049B0393039B002B05D0154A4FF40E
:10D470009B710398FAF760FB049B112BD6D0059B98
:10D4800001330593019B9B8A1A46059B9342CDD39A
:10D49000019B1A69019B9B8A013B13441B780D2B4E
:10D4A00006D100BF0A20FBF775FC0346112BF9D00B
:10D4B00000BF07B05DF804FB6819030040190300C2
:10D4C000F02803009028030000B587B000230193E3
:10D4D000174B019301AB1946164802F011FD059058
:10D4E000059B0493049B002B05D0134A4FF4A871AD
:10D4F0000498FAF721FB02AB04220021184603F03E
:10D50000D9FD0E4B029302AB19460D4802F03AFFCB
:10D510000590059B0393039B002B05D0064A4FF40F
:10D52000AC710398FAF708FB00BF07B05DF804FB85
:10D53000F9D30200383400209028030019D40200E7
:10D54000F82A002000B585B00190019B1B78002BC4
:10D5500011D10B4B1B883B211846FFF7B1FE0390FE
:10D56000039B0293029B002B05D0064A4FF4B77130
:10D570000298FAF7E1FA00BF05B05DF804FB00BFBE
:10D58000142B00209028030000B583B00190054AB9
:10D5900040F279110198FAF7CFFA00BF03B05DF8B5
:10D5A00004FB00BF9028030000B58BB001AB1C2228
:10D5B0000021184603F07EFD002301934FF4203331
:10D5C00002934FF47023039303238DF8103000234C
:10D5D000ADF8123000238DF814300C4B06930C4B31
:10D5E000079301AB184601F067FC0990099B08936B
:10D5F000089B002B05D0074A4FF4C8710898FAF72A
:10D600009BFA00BF0BB05DF804FB00BF45D50200DC
:10D6100089D502009028030000B58BB001900091DD
:10D62000019B1B88562B00F0C780562B00F3D78038
:10D63000522B00F09A80522B00F3D180212B2DDC4D
:10D64000102BC0F2CC80103B112B00F2C88001A23D
:10D6500052F823F0A3D60200EFD60200DFD7020073
:10D6600043D70200DFD70200DFD70200DFD7020076
:10D67000DFD70200DFD70200DFD70200DFD70200CA
:10D68000DFD70200DFD70200DFD70200DFD70200BA
:10D69000DFD70200DFD702000FD702003B2B78D084
:10D6A0009DE0574A574BD31ADB081B0443F0030392
:10D6B00055491846F9F704FB544B00221A70019B98
:10D6C0009A88534B1A80524B1B881946514802F0D6
:10D6D00039FC0990099B0393039B002B00F0818088
:10D6E0004D4A40F2D3110398FAF726FA79E0444AFA
:10D6F000444BD31ADB081B0443F003034749184685
:10D70000F9F7DEFA424B4FF6FF721A8074E00023FD
:10D710008DF8083000238DF80930019B9B8802AA00
:10D7200011461846FFF7E0FD0990099B0593059BFC
:10D73000002B58D0384A40F2E5110598FAF7FCF969
:10D7400051E0334B1888002300228521FFF7C8FDE4
:10D750000990099B0493049B002B46D02E4A40F26B
:10D76000EB110498FAF7E8F93FE0294B18880023F9
:10D7700000220021FFF7BCFD0990099B0793079B3E
:10D78000002B34D0244A40F2F1110798FAF7D4F96B
:10D790002DE0019B9B8813211846FFF791FD09900E
:10D7A000099B0693069B002B23D01B4A4FF4FC7168
:10D7B0000698FAF7C1F91CE0019B9B8813211846D3
:10D7C000FFF77EFD0990099B0893089B002B12D060
:10D7D000114A40F2FF110898FAF7AEF90BE000BFCA
:10D7E0000AE000BF08E000BF06E000BF04E000BFA1
:10D7F00002E000BF00E000BF00BF0BB05DF804FB1B
:10D8000068190300401903001C2903004434002058
:10D81000142B00203834002090280300282903000E
:10D8200000B589B002F0F2FF0790079B0693069BB4
:10D83000002B05D0254A40F212210698FAF77CF910
:10D840000023019301AB1946012003F097F80790DC
:10D85000079B0593059B002B05D01C4A4FF40671CE
:10D860000598FAF769F901AB184603F0A5F9079096
:10D87000079B0493049B002B05D0144A4FF40771B7
:10D880000498FAF759F90120FFF736FD0790079B36
:10D890000393039B002B05D00C4A40F21F210398F1
:10D8A000FAF74AF90120FFF72BFD0790079B029337
:10D8B000029B002B05D0054A40F222210298FAF77C
:10D8C0003BF900BF09B05DF804FB00BF90280300DE
:10D8D00000B583B001900091009B5A88114B1B88C2
:10D8E0009A421AD1009B1B8840F67722934214D1AA
:10D8F000009B9B88033B9AB20B4B1A800B4A0C4B44
:10D90000D31ADB081B0443F00300074B1B881A469D
:10D91000054B1B880749F9F7F2F900BF03B05DF822
:10D9200004FB00BF142B0020162B002068190300F5
:10D93000401903003829030000B585B01149124889
:10D9400002F0DEF90390039B0293029B002B05D0AB
:10D950000E4A40F23D210298FAF7EEF8F7210A4804
:10D9600002F0F9F90390039B0193019B002B05D072
:10D97000064A4FF410710198FAF7DEF800BF05B0BF
:10D980005DF804FBD1D80200243400209028030065
:10D9900000B583B003460A468DF8073013468DF86C
:10D9A00006309DF807300B3B0E2B24D801A252F80D
:10D9B00023F000BF09DA020009DA0200F7D90200F9
:10D9C000F7D90200F7D90200F7D90200F7D902000F
:10D9D000F7D90200F7D90200F7D90200F7D90200FF
:10D9E000F7D90200F7D9020009DA0200F1D90200E2
:10D9F00000F0DAF909E09DF80730064A40F29F216D
:10DA00001846FAF799F800E000BF00BF03B05DF8D0
:10DA100004FB00BF9028030000B583B040F26662AB
:10DA200004210948F9F7BEFF0190019B0093009B78
:10DA3000002B05D0054A40F2B6210098FAF77CF891
:10DA400000BF03B05DF804FB442B002090280300C6
:10DA500000B587B00190019B1B78022B56D0022B9A
:10DA600066DC002B02D0012B59D061E0344B1B78CF
:10DA70001A46344B13441846FBF752F9304B1B78C7
:10DA80000133DAB22E4B1A702D4B1B78013B2D4A15
:10DA9000D35C0A2B0DD02A4B1B78013B294AD35C5F
:10DAA0000D2B06D0264B1B789AB2274B1B889A4227
:10DAB00040D3234B1B78012B24D9214B1B789BB2DD
:10DAC000ADF80E30214B1B880DF10E021D49204888
:10DAD00002F0FEFC0590059B082B10D0059B132B34
:10DAE0000DD0059B052B0AD0059B0493049B002BAE
:10DAF00005D0184A40F2DE210498FAF71DF8059B7C
:10DB0000132BDAD00E4B00221A7013E0019B5B68D6
:10DB1000104A4FF43A711846FAF70EF80BE0019BE1
:10DB20005B680C4A4FF43B711846FAF705F802E0BF
:10DB300000BF00E000BF00BF07B05DF804FB00BFFE
:10DB40008734002088340020162B0020142B00205E
:10DB5000F82A00209028030030B58DB0134B04AC98
:10DB60001D460FCD0FC495E8030084E80300104B59
:10DB700000934FF4807301930E4B02934FF4807324
:10DB80000393694604A807230B4AFBF739F80B9067
:10DB90000B9B0A930A9B002B05D0084A40F21131D7
:10DBA0000A98F9F7C9FF00BF0DB030BD5429030032
:10DBB0007C3500207C36002051DA020090280300DA
:10DBC00000B5ADB018AB3C220021184603F072FA44
:10DBD00000238DF8623006238DF8633018AB3C22A9
:10DBE0000021184603F066FA5923ADF818301323C4
:10DBF000ADF81C30444B089306AB219302238DF8FB
:10DC0000603000238DF8623006238DF8633009AB55
:10DC10003C220021184603F04DFA6B4618220021E1
:10DC2000184603F047FA394B196818AB384A1846BA
:10DC300000F0FDFE2B902B9B2A932A9B002B05D0F6
:10DC4000344A40F25E312A98F9F776FF2F4B9968F3
:10DC500009AB314A184600F0EAFE2B902B9B299322
:10DC6000299B002B05D02B4A40F263312998F9F704
:10DC700063FF2A4A2A4BD31ADB081B0443F0030331
:10DC8000224A1168214A92881846F9F767F8042356
:10DC90008DF8153004238DF8163006238DF80030EA
:10DCA0000023ADF80C300023019300238DF81430CD
:10DCB000202302936B461A4614491A48FFF7F8FAD4
:10DCC0002B902B9B2893289B002B05D0114A4FF4B7
:10DCD0005F712898F9F730FF124B1B789BB208222E
:10DCE00019460120FFF7F0FA2B902B9B2793279BD7
:10DCF000002B05D0074A40F27F312798F9F71CFF27
:10DD000000BF2DB05DF804FB182B0020342B002041
:10DD1000382B002090280300402B002068190300B6
:10DD200040190300302B002000B583B04FF40041B0
:10DD30000020F8F7E5FC0190019B0093009B002B6D
:10DD400005D0064A40F28B310098F9F7F5FEF8F756
:10DD50006DFC00BF03B05DF804FB00BF902803001A
:10DD600000B583B0FCF7CEF80190019B0093009BB7
:10DD7000002B05D0044A40F297310098F9F7DCFEF9
:10DD800000BF03B05DF804FB9028030008B5F9F765
:10DD900095F8034683F00103DBB2002B01D0FCF7BA
:10DDA000C7F800BF08BD000000B583B00F4B1B785B
:10DDB00083F00103DBB2002B14D00D4B1B78012143
:10DDC0001846FFF779FA0190019B0093009B002B06
:10DDD00005D0084A40F2B9310098F9F7ADFE034B7F
:10DDE00001221A7000BF03B05DF804FB4434002028
:10DDF000302B00209028030008B5FFF7ADFEFFF799
:10DE000093FFFFF795FAFFF707FEFFF7A9FFFFF76C
:10DE100007FDFFF7A3FAFFF78FFDFFF755FBFFF7AD
:10DE2000CFFEFFF7C1FB044803F04CFAFFF7BCFF3D
:10DE3000FFF7ACFFFCE700BF6C29030082B0204B6A
:10DE40000193019B02221A61019B02225A61019BEC
:10DE50001C4A9A61019B1C4ADA61019B4FF40072D3
:10DE60001A62019B00229A62019B00225A62019B66
:10DE70000022DA62019B134A9A64019B134ADA6416
:10DE8000019B10221A65019B00229A65019B0022CA
:10DE90005A65019B0022DA65019B07330C4A106822
:10DEA0001860019B0B4A10681860918892799980DC
:10DEB0009A71019B20229A7100BF02B0704700BF87
:10DEC0007C3700208C290300F4370020F43900202F
:10DED000982903009C29030000B589B003900291A2
:10DEE000019200230693039BDB680593039B1B6948
:10DEF0000493049A059B9A4205D9049A059BD31A68
:10DF0000013B079307E0039B9A680499059BCB1A92
:10DF10001344013B0793039B9A68059BD31A079A06
:10DF2000934228BF13460793079A019B934228BF49
:10DF300013460793039B5A68059B1344079A02995B
:10DF4000184603F081F8069A079B13440693029A39
:10DF5000079B13440293019A079BD31A0193059AD6
:10DF6000079B13440593039B9B68059A9A4201D132
:10DF700000230593039B059ADA60019B002BB5D122
:10DF8000069B184609B05DF804FB00B589B0039004
:10DF900002910192039BDB680793039B9A68079B9E
:10DFA000D31A0693069A019B9A420ED9039B5A688C
:10DFB000079B1344019A0299184603F045F8079A03
:10DFC000019B1A44039BDA601AE0069B0593039BAE
:10DFD0005A68079B1344059A0299184603F034F8CF
:10DFE000019A069BD31A0593039B5868029A069BD5
:10DFF0001344059A194603F027F8039B059ADA6043
:10E0000000BF09B05DF804FB86B00190019B1B695D
:10E010000493019BDB680393049A039B9A4208D8FC
:10E02000019B9A68039BD21A049B1344013B0593FE
:10E0300004E0049A039BD31A013B0593059B184601
:10E0400006B0704700B589B0039002910192029B1F
:10E050000693039B5A1C13465B001344DB00204AC3
:10E0600013440593059B5B69022B29D0022B2ED804
:10E07000002B02D0012B13D029E00598FFF7C4FF35
:10E080000490049A019B9A4202D20023079321E054
:10E09000019B0793019A06990598FFF776FF19E00F
:10E0A0000598FFF7B1FF0490019A049B934228BFA3
:10E0B00013460793079A06990598FFF766FF09E04C
:10E0C000019A06990598FFF707FF079002E00023E1
:10E0D000079300BF079B184609B05DF804FB00BF1B
:10E0E0007C37002000B587B00390029101920F4B5E
:10E0F0001B78002B01D1FFF7A1FE00238DF8133010
:10E100000DF113031846FAF7E9FE019A02990398F4
:10E11000FFF798FF05909DF813301846FAF7F4FEC4
:10E12000059B184607B05DF804FB00BF7C37002054
:10E1300008B5FFF783FE00BF08BD6DDF704700BF65
:10E14000184679DF704700BF18467DDF704700BF73
:10E15000184664DF704700BF184682B0034600913E
:10E16000ADF80630BDF80630DAB2009B1A70BDF883
:10E1700006301B0A9AB2009B0133D2B21A700223F6
:10E18000184602B0704700B589B00390029113465B
:10E19000ADF80630029B1B8803F10902BDF806307A
:10E1A0009A4201D90C2353E004AB1846FFF7C5FF90
:10E1B0000790079B0693069B002B01D0069B47E028
:10E1C000029B1B881A46039B134408221A70029B69
:10E1D0001B8801339AB2029B1A80029B1B881A4645
:10E1E000039B13441B221A70029B1B8801339AB2B3
:10E1F000029B1A80029B1B881A46039B981804AB4B
:10E2000001330622194602F01FFF029B1B880633CA
:10E210009AB2029B1A809DF8103023F00103DBB202
:10E22000002B07D1029B1B881A46039B1344002234
:10E230001A7006E0029B1B881A46039B13440122B6
:10E240001A70029B1B8801339AB2029B1A8000232A
:10E25000184609B05DF804FB00B589B0039002913F
:10E260000192ADF80230039B1B78012B05D1039B73
:10E270005B78002B01D1072392E0019B1B889A1C3D
:10E28000BDF802309A420ED8039B1B78012B0CD1AB
:10E29000019B1B881A46039B5B7813449A1CBDF8AC
:10E2A00002309A4201D90C237AE0019B1B88BDF809
:10E2B0000220D31A9BB2023BADF81C30BDF81C30D3
:10E2C000ADF81230019B1B880233029A13440DF102
:10E2D000120211461846FFF738FF0690069B059379
:10E2E000059B002B01D0059B5AE0039B1B78022B5A
:10E2F00006D0039B5B789AB2BDF812309A4209D3DC
:10E30000BDF81230BDF81C209A4203D309238DF8C2
:10E310001F3017E008238DF81F30039B1B78012B5B
:10E320000CD1039B5B789BB2BDF81C209A4205D3AD
:10E33000039B5B789BB2ADF8123003E0BDF81C3054
:10E34000ADF81230BDF81230FE2B01D90C2327E0B6
:10E35000BDF81230DAB2019B1B881946029B0B44B0
:10E360000132D2B21A70019B1B8801339AB2019B11
:10E370001A80019B1B881A46029B13449DF81F209C
:10E380001A70019B1B8801339AB2019B1A80019B72
:10E390001A88BDF8123013449AB2019B1A800023E8
:10E3A000184609B05DF804FB00B589B003900291EE
:10E3B0001346ADF80630029B1B881A1DBDF80630C7
:10E3C0009A4201D90C233BE00DF116031846FFF7E2
:10E3D000B8FE0790079B0693069B002B01D0069B77
:10E3E0002EE0029B1B881A46039B134403221A70DB
:10E3F000029B1B8801339AB2029B1A80029B1B88E6
:10E400001A46039B134419221A70029B1B8801337E
:10E410009AB2029B1A80BDF81620029B1B881946EF
:10E42000039B0B4419461046FFF797FE0346194617
:10E43000029B1A888BB213449AB2029B1A80002363
:10E44000184609B05DF804FB84B0029101921A46A7
:10E4500003468DF80F301346ADF80C30019B1B8836
:10E46000DA1CBDF80C309A4201D90C2328E0019B3C
:10E470001B881A46029B134402221A70019B1B88B8
:10E4800001339AB2019B1A80019B1B881A46029B9A
:10E49000134401221A70019B1B8801339AB2019B1D
:10E4A0001A80019B1B881A46029B13449DF80F207B
:10E4B0001A70019B1B8801339AB2019B1A800023BA
:10E4C000184604B0704784B0029101921A46034680
:10E4D0008DF80F301346ADF80C30019B1B88DA1C09
:10E4E000BDF80C309A4201D90C2328E0019B1B880F
:10E4F0001A46029B134402221A70019B1B880133A7
:10E500009AB2019B1A80019B1B881A46029B1344F6
:10E510000A221A70019B1B8801339AB2019B1A8050
:10E52000019B1B881A46029B13449DF80F201A700A
:10E53000019B1B8801339AB2019B1A800023184665
:10E5400004B0704700B58FB0039001930B468DF86F
:10E550000B3013468DF80A3000238DF83330109BB2
:10E560001B88ADF8303000230D9371E0039B5A688F
:10E570000D9B9B001A4405AB106818600DF11B0140
:10E5800005AB00221846FFF7E4FD0A900A9B0993A9
:10E59000099B002B01D0099B7CE09DF81B309DF866
:10E5A0000A209A4251D19DF83330002B01D000232C
:10E5B00000E002238DF82330109B1B881A469DF83B
:10E5C0001B301A449DF823301A44BDF844309A4257
:10E5D00001DD0C235EE09DF8333083F00103DBB2F4
:10E5E000002B16D0109B1B8801339AB2109B1A8007
:10E5F000109B1B881A46019B13449DF80B201A7030
:10E60000109B1B8801339AB2109B1A8001238DF84E
:10E610003330109B1B881A46019B1A440DF11B01D5
:10E6200005AB1846FFF795FD0A900A9B0793079BD9
:10E63000002B01D0079B2DE0109B1A889DF81B3002
:10E640009BB213449AB2109B1A800D9B01330D9319
:10E65000039B1B881A460D9B934287DB9DF8333042
:10E66000002B16D0109B1A88BDF83030D31A9BB2FD
:10E67000013BADF82E30BDF82E30FF2B01D90C2315
:10E6800008E0BDF83030019A1344BDF82E20D2B214
:10E690001A70002318460FB05DF804FB00B58BB06C
:10E6A000059003930B468DF8133013468DF8123006
:10E6B0009DF81310BDF8343001930C9B0093039B1D
:10E6C00002220598FFF73EFF0990099B0893089BDB
:10E6D000002B01D0089B14E09DF81210BDF83430D7
:10E6E00001930C9B0093039B10220598FFF72AFFD0
:10E6F0000990099B0793079B002B01D0079B00E023
:10E70000002318460BB05DF804FB82B00190019B1A
:10E710001B88052B0AD9019B1B88B3F5486F07D9C5
:10E72000019B1B884FF6FF72934201D0072325E01F
:10E73000019B5B88052B0AD9019B5B88B3F5486F69
:10E7400007D9019B5B884FF6FF72934201D00723E4
:10E7500014E0019B1B884FF6FF7293420DD0019B82
:10E760005B884FF6FF72934207D0019B1A88019B8A
:10E770005B889A4201D9072300E00023184602B0C3
:10E78000704700B587B0039002910192ADF8023056
:10E79000019B1B889A1DBDF802309A4201D90C23B7
:10E7A0004DE00398FFF7B1FF0590059B0493049B90
:10E7B000002B01D0049B42E0019B1B881A46029B60
:10E7C000134405221A70019B1B8801339AB2019BE6
:10E7D0001A80019B1B881A46029B134412221A704E
:10E7E000019B1B8801339AB2019B1A80039B1A88F4
:10E7F000019B1B881946029B0B4419461046FFF7E4
:10E80000ACFC03461946019B1A888BB213449AB29A
:10E81000019B1A80039B5A88019B1B881946029B07
:10E820000B4419461046FFF798FC03461946019B16
:10E830001A888BB213449AB2019B1A80002318469F
:10E8400007B05DF804FB00B587B003900291019218
:10E85000ADF80230039B9B8802330593019B1B8814
:10E860001A46059B13449A1CBDF802309A4201D9FE
:10E870000C2354E0059BFE2B01D90C234FE0059B94
:10E88000DAB2019B1B881946029B0B440132D2B2BB
:10E890001A70019B1B8801339AB2019B1A80019B5D
:10E8A0001B881A46029B1344FF221A70019B1B8887
:10E8B00001339AB2019B1A80039B1A88019B1B8823
:10E8C0001946029B0B4419461046FFF746FC0346C7
:10E8D0001946019B1A888BB213449AB2019B1A8085
:10E8E000039B9B88002B19D0039B9B68002B01D1B5
:10E8F000072314E0019B1B881A46029B9818039B70
:10E900009968039B9B881A4602F09EFB019B1A881C
:10E91000039B9B8813449AB2019B1A8000231846DC
:10E9200007B05DF804FB00B589B003900291019235
:10E93000ADF80230039B9B6A002B01D1072372E0E4
:10E9400000238DF81F3066E0039B996A9DF81F2015
:10E9500013465B0013449B000B440693069B9B8865
:10E9600002330593059BFE2B01D90C235BE0059B2D
:10E97000DAB2019B1B881946029B0B440132D2B2CA
:10E980001A70019B1B8801339AB2019B1A80019B6C
:10E990001B881A46029B134416221A70019B1B887F
:10E9A00001339AB2019B1A80069B1A88019B1B882F
:10E9B0001946029B0B4419461046FFF7CEFB03464F
:10E9C0001946019B1A888BB213449AB2019B1A8094
:10E9D000069B9B88002B19D0069B9B68002B01D1BE
:10E9E000072320E0019B1B881A46029B9818069B70
:10E9F0009968069B9B881A4602F026FB019B1A88A1
:10EA0000069B9B8813449AB2019B1A809DF81F3085
:10EA100001338DF81F30039B93F82C309DF81F2095
:10EA20009A4291D30023184609B05DF804FB00B563
:10EA300095B005900491039200231393039B1B88C8
:10EA4000ADF84A30039B00221A80059B93F82D30C5
:10EA5000002B0ED0BDF84A301A4603990498FFF7F0
:10EA600092FB1390139B1193119B002B01D0119BD0
:10EA7000D8E0059B9B78002B0ED0BDF84A301A4693
:10EA800003990498FFF790FC1390139B1093109B2D
:10EA9000002B01D0109BC5E0059BDB78002B10D02C
:10EAA000059BDB7858B2BDF84A30039A0499FFF70A
:10EAB000CBFC1390139B0F930F9B002B01D00F9B4C
:10EAC000B0E0059B5B68002B11D0059B5B6893F958
:10EAD0000000BDF84A30039A0499FFF7F4FC139044
:10EAE000139B0E930E9B002B01D00E9B9AE0059B6F
:10EAF0001B89002B14D0059B03F10800BDF84A3098
:10EB00000193039B0093049B06220221FFF7C6FD9D
:10EB10001390139B0D930D9B002B01D00D9B81E057
:10EB2000059B1B8A002B14D0059B03F11000BDF838
:10EB30004A300193039B0093049B07220321FFF7B4
:10EB4000ADFD1390139B0C930C9B002B01D00C9BE1
:10EB500068E0059B1B8B002B14D0059B03F118006C
:10EB6000BDF84A300193039B0093049B15221421A6
:10EB7000FFF794FD1390139B0B930B9B002B01D07D
:10EB80000B9B4FE0059B1B6A002B0FD0059B186A5F
:10EB9000BDF84A30039A0499FFF7F3FD1390139BD5
:10EBA0000A930A9B002B01D00A9B3BE0059B5B6A02
:10EBB000002B0FD0059B586ABDF84A30039A049980
:10EBC000FFF741FE1390139B0993099B002B01D083
:10EBD000099B27E0059B93F82C30002B0ED0BDF845
:10EBE0004A30039A04990598FFF79DFE1390139BF2
:10EBF0000893089B002B01D0089B13E0059B1B7812
:10EC0000002B0ED0BDF84A30039A04990598FFF7FF
:10EC100023FB1390139B0793079B002B01D0079BAB
:10EC200000E0139B184615B05DF804FB75DF7047D4
:10EC300000BF184676DF704700BF18467ADF70477E
:10EC400000BF18467BDF704700BF184684B00346FC
:10EC5000ADF806300023039316E00F49039A1346DC
:10EC60009B0013449B000B441B88BDF806209A426E
:10EC700007D1039A13469B0013449B00064A134492
:10EC800006E0039B01330393039B002BE5D0002395
:10EC9000184604B0704700BF243A002082B00190AB
:10ECA0000B46ADF80230019BBDF802201A80019B93
:10ECB00000221A72019B054903F10A020B4603CB9D
:10ECC0001060516000BF02B0704700BF543A00208E
:10ECD00082B00190019B4FF6FF721A8000BF02B014
:10ECE000704788B00390029111461A460B46ADF862
:10ECF00006301346ADF80430039B9B881A46BDF8D6
:10ED0000063013440793039B9B881946039B9B88FB
:10ED1000BDF80620934228BF13469BB2CB1A069338
:10ED2000039BDB881A46BDF8043013440593039B0C
:10ED3000DB881946039BDB88BDF80420934228BF7B
:10ED400013469BB2CB1A0493029B5A88039B1B88E1
:10ED50009A4205D3029B5A88039B5B889A4201D949
:10ED600000231CE0029B9B881A46069B934205D811
:10ED7000029B9B881A46079B934201D200230EE018
:10ED8000029BDB881A46049B934205D8029BDB88D2
:10ED90001A46059B934201D2002300E00123184646
:10EDA00008B0704700B583B00190064B9B69002BFB
:10EDB00003D0044B9B690198984700BF03B05DF8EE
:10EDC00004FB00BF383A002000B585B0034600912F
:10EDD000ADF80630BDF8063000991846FFF726FF5B
:10EDE0000390039B002B05D0039B112B02D00398AB
:10EDF000FFF7D8FF039B002B0CBF01230023DBB2DE
:10EE0000184605B05DF804FB00B589B00190019B80
:10EE10000793079B9BB21846FFF718FF0690069BC7
:10EE2000002B42D0069B1A7A224B1B7B9A4215D2AA
:10EE3000079B9AB2069B0A3319461046FFF7C4FF98
:10EE400003468DF813309DF81330002B2DD0069B10
:10EE50001B7A0133DAB2069B1A7226E0069B002267
:10EE60001A72144B1B7C002B0FD0079B9BB23B21CB
:10EE70001846FFF7DFFE0590059B002B05D0059B8C
:10EE8000082B02D00598FFF78DFF0A4B5B69002B1A
:10EE90000BD000238DF80C30079B9BB2ADF80E30E1
:10EEA000044B5B6903AA1046984700BF09B05DF8A0
:10EEB00004FB00BF383A002030B587B00190019BB9
:10EEC000002B01D10E2353E02B4A019B14461D4613
:10EED0000FCD0FC495E8070084E80700264B274AAA
:10EEE0001A60019B1B68002B11D0019B1B68184600
:10EEF000FFF7A4FE0490049B002B01D0049B37E095
:10EF0000019B1A681D4B1068516803C308E01B4839
:10EF1000FFF798FE0490049B002B01D0049B27E090
:10EF20000023059320E0059A13469B0013449B00A1
:10EF3000134A134403930398FFF7CAFE059B5B0132
:10EF4000104A1A44039B5A60039B04330E4A002163
:10EF50001846F9F7B5FC0490049B002B01D003235D
:10EF600006E0059B01330593059B002BDBD00023B6
:10EF7000184607B030BD00BF383A0020543A002090
:10EF8000243A0020043A002009EE020000B587B0C0
:10EF900003460091ADF80630009B5B7A002B1AD136
:10EFA000009B1B7A002B03D1164B5B68059302E094
:10EFB000144B9B680593009B5B68BDF80620059980
:10EFC0001846F9F7ADFC0490049B002B16D004986A
:10EFD000FFF7E8FE12E0009B00221A72094B5B6902
:10EFE000002B0BD001238DF80C30BDF80630ADF8A6
:10EFF0000E30044B5B6903AA1046984700BF07B068
:10F000005DF804FB383A002000B585B00190019B03
:10F01000DB7B8DF80F30019B9B88ADF80C309DF8A1
:10F020000F30012B2CD14FF6FF70FFF70FFE02902F
:10F03000029B002B03D10420FFF7B4FE21E0BDF8B2
:10F040000C3019460298FFF729FE029B03F10A00D3
:10F05000019B03F110014FF6FF7340F2F312FFF72B
:10F0600040FE03461A46029B5A72074BDB89002B6F
:10F0700007D1BDF80C3002991846FFF787FF00E072
:10F0800000BF05B05DF804FB383A002000B587B03A
:10F090000190019B9B88ADF81630BDF816301846DC
:10F0A000FFF7D4FD0490049B002B0ED0049B5B68FB
:10F0B0001846F9F767FC0390039B002B02D00398D6
:10F0C000FFF770FE0498FFF703FE00BF07B05DF87E
:10F0D00004FB000000B587B00190019B0633059347
:10F0E000059B1A88194BDB899A422BD1059B5B89BA
:10F0F000022B27D1019B9B88ADF81230BDF812304E
:10F100001846FFF7A3FD0390039B002B1AD0059B25
:10F110000C33184600F036FA0346002B06D0BDF833
:10F12000123003991846FFF731FF0BE0039B5B6831
:10F130001846F9F727FC0290029B002B02D0029898
:10F14000FFF730FE00BF07B05DF804FB383A00203F
:10F1500000B585B00190019B9B88ADF80E30BDF8DD
:10F160000E301846FFF772FD0290029B002B15D05F
:10F17000029B03F10A00019B03F108014FF6FF73A4
:10F1800040F2F312FFF7ADFD03461A46029B5A7296
:10F19000BDF80E3002991846FFF7F8FE00BF05B023
:10F1A0005DF804FB00B583B001900091019B1B88C2
:10F1B000502B12D0502B18DC122B12D0122B14DC37
:10F1C000102B02D0112B04D00FE00198FFF71CFF89
:10F1D0000CE00198FFF75AFF08E00198FFF77AFF6B
:10F1E00004E00198FFF7B4FF00E000BF00BF03B0E8
:10F1F0005DF804FB30B58FB00190009100230293BD
:10F20000009B002B1AD000230D9314E06B460D9940
:10F210001846F9F7E1FE0346002B09D0029B5A1C61
:10F2200002920D9A92B25B0038336B4423F82C2C77
:10F230000D9B01330D930D9B132BE7D9019B1D46AD
:10F2400002AC0FCC0FC50FCC0FC594E8070085E8C2
:10F25000070001980FB030BD00B583B00346ADF88C
:10F260000630BDF80630132B01D900230CE0BDF8A1
:10F27000063019460648F9F77EFEBDF806301946F5
:10F280000448F9F778FE0123184603B05DF804FB43
:10F29000643A0020603A002000B585B00346ADF81E
:10F2A0000630002303930DE0039B9B00094A13449F
:10F2B0000433BDF8062011461846F9F774FE039B87
:10F2C00001330393039B1C2BEED900BF00BF05B095
:10F2D0005DF804FB5C3A002000B583B00346ADF84E
:10F2E0000630BDF8063019460348F9F75CFE00BF4A
:10F2F00003B05DF804FB00BF643A002030B59BB05A
:10F30000184B9B68DB431893164B5A6818AB114691
:10F310001846F9F7C0FE189A6B4611461846FFF7D3
:10F3200069FF0DAC6D460FCD0FC40FCD0FC495E82E
:10F33000070084E80700002319930BE0199B5B008A
:10F3400068336B4433F8303C1846FFF7A5FF199B30
:10F35000013319930D9B199A9A42EFD300BF00BF56
:10F360001BB030BD5C3A002000B585B00190009123
:10F37000019B9B88ADF80E30019B1B881A2B2AD06D
:10F380001A2B68DC102B02D0112B1ED063E0FFF784
:10F39000B5FFBDF80E301846FFF75EFF034683F059
:10F3A0000103DBB2002B05D02D4AE3210420F8F73E
:10F3B000C3FB4FE0019BDB7B012B4BD0BDF80E3034
:10F3C00019462848F9F7D7FD44E0BDF80E30184635
:10F3D000FFF782FF3FE0019B1B7AC3F30313DBB20D
:10F3E000012B8CBF012300238DF80D30019B1B7A6C
:10F3F000C3F30313DBB2022B8CBF012300238DF870
:10F400000C309DF80D30002B17D0BDF80E3019468A
:10F410001548F9F7B0FD9DF80C30002B06D0BDF86B
:10F420000E3019461148F9F7A6FD14E0BDF80E306C
:10F4300019460E48F9F7B7FD0DE0BDF80E30194634
:10F440000948F9F7B0FDBDF80E3019460748F9F73D
:10F45000AAFD00E000BF00BF05B05DF804FB00BFDF
:10F46000A4290300683A00206C3A0020703A00207A
:10F4700000B583B00346ADF80630BDF80630132B57
:10F4800001D9002306E0BDF8063019460348F9F714
:10F49000A3FD0346184603B05DF804FB603A002064
:10F4A00000B583B00346ADF80630BDF80630184607
:10F4B000FFF7DEFF0346002B02D0BDF8063000E068
:10F4C0001423184603B05DF804FB00B587B0039021
:10F4D0000B460192ADF80A30019B002B01D10E239F
:10F4E00038E0019B00221A60039B002B01D10E2300
:10F4F00030E0039B1B68002B01D10E232AE0039B05
:10F50000DB8803F003039BB2002B01D0072321E02B
:10F51000BDF80A301846FFF7C3FF03468DF81730D1
:10F520009DF81730142B01D1052313E0039B1B79A1
:10F530009DF817209A4201D304230BE0039B1B681C
:10F540009DF817200399C98801FB02F21A44019B18
:10F550001A600023184607B05DF804FB82B00190E2
:10F56000019B1B781AB2019B01331B781B021BB253
:10F5700013431BB29BB2184602B07047AADF704714
:10F5800000BF184600B585B001900198FFF7E6FF6F
:10F590000346ADF80E30BDF80E3003F00103002B2A
:10F5A00014BF01230023DBB2184605B05DF804FB4D
:10F5B00082B0034600918DF80730009A13786FF3FC
:10F5C00003031370009A13786FF3071313709DF8F9
:10F5D0000730052B5BD801A252F823F0F5F50200A5
:10F5E0000BF6020025F602003FF6020059F6020073
:10F5F00073F60200009A13786FF303031370009AF6
:10F6000013786FF30713137040E0009A1378012109
:10F6100061F303031370009A1378012161F3071358
:10F62000137033E0009A1378012161F30303137020
:10F63000009A1378022161F30713137026E0009AF1
:10F640001378012161F303031370009A13780321E7
:10F6500061F30713137019E0009A1378022161F324
:10F6600003031370009A1378012161F307131370D9
:10F670000CE0009A1378022161F303031370009ADF
:10F680001378022161F30713137000BF00BF00BF9E
:10F6900002B0704700B595B0034602910192ADF8F3
:10F6A0000E30029B9B78002B03D101238DF81E3076
:10F6B00003E0029B9B788DF81E30029B1B88ADF8FF
:10F6C0001C3006AB03220021184601F0F3FC029B1C
:10F6D0005B7C06AA11461846FFF76AFF029B9A7CDC
:10F6E00006AB013319461046FFF762FF029BDA7B37
:10F6F0009DF81A3062F3C3038DF81A30029B1A7C0E
:10F700009DF81A3062F304138DF81A30029B1A7BAD
:10F710009DF81A3062F300038DF81A30029B1B7DAE
:10F72000002B01D0022200E001229DF81A3062F382
:10F7300042038DF81A300DAB1C220021184601F04F
:10F74000B9FC029B5B7B03F01003DBB2002B06D1FC
:10F75000029B5B7B03F02003DBB2002B24D004ABC5
:10F7600003220021184601F0A5FC029BDA7C04ABC1
:10F77000013319461046FFF71BFF9DF81030012298
:10F7800062F303038DF810309DF81030012262F30C
:10F7900007138DF810309DF81230012262F34203F6
:10F7A0008DF8123004AB1293029B5B7B8DF83430E2
:10F7B000029B9B7B8DF8353008AB14220021184644
:10F7C00001F078FC07AB089306AB0993029B9B887A
:10F7D000ADF82C30029B9B68002B06D0029BDB8887
:10F7E000ADF82830029B9B680C93029B9B69002B11
:10F7F0004FD005AB03220021184601F05BFC029BB1
:10F800009B691B88ADF83C30029B9B695B88ADF817
:10F810003E30029B9B695B680E9305AB1193029B84
:10F820009B691B7B05AA11461846FFF7C1FE029B88
:10F830009B695A7B05AB013319461046FFF7B8FEAA
:10F84000029B9B699A7A9DF8163062F3C3038DF888
:10F850001630029B9B69DA7A9DF8163062F3041326
:10F860008DF81630029B9B691A7A9DF8163062F368
:10F8700000038DF81630029B9B699B7B002B01D007
:10F88000022200E001229DF8163062F342038DF857
:10F890001630029BDB69002B02D0029BDB691093C0
:10F8A00008AA0DA9BDF80E00019BFFF767FE0346ED
:10F8B000184615B05DF804FB90DF704700BF18468E
:10F8C000A5DF704700BF1846B5DF704700BF184678
:10F8D00082B00190019BF7221A80019B17225A8067
:10F8E000019B00221A71019B00225A71019BFB228D
:10F8F0009A71019B1B22DA7100BF02B070470000B1
:10F9000030B589B003460A46ADF806301346ADF867
:10F910000430BDF80430ADF81430BDF80430ADF853
:10F9200016300023ADF818300023ADF81A3003ABC1
:10F9300000221A609A8003AA05A9BDF8063018466D
:10F94000FFF7BAFF0790079B002B39D01E4A1F4BC9
:10F95000D31ADB081B0443F00104BDF806500798D6
:10F96000FAF784FB03462A4619492046F7F7C7F9F8
:10F97000BDF80C30002B03D1BDF80E30002B0ED09B
:10F98000114A124BD31ADB081B0443F00100BDF8E7
:10F990000C301A46BDF80E300E49F7F7B0F9BDF835
:10F9A0001030002B0CD0084A084BD31ADB081B047C
:10F9B00043F00103BDF8102007491846F7F78EF908
:10F9C000079B184609B030BD801903004019030099
:10F9D000042A0300502A0300902A030010B586B0C1
:10F9E00001900091009B9B88ADF80E30BDF80E3061
:10F9F000DB00019A134406330593019B1A79059B9A
:10FA00009A71009BDB7B012B02D0022B05D009E011
:10FA1000019B1A88059B1A8004E0019B5A88059B6C
:10FA20001A8000BF059B1A88059B5B889A4226D9DD
:10FA3000059B1A88BDF80E3011461846FFF740FFA7
:10FA40000490049B002B03D1059B01225A7116E000
:10FA5000049B112B03D1059B01221A710FE0114A5F
:10FA6000114BD31ADB081B0443F001040498FAF786
:10FA7000FDFA03461A460D492046F7F72FF9059B74
:10FA80009A79059BDB799A4208D9059B9B799AB2B2
:10FA9000BDF80E3011461846FFF732FF00BF06B022
:10FAA00010BD00BF8019030040190300E82A0300BD
:10FAB00000B583B001900091009B9B88DB00019A08
:10FAC000134406331846FFF703FF00BF03B05DF889
:10FAD00004FB00B587B001900091009B9B88ADF8B6
:10FAE0001630009B5B89ADF81430BDF81630DB0092
:10FAF000019A134406330493049B1B88BDF8142019
:10FB0000934228BF13469AB2049B5A80049B5B8899
:10FB1000172B38BF17239AB2049B5A80019B1B698D
:10FB2000002B15D0049B5B79002B11D040F6772376
:10FB3000ADF80830BDF81630ADF80A30049B5B888C
:10FB4000ADF80C30019B1B6902AA11460198984739
:10FB5000049B00225A71049B00221A7100BF07B057
:10FB60005DF804FB10B588B001900091009B9B8864
:10FB7000ADF81A30009BDB88ADF81830BDF81A30AC
:10FB8000DB00019A134406330593BDF81830172B98
:10FB900038BF1723ADF81830059B1B88BDF8182017
:10FBA000934228BF13469AB2059B5A80059B0022B8
:10FBB0001A71059B1A88BDF81A3011461846FFF7CE
:10FBC00083FE0790079B002B0FD0174A174BD31AC1
:10FBD000DB081B0443F001040798FAF747FA0346D1
:10FBE0001A4613492046F7F779F8059B5B79002BF5
:10FBF00016D1019B1B69002B13D040F67723ADF87B
:10FC00000C30BDF81A30ADF80E30059B5B88ADF8AE
:10FC10001030019B1B6903AA11460198984700E028
:10FC200000BF08B010BD00BF8019030040190300D9
:10FC30001C2B030030B591B001900091009B04ACE7
:10FC40001D1D0FCD0FC40FCD0FC495E8070084E82C
:10FC50000700BDF81030ADF83E30BDF81420BDF8F7
:10FC60003E30D1B2019ADB0013440A465A73019B1D
:10FC70001B69002B19D002AB00221A609A804DF646
:10FC80007A23ADF80830BDF83E30ADF80A30BDF843
:10FC90003E30019ADB0013445B7B8DF80C30019BF6
:10FCA0001B6902AA11460198984700BF11B030BDE8
:10FCB00000B587B001900091009B04330593059B2C
:10FCC0001B88DB00019A134406330493059B9B8831
:10FCD0008DF80F30049B9B799DF80F20934228BF2D
:10FCE00013468DF80E30059B1B889DF80E2092B2AE
:10FCF00011461846FFF704FE00BF07B05DF804FB8D
:10FD000000B585B001900091019B002B01D10E231D
:10FD10001DE0019B009A1A61019BF7221A80019B4A
:10FD2000F7225A80019BFB221A71002303930AE0F9
:10FD3000039BDB00019A134406331846FFF7C8FD06
:10FD4000039B01330393039B002BF1D00023184640
:10FD500005B05DF804FB82B001900B46ADF80230AF
:10FD6000019B002B01D10E230EE0BDF80230162BB3
:10FD700003D9BDF80230F72B01D9072304E0019B1A
:10FD8000BDF802201A800023184602B07047000018
:10FD900010B586B001900091009B0593019B9B8854
:10FDA000ADF81230BDF81230002B40F09880019B66
:10FDB0001B88552B48D0552B55DC242B32DC102BBF
:10FDC00051DB103B142B4ED801A252F823F000BF98
:10FDD0002BFE020035FE020067FE020067FE0200F5
:10FDE00067FE020067FE020067FE020067FE020077
:10FDF00067FE020067FE020067FE020067FE020067
:10FE000067FE020067FE020067FE020067FE020056
:10FE100067FE020067FE020067FE02005DFE020050
:10FE200053FE02003A2B0AD01DE001990598FFF716
:10FE3000D5FD19E001990598FFF73AFE14E0019904
:10FE40000598FFF746FE0FE001990598FFF78AFE37
:10FE50000AE001990598FFF7EDFE05E00199059884
:10FE6000FFF726FF00E000BFBDF81230059ADB0067
:10FE700013449B7A002B33D0BDF81230059ADB0077
:10FE80001344DA88BDF8123011461846FFF718FD02
:10FE90000390039B002B0ED1BDF81230059ADB00B6
:10FEA000134400229A72BDF81230059ADB00134405
:10FEB0000122DA7214E0039B112B11D0094A0A4B7C
:10FEC000D31ADB081B0443F001040398FAF7CEF8B9
:10FED00003461A4605492046F6F700FF00E000BF3A
:10FEE00006B010BD8019030040190300E82A030082
:10FEF000B0DF704700BF184666DF704700BF184686
:10FF000082B001900091019B002B01D10E2316E0DD
:10FF1000009B002B01D10E2311E0019B1B78DE2BEF
:10FF200001D108230BE0009B1A68019B5A60019BDA
:10FF3000DE221A70019B4FF6FF725A80002318468A
:10FF400002B0704782B001900B46ADF80230019BC1
:10FF5000002B01D10E230AE0019B1B78DE2B01D080
:10FF6000082304E0019BBDF802205A8000231846B4
:10FF700002B0704700B585B00190019B1B7A002B41
:10FF800018D0019B5B8800211846FFF7B5FF03904E
:10FF9000039B002B03D1019B00221A720AE0039BF2
:10FFA000112B03D1019B01221A7203E0019B5B68B4
:10FFB0000398984700BF05B05DF804FB00B583B017
:10FFC00001900091009B1B79012B0BD1009B1A889B
:10FFD000019B5B889A4205D1019B01221A7201980C
:10FFE000FFF7C8FF00BF03B05DF804FB82B00190CB
:10FFF000009100BF02B0704700B589B00190009138
:020000023000CC
:10000000009B1A88019B5B889A4236D1009B023381
:100010000793079B1B78022B31D1079B1B7A042B7C
:1000200007D0079B1B7A062B03D0079B1B7A052B57
:1000300027D102AB00221A605A609A60DA6002236C
:100040008DF808304FF4C073ADF80C30079B1B7A65
:10005000052B02D10023ADF80C30009B1B8802AAAF
:1000600011461846FFF744FF0690069B002B09D067
:10007000019B5B680698984704E000BF02E000BF60
:1000800000E000BF09B05DF804FB00B585B0019049
:100090000091009B002B40D0019B002B3FD0009B88
:1000A0000393039B1B78DE2B3BD1019B9A88039B18
:1000B0005B889A4202D10398FFF75CFF019B1B8883
:1000C000512B18D0512B2EDC112B1BD0112B2ADCDD
:1000D000012B02D0022B07D025E0019B04331946E7
:1000E0000398FFF76BFF21E0019B04331946039847
:1000F000FFF77CFF1AE0019B043319460398FFF7D2
:100100007BFF13E0019B9A88039B5B889A420CD18A
:10011000039B4FF6FF725A8007E000BF06E000BF66
:1001200004E000BF02E000BF00E000BF05B05DF8E2
:1001300004FBA8DF704700BF1846ADDF704700BF63
:100140001846AEDF704700BF184662DF704700BF39
:10015000184600B58FB00190009100230393019BD6
:100160005869009B9B8803AA1946FFF7AEF90D90CA
:1001700005AB08220021184600F09CFF04AB069353
:100180000223ADF814300023ADF81630009B988898
:10019000019B1B8A05AA1946FFF7CFFF0D900D9B07
:1001A000002B26D1019B9B69002B22D0069B184671
:1001B000FFF7E8F90346002B1BD0039B002B02D06E
:1001C000039B01221A7007AB18220021184600F089
:1001D00071FF02238DF81C30019B0893009B9B88C4
:1001E000ADF82430039B0A93019B9B6907AA104634
:1001F000984700BF0FB05DF804FB00B58DB00190CB
:100200000091009B06330B93019B5869009B9B88D0
:1002100003AA1946FFF759F90A9004AB18220021E6
:10022000184600F047FF019B0593009B9B88ADF8A3
:100230001830039B07930B9B1A88019B1B899A42DA
:1002400025D10B9B5B89022B21D1039B002B38D03E
:100250000B9B0C331846FFF795F90346002B06D08D
:10026000039B01221A7002238DF8103005E0039BD6
:1002700000221A7003238DF81030019B9B69002B1C
:100280001FD0019B9B6904AA1046984719E00B9B5D
:100290001A88019B9B899A4214D1019B9B69002B70
:1002A00010D000238DF810300B9B0C3308930B9B60
:1002B0005B89ADF82430019B9B6904AA10469847DE
:1002C00000E000BF00BF0DB05DF804FB00B58BB0CF
:1002D00001900091019B5869009B9B8802AA1946D6
:1002E000FFF7F3F80990099B002B1AD1029B1B78AA
:1002F000002B17D003AB18220021184600F0DAFEBD
:1003000001238DF80C30019B0493009B9B88ADF872
:100310001430029B0693019B9B6903AA10469847E1
:1003200000E000BF0BB05DF804FB00B585B00190A4
:100330000091009B002B1ED0019B002B1BD0009B2B
:100340000393019B1B88572B10D0572B15DC102BC8
:1003500002D0502B05D010E001990398FFF7F9FE69
:100360000CE001990398FFF748FF07E00199039813
:10037000FFF7ACFF02E000BF00E000BF05B05DF892
:1003800004FB000010B592B0019000914F4B0AACF5
:100390000FCB84E80F00019B002B01D10E2391E0CD
:1003A000009B002B01D10E238CE0009B1A68019B5F
:1003B0009A61019A0AAB11461846FFF7C6FE1190E2
:1003C000119B1093109B002B01D0109B7AE0019B96
:1003D0001B788DF83A300123ADF83830019B9A1C18
:1003E0000EAB19460120FFF7A4FE1190119B0F934D
:1003F0000F9B002B01D00F9B64E002AB2022002159
:10040000184600F057FE0223ADF80830019B1B7818
:100410008DF80A30F423ADF80C300123ADF80E301E
:1004200001238DF814309DF8153043F008038DF842
:1004300015309DF8153043F004038DF81530012375
:100440008DF8193001238DF81A30019B5888019BD3
:1004500003F10C0202AB1946FFF71CF91190119B36
:10046000002B01D0119B2DE002AB20220021184669
:1004700000F020FE0323ADF80830019B1B788DF8B7
:100480000A30F423ADF80C300123ADF80E3001230F
:100490008DF814309DF8153043F010038DF81530A9
:1004A00001238DF8193001238DF81A3001238DF8BE
:1004B0001B30019B5888019B1A1D02AB1946FFF7A0
:1004C000E9F80346184612B010BD00BF542B0300D4
:1004D00000B58DB0039002910192ADF80230039BFC
:1004E000002B01D10E2342E0039B5B6905AABDF8F6
:1004F00002101846FEF7E9FF0B900B9B0A930A9B2C
:10050000002B01D00A9B32E0BDF802304FF6FF729B
:10051000934202D0059B002B01D1052327E0059BC8
:100520001B7883F00103DBB2002B01D008231EE00F
:10053000019B1B88F42B01D9072318E006AB10227E
:100540000021184600F0B6FD039B9B88ADF81830DB
:10055000029B0993019B089301238DF81A3006AA88
:10056000BDF8023011461846FFF7EBFD034618466A
:100570000DB05DF804FB000082B003468DF8073033
:100580009DF8073003F01F0205499DF907305B090C
:10059000012000FA02F241F8232000BF02B07047A8
:1005A00000E100E082B003468DF807309DF9073086
:1005B000002B0BDA0B4A9DF8073003F00F03043BC6
:1005C00013441B7EDBB25B09DBB208E0064A9DF9EF
:1005D0000730134493F80033DBB25B09DBB21846F3
:1005E00002B0704700ED00E000E100E000B583B02C
:1005F0000190019B002B03D10449C420FCF784FE29
:10060000019B5B68184603B05DF804FB642B030094
:1006100010DF704700BF184682B003468DF80730E0
:100620009DF907301F2B0CDC9DF907300F4A22FA89
:1006300003F303F00103002B14BF01230023DBB2FB
:1006400010E09DF907303F2B0BDC9DF90730203B74
:10065000012202FA03F3002B14BF01230023DBB2B3
:1006600000E00123184602B0704700BFFC06FFBD42
:1006700082B00190019B072B07D8EC22019B42FA24
:1006800003F303F00103002B01D1002300E0012359
:10069000184602B07047000000B583B003468DF8DD
:1006A00007309DF907301846FFF7B6FF0346002BC9
:1006B00002D142F201032EE09DF907301846FFF700
:1006C00071FF03461846FFF7D3FF0346002B02D104
:1006D00042F202031FE0124B9B68002B15D09DF9DC
:1006E00007305B090E4A52F823209DF8073003F0CB
:1006F0001F03012101FA03F319469DF907305B0935
:100700000A43074941F8232004E09DF907301846C1
:10071000FFF732FF0023184603B05DF804FB00BF6B
:10072000FC32002000B587B003468DF8073002ABDD
:1007300014491846F9F73EFC17E002AB1846FFF7DC
:1007400055FF0590059B1B680493059B59689DF810
:100750000720049B104698470346002B01D1112324
:100760000BE002AB1846F9F74FFC02AB1846FFF757
:100770003DFF0346002BE0D10023184607B05DF88B
:1007800004FB00BF142C030000B587B003468DF8AE
:10079000073002AB11491846F9F70CFC12E002AB26
:1007A0001846FFF723FF0590059B1B680493059BE4
:1007B00059689DF80720049B1046984702AB1846DD
:1007C000F9F722FC02AB1846FFF710FF0346002B97
:1007D000E5D100BF00BF07B05DF804FB202C03008B
:1007E00000B583B01620FFF757FF0190019B0093DF
:1007F000009B002B04D0044AA1210098F7F79CF934
:1008000000BF03B05DF804FBC02B030000B585B04A
:10081000234B1B78002B01D008233CE0214B012205
:100820001A700020FFF77EFF0346112B01D1002331
:1008300031E00020FFF7A8FF1B4B1B680293002349
:100840008DF807300DF107031846F8F747FB02ABA8
:1008500016491846FFF7DCFE0390039B002B0CBFE4
:1008600001230023DAB20E4B1A709DF807301846A8
:10087000F8F74AFB039B002B01D0039B0BE0094BCD
:1008800000221A700A4B00221A70FFF7A9FF0120FC
:10089000FFF77AFF0023184605B05DF804FB00BFA0
:1008A000D43A0020D63A0020102C0300557B0200D9
:1008B000D53A0020014B1B7818467047D43A0020E7
:1008C00000B585B06B4611491846F9F773FB10E087
:1008D0006B461846FFF78AFE0390039B1B68029342
:1008E000039B5A68029B104698476B461846F9F7D7
:1008F0008BFB6B461846FFF779FE0346002BE7D1CA
:1009000000BF00BF05B05DF804FB00BF2C2C030046
:1009100008B5FFF7D5FF00BF08BD60DF704700BF17
:10092000184669DF704700BF184661DF704700BF97
:100930001846000000B583B00190019B002B03D145
:100940000449C420FCF7E0FC019B5B68184603B037
:100950005DF804FB382C030082B00190019B002B52
:1009600001D10E2304E0044B1A46019B1A600023B8
:10097000184602B0704700BF982A002010B586B014
:10098000034600918DF807300098FFF7E5FF0590CA
:10099000059B002B01D0059BECE002AB0C22002153
:1009A000184600F087FB9DF807308DF808300123CA
:1009B0008DF80A300623ADF80C30009B1A6802ABA4
:1009C00019462020FFF7ADFF0590059B002B0FD0A7
:1009D0006A4A6B4BD31ADB081B0443F001040598E9
:1009E000F9F744FB03461A4666492046F6F776F9BE
:1009F00002AB0C220021184600F05CFB01238DF8AD
:100A0000093000238DF80A3000238DF80B30009B4D
:100A10001A6802AB19464020FFF783FF0590059B3B
:100A2000002B0FD0554A564BD31ADB081B0443F05A
:100A300001040598F9F71AFB03461A465249204665
:100A4000F6F74CF902AB0C220021184600F032FBFD
:100A50009DF807308DF80830F723ADF80A30009B79
:100A60001A6802AB19462320FFF75BFF0590059B30
:100A7000002B0FD0414A424BD31ADB081B0443F032
:100A800001040598F9F7F2FA03461A463F49204651
:100A9000F6F724F902AB0C220021184600F00AFBFD
:100AA00001238DF80830009B1A6802AB194601201B
:100AB000FFF737FF0590059B002B0FD02F4A304BD7
:100AC000D31ADB081B0443F001040598F9F7CEFAAA
:100AD00003461A462E492046F6F700F902AB0C22CF
:100AE0000021184600F0E6FA4FF4B0630293009B31
:100AF0001A6802AB1946A120FFF713FF0590059B6A
:100B0000002B0FD01D4A1E4BD31ADB081B0443F0E9
:100B100001040598F9F7AAFA03461A461D4920462A
:100B2000F6F7DCF802AB0C220021184600F0C2FAFE
:100B30009DF808306FF300038DF80830009B1A68A9
:100B400002AB1946A020FFF7ECFE0590059B002B99
:100B50000FD00A4A0A4BD31ADB081B0443F00104E6
:100B60000598F9F783FA03461A460B492046F6F72B
:100B7000B5F80023184606B010BD00BF9019030059
:100B800040190300982C0300E02C03002C2D0300D7
:100B9000742D0300C02D0300142E030082B04FF00B
:100BA0008053D3F80C319B020193019B03F1005356
:100BB000184602B07047000010B584B00190019B48
:100BC0001B6803930198FFF7A8FE0290019B1B6826
:100BD000039A9A4229D2224A224BD31ADB081B04D9
:100BE00043F0020320491846F6F76AF81C4A1D4BE9
:100BF000D31ADB081B0443F00200019B1B68039A15
:100C00001A49F6F77CF8164A164BD31ADB081B0470
:100C100043F00204FFF7C2FF0246019B1B68D31A90
:100C20001A4613492046F6F759F8029B002B03D1C8
:100C3000104B01221A700FE0094A0A4BD31ADB0845
:100C40001B0443F001040298F9F710FA03461A4610
:100C500009492046F6F742F8029B184604B010BD39
:100C60009019030040190300682E0300982E03001A
:100C7000CC2E0300D73A0020F82E030000B5ADF5C6
:100C8000077D86ABA3F505731860244B1B7883F0B2
:100C90000103DBB2002B3BD14FF4FA73ADF80632FF
:100CA0000DF2062202AB11461846FFF73EFE859074
:100CB000859B002B03D0859B052B22D129E002AB1D
:100CC00084937FAB16491846F9F774F911E07FABAE
:100CD0001846FFF72FFE8390839B1B688293839BAC
:100CE0005A68829B1146849898477FAB1846F9F75B
:100CF0008BF97FAB1846FFF71DFE0346002BE6D1AC
:100D0000CAE7084A40F239118598F6F715FF00E066
:100D100000BF0DF5077D5DF804FB00BFD73A00204A
:100D20006C2F0300182F030000B583B00190019BC6
:100D3000002B03D10449C420FCF7E6FA019B5B6851
:100D4000184603B05DF804FB782F03004BDF7047B3
:100D500000BF184600B589B0019004AB1846FFF7F4
:100D6000F5FF0790079B002B03D0079B052B20D195
:100D700024E002AB13491846F9F71CF911E002AB65
:100D80001846FFF7D1FF0690069B1B680593049A4F
:100D9000069B5968059B1046984702AB1846F9F721
:100DA00033F902AB1846FFF7BFFF0346002BE6D12D
:100DB000D3E7054A6B210798F6F7BEFE00BF09B0DE
:100DC0005DF804FB2C300300D82F0300002B35D135
:100DD00029B9B0FBF2FC0CFB12026046704791424D
:100DE00015D22DE9F041B2FA82F39A409940D3F13D
:100DF000200C30FA0CFC51EA0C01984000F04EF83F
:100E0000280036FA03F200210023BDE8F081F0B596
:100E1000B1FBF2FC0CFB1211B2FA82F39A4099403A
:100E2000D3F1200630FA06F63143984000F036F848
:100E3000614628003200DA400023F0BDF3B5B3FA72
:100E400083FC49085FEA300013FA0CF3DCF120045C
:100E500032FA04F423430CB41A0000F01FF80CBC5F
:100E600033FA0CF3DCF11F0C35FA0CF518BF013D19
:100E700003BCA5FB026705FB0377801BB9419042C9
:100E800071EB030C05D3821A71EB0303681C00217C
:100E9000F0BD02000B0028000021F0BD940D4FF6BC
:100EA000C2752D02B5FBF4F4D60A013604FB04F535
:100EB000A5FB0656F64306EB0416550832BF00277D
:100EC0007708013505FB1677A6FB07477F0807EB78
:100ED000C63714001500E7FB02457F1B4D1C0400BC
:100EE000E7FB014505FB1206A64284BF013DB6188B
:100EF000964224BF0135B61A704700BF43F6D82189
:100F0000C2F20001086800B1704742F66430C2F2D4
:100F10000000086070479AB18446097848B20028FA
:100F200044BF6FF001007047BCF1000F18BFCCF850
:100F300000100021C3E90011002818BF01207047EC
:100F4000002070477F298EBF6FF0010001700120E3
:100F5000704743F6D822C2F20002136823B942F662
:100F60006433C2F2000313605A6892681268104733
:100F70000921FFF7EEBF7F2884BF0020704743F2AE
:100F80004C22C0F20302515C43F2CC12C0F20302C5
:100F9000105C08407047A0F161011A2938BF203861
:100FA0007047A0F141011A2938BF203070477F28CF
:100FB00084BF0020704743F24C22C0F20302515C10
:100FC00043F2CC12C0F20302105C08407047A0F15B
:100FD00061011A2938BF20387047A0F141011A2950
:100FE00038BF203070470000411C82070CD010F839
:100FF000012B3AB3820707D010F8012B12B38207F6
:1010000002D010F8012BEAB14FF0013C50F8042B4C
:10101000CCFA52F37BB950F8042BCCFA52F353B903
:1010200050F8042BCCFA52F32BB950F8042BCCFA1D
:1010300052F3002BEAD004381BBAB3FA83F300EB67
:10104000D3000130401A704772B3844690EA01031E
:101050009B0721D1830709D011F8013B00F8013B20
:10106000013A20D08307F7D100E08446202A0AD332
:101070002DE9F007B1E8F807A0E8F807203A202AA0
:10108000F8D2BDE8F007042A06D351F8043B40F833
:10109000043B043A042AF8D22AB111F8013B00F8C3
:1010A000013B013AF9D16046704700BF00220B00B6
:1010B00011001A0084465AB3830704D000F8011BBC
:1010C000013AF9D124E0C9B241EA012141EA0141E2
:1010D000202A11D3203A2DE9F0030B460C460D4689
:1010E0000E460F4688468946A0E8FA03203AFBD20E
:1010F000BDE8F00320320BD0042A05D340F8041BCE
:10110000043A05D0042AF9D200F8011B013AFBD1B8
:101110006046704700B5F9B10278EAB1D0F800E056
:101120000429034609D34FF0013CCCFA5EF222B900
:1011300053F804EF04390329F7D8181A4FF0013295
:10114000C2FA5EF292FAA2F2B2FA82F2B1EBD20FD6
:1011500028BFD108084400BD002000BD10B582B0F2
:10116000044600698DF8071078B1D4E900239A424B
:101170001CD26269531C63618154D4E90501884221
:1011800014D1204600F032F810E0D4F80CC0BCF1C5
:10119000000F10D0D4E90023501C984204BF002156
:1011A0008DF807109A4238BF0CF802102068013001
:1011B000206002B010BDA06858B1D4E9002C62458F
:1011C000F4D2531CB3EB0C0318BFCBB240F822305F
:1011D000ECE7236A002BE9D0D4E900018842E5D28C
:1011E0000DF10701204601229847DFE710B542695B
:1011F00032B10446036A0BB121699847002060614F
:1012000010BD70B5012AB8BF70BD0C460546561C0E
:1012100028462146FFF7A2FF013E012EF8D870BDF7
:10122000CB0648BF704789054CBF30212021FFF70E
:10123000E8BF70B514460D460646FFF75FFE01464F
:1012400030462A462346BDE8704000F000B82DE93C
:10125000F04F03AF8DB047F83C3C91460E46044634
:1012600000F028FB0546EB46073020F00700ADEB09
:101270000008C546A7F1380A504600212422FFF78E
:1012800019FF41F2BB20C0F2030047E907606FF08D
:10129000004047F8340C47F8144C47F8205C47F8F6
:1012A000288C5046494657F83C2C00F021F8DD4682
:1012B000A7F10C04A546BDE8F08F436A084601215A
:1012C00000F0C9BA83B000B582B00DF10C0C8CE807
:1012D0000E0042F68032C2F200020146106803AAF4
:1012E0000192FFF7A6FF02B0BDE8004003B07047CF
:1012F0002DE9F04F8DB00692894683460020CBF849
:1013000000000DF11E04A4F10108CDF81080CDF805
:1013100004B019F8011B252906D0002900F08482A9
:101320005846FFF71BFFF4E70027484619F8012B42
:10133000A2F12003102B0DD88021DFE803F0091B58
:101340001B191B1B1B101B1B31131B151B1B170011
:1013500040210DE05E2A0DD14FF4805108E04FF49A
:10136000004105E0202103E0102101E04FF400716D
:101370000F43DAE700F10109A2F13000C0B20928F9
:101380001DD8002119F8010B01EB810102EB41018D
:101390003039A0F13002D2B20A2A0246F2D30BE071
:1013A000069A52F8041B0692002944BF47F0100722
:1013B0004942427800F1020921EAE17A01E04FF066
:1013C000000A2E2A0DD1484610F8012B2A2A0AD1EC
:1013D000069899F8012050F8045B069009F102097B
:1013E00016E000251CE0A2F13001C9B20025092950
:1013F00013D810F8011B05EB850302EB4302A2F1A1
:101400003005A1F13002D2B20A2A0A46F1D3814650
:10141000002D58BF47F4807702E0814647F480777B
:10142000A2F16800C1B2C00140EA5100C0B209286F
:101430002AD8DFE800F008141729292905292905E9
:1014400019F8012B20E0484610F8012B682A15D125
:1014500099F8012009F1020947F0080714E019F88A
:10146000012B08E0484610F8012B6C2A09D199F8A5
:10147000012009F1020947F0020705E047F00407DF
:1014800001E047F001078146622A15DDA2F1630001
:1014900015283FF63EAFDFE800F0240C0B0B0B0BDA
:1014A0000C0B0B0B0B37434D0B0B5B0B6A0B0B172A
:1014B0002FE747F480475EE0252A00F0A980582AEC
:1014C00040F07A8147F40057F8054FEA076048BFBB
:1014D00027F40077782A43F2580108BF43F27801D5
:1014E00025E0069DA0462C78AAF10106584639460B
:1014F0003246FFF795FE584621464446DDF81080F7
:10150000FFF72CFE28467CE1380700F15981B80727
:10151000DBF8001000F18081069A1068016054E148
:10152000F8054FEA076048BF27F40077302101EA49
:10153000E07321E03806232101EAE070059047F4CA
:101540008077069A002152F8040B06920825CCE019
:1015500006980468002C04BF43F27924C0F2030407
:10156000F805204600F13381FFF73EFD32E1F80532
:1015700048BF27F40077002307F0020079040593A1
:1015800006D4AC460028069809D1031D00210CE0C2
:10159000A0B9069951F8040B0691C11716E007305F
:1015A00020F0070000F10803416800687D0715D4AA
:1015B00017F008051CBFC0B2002111E006980730E3
:1015C00020F00703596853F8080B06937B070AD4E9
:1015D00017F008031CBFC0B2002107E080B2002151
:1015E000069365461BE040F3C03100B2002909DBD9
:1015F000BB0612D47B06A446059C48BF2024059454
:1016000064460CE00023404263EB01012D2305E01A
:1016100058462521FFF7A2FD7BE62B230593FB050A
:1016200048BF27F40077FB0558BF012500266E2A26
:1016300023DD6F3A092A00F27E80DFE802F00556CA
:101640007C7C7C7C247C7C5650EA010272D0AC46C7
:10165000C20842EA417200260625134665F3DF0000
:10166000A055013652EAD1004FEAD1014FEAD2002B
:1016700040EA41721846F0D15AE0582A35D0642A1F
:1016800018BF692A57D150EA010253D0CDE9025A56
:10169000A24607F4004B00260C460546BBF1000F9E
:1016A00007D006F00300032802BF2C200AF806002A
:1016B0000136D046284621460A220023FFF786FB42
:1016C00000EB8002A5EB420242F0300208F806204F
:1016D0000136D5F109024FF00002A241DCD3544695
:1016E000DDE903A8DDE901B525E050EA010221D0DA
:1016F000AC46BA0443F25922C0F203025CBF43F283
:101700006922C0F203024FEA101343EA01734FF05B
:10171000000600F00F051846535DA355013650EA48
:1017200011134FEA11114FEA101343EA0173F0D17C
:10173000654600E00026AAEB06000599FF2988BF50
:10174000013800290A4618BF0122801AAA1B22EA82
:10175000E275A0EB050AB80507D45846394652464B
:10176000FFF75EFD05994FF0000AFF2904D9090A29
:101770005846FFF7F3FC059911B15846FFF7EEFC08
:10178000584639465246FFF74BFD584630212A4607
:10179000FFF737FD012E06DB18F806105846FFF755
:1017A000DDFC013EF8D8F8067FF5B3AD58462021A0
:1017B0005246FFF726FDACE5002A7FF4AAAD44E0CF
:1017C000069A1068DBF800100170104629E02946DF
:1017D000FFF7A0FC054627F40077AAEB0006584661
:1017E00039463246FFF71CFD35B114F8011B584647
:1017F000FFF7B4FC013DF8D1DDF8108006980DF13B
:101800001E0404300690F8067FF583AD584620216B
:101810003246FFF7F6FC7CE5069B1868002206C0FE
:1018200018460430069074E5DBF80C0028B1DBE9BB
:10183000001291423CBF002242545846FFF7D6FCAA
:10184000DBF800000DB0BDE8F08F5846FFF7CEFC86
:101850004FF0FF30F6E7F8B51D4617460C46064632
:10186000184600F00FF8002803D407FB04F2A24248
:1018700001D20020F8BD2846314600F01DF8B0FB2B
:10188000F4F0F8BD084B1B6883420AD0074B1B6875
:10189000834206D0064B1B68181A18BF4FF0FF3062
:1018A00070470020704700BF7C2B0020802B002059
:1018B000782B0020402070470068FCF713BC00BF65
:1018C000072904D90023024AC0E90031106070479B
:0418D000E83A0020D2
:0818D400D1A602000000000093
:1018DC0069F302000000000029D2020000000000A1
:1018EC0091FD020024340020A5F10200000000004C
:1018FC002B030300F82A00208B000300383400204F
:08190C0019D6020000000000E2
:08191400F9A60200000000002A
:10191C007D0C030000000000550D030000000000CA
:10192C00902C0020C82B0020D02B0020D02B002086
:04193C00180000008F
:10194000B025030000000000702603000000000026
:10195000C8260300000000007C27030000000000F0
:101960003428030000000000541A030000000303A1
:101970004C2B030000000000D824030000000000EE
:10198000F429030000000303B82B03000000030345
:101990008C2C030000000303CC2F03000000030382
:0819A000D81E03000000000046
:1019A800B819030000000000D8190300982A002085
:1019B800B9640200EB640200E16402000000000068
:1019C80000000000000000000338FDD87047000048
:1019D8007274745F6C6F675F6261636B656E6400DD
:1019E800433A5C4E6F726469635F73656D695C6EE0
:1019F8005246355F53444B5F31352E332E305F35B9
:101A08003961633334355C636F6D706F6E656E7406
:101A1800735C6C69627261726965735C6C6F675C38
:101A28007372635C6E72665F6C6F675F6465666134
:101A3800756C745F6261636B656E64732E6300001E
:101A4800982C00207F000000182D00206170700085
:101A5800433A5C4E6F726469635F73656D695C6E6F
:101A68005246355F53444B5F31352E332E305F3548
:101A78003961633334355C636F6D706F6E656E7496
:101A8800735C6C69627261726965735C6C6F675CC8
:101A98007372635C6E72665F6C6F675F66726F6E9F
:101AA80074656E642E6300004261636B656E6473D7
:101AB80020666C7573686564000000006572726F5B
:101AC800720000007761726E696E6700696E666FFA
:101AD8000000000064656275670000001B5B306DE4
:101AE800000000001B5B313B33306D001B5B313B5A
:101AF80033316D001B5B313B33326D001B5B313B77
:101B080033336D001B5B313B33346D001B5B313B62
:101B180033356D001B5B313B33366D001B5B313B4E
:101B280033376D0025734C6F67732064726F707064
:101B38006564202825642925730D0A002573000093
:101B48003C25733E2025733A200000000D0A000052
:101B58002025303278000000202020007C00000082
:101B6800256300002000000060310020534F4654D8
:101B78004445564943453A20415353455254494FE9
:101B88004E204641494C454400000000534F4654FE
:101B98004445564943453A20494E56414C4944200C
:101BA8004D454D4F52592041434345535300000082
:101BB800415353455254494F4E204641494C4544A0
:101BC8002061742025733A25750000004552524F54
:101BD80052202575205B25735D2061742025733A9A
:101BE80025750D0A50432061743A20307825303825
:101BF80078000000456E64206F66206572726F720F
:101C0800207265706F727400554E4B4E4F574E20C0
:101C18004641554C5420617420307825303858009E
:101C280000000000000000000338FDD870470000E5
:101C3800FFFFFFFFFFFFFFFFFFFFFFFFFFFFFFFFAC
:101C480000000000000000000000D60106010000AE
:101C5800433A5C4E6F726469635F73656D695C6E6D
:101C68005246355F53444B5F31352E332E305F3546
:101C78003961633334355C636F6D706F6E656E7494
:101C8800735C6C69627261726965735C75617274A8
:101C98005C6170705F756172745F6669666F2E63F0
:101CA80000000000433A5C4E6F726469635F7365BD
:101CB8006D695C6E5246355F53444B5F31352E3348
:101CC8002E305F353961633334355C636F6D706F07
:101CD8006E656E74735C6C69627261726965735C5F
:101CE8007574696C5C6170705F7574696C5F706C39
:101CF8006174666F726D2E6300000000433A5C4E9B
:101D08006F726469635F73656D695C6E5246355FB7
:101D180053444B5F31352E332E305F353961633391
:101D280034355C636F6D706F6E656E74735C6C696F
:101D3800627261726965735C62616C6C6F635C6E20
:101D480072665F62616C6C6F632E6300433A5C4E2F
:101D58006F726469635F73656D695C6E5246355F67
:101D680053444B5F31352E332E305F353961633341
:101D780034355C65787465726E616C5C6670726926
:101D88006E74665C6E72665F667072696E74662EDB
:101D980063000000433A5C4E6F726469635F736569
:101DA8006D695C6E5246355F53444B5F31352E3357
:101DB8002E305F353961633334355C65787465720C
:101DC8006E616C5C667072696E74665C6E72665F7A
:101DD800667072696E74665F666F726D61742E6389
:101DE800000000003031323334353637383941425B
:101DF80043444546433A5C4E6F726469635F73655A
:101E08006D695C6E5246355F53444B5F31352E33F6
:101E18002E305F353961633334355C636F6D706FB5
:101E28006E656E74735C6C69627261726965735C0D
:101E38006D656D6F626A5C6E72665F6D656D6F620F
:101E48006A2E63002E2E2F2E2E2F2E2E2F2E2E2F63
:101E58002E2E2F2E2E2F636F6D706F6E656E74731E
:101E68002F6C69627261726965732F65787065722B
:101E7800696D656E74616C5F73656374696F6E5FBD
:101E8800766172732F6E72665F73656374696F6EC5
:101E98005F697465722E68002E2E2F2E2E2F2E2E1F
:101EA8002F2E2E2F2E2E2F2E2E2F636F6D706F6ECE
:101EB800656E74732F6C69627261726965732F6DD8
:101EC800757465782F6E72665F6D74782E68000081
:101ED8007077725F6D676D7400000000433A5C4E66
:101EE8006F726469635F73656D695C6E5246355FD6
:101EF80053444B5F31352E332E305F3539616333B0
:101F080034355C636F6D706F6E656E74735C6C698D
:101F1800627261726965735C7077725F6D676D7408
:101F28005C6E72665F7077725F6D676D742E6300AA
:101F3800141903001419030004000000433A5C4E0E
:101F48006F726469635F73656D695C6E5246355F75
:101F580053444B5F31352E332E305F35396163334F
:101F680034355C636F6D706F6E656E74735C6C692D
:101F7800627261726965735C6578706572696D65B6
:101F88006E74616C5F73656374696F6E5F7661729E
:101F9800735C6E72665F73656374696F6E5F697494
:101FA80065722E6300000000556E6B6E6F776E20B1
:101FB8006572726F7220636F646500004E52465FEF
:101FC80053554343455353004E52465F4552524F73
:101FD800525F5356435F48414E444C45525F4D490A
:101FE8005353494E470000004E52465F4552524FE8
:101FF800525F534F46544445564943455F4E4F54EC
:102008005F454E41424C4544000000004E52465F39
:102018004552524F525F494E5445524E414C000072
:102028004E52465F4552524F525F4E4F5F4D454D9F
:10203800000000004E52465F4552524F525F4E4FCD
:10204800545F464F554E44004E52465F4552524FDC
:10205800525F4E4F545F535550504F5254454400B1
:102068004E52465F4552524F525F494E56414C4977
:10207800445F504152414D004E52465F4552524FC7
:10208800525F494E56414C49445F535441544500B0
:102098004E52465F4552524F525F494E56414C4947
:1020A800445F4C454E475448000000004E52465F7E
:1020B8004552524F525F494E56414C49445F464C37
:1020C800414753004E52465F4552524F525F494E68
:1020D80056414C49445F4441544100004E52465FCA
:1020E8004552524F525F444154415F53495A45004B
:1020F8004E52465F4552524F525F54494D454F55D7
:10210800540000004E52465F4552524F525F4E55A2
:102118004C4C00004E52465F4552524F525F464F5C
:102128005242494444454E004E52465F4552524F32
:10213800525F494E56414C49445F41444452000065
:102148004E52465F4552524F525F42555359000016
:102158004E52465F4552524F525F434F4E4E5F4379
:102168004F554E54000000004E52465F4552524FA4
:10217800525F5245534F5552434553004E52465FA6
:102188004552524F525F4D4F44554C455F4E4F5448
:102198005F494E495449414C495A454400000000A2
:1021A8004E52465F4552524F525F4D555445585F07
:1021B800494E49545F4641494C4544004E52465F9A
:1021C8004552524F525F4D555445585F4C4F434B03
:1021D8005F4641494C4544004E52465F4552524F76
:1021E800525F4D555445585F554E4C4F434B5F46D3
:1021F80041494C45440000004E52465F4552524FFB
:10220800525F4D555445585F434F4E445F494E49C0
:10221800545F4641494C4544000000004E52465F19
:102228004552524F525F4D4F44554C455F414C52B9
:10223800454144595F494E495449414C495A4544DE
:10224800000000004E52465F4552524F525F5354B1
:102258004F524147455F46554C4C00004E52465F31
:102268004552524F525F4150495F4E4F545F494D5E
:10227800504C454D454E5445440000004E52465F73
:102288004552524F525F464541545552455F4E4F55
:10229800545F454E41424C45440000004E52465F53
:1022A8004552524F525F494F5F50454E44494E4741
:1022B800000000004E52465F4552524F525F445252
:1022C800565F5457495F4552525F4F5645525255D3
:1022D8004E0000004E52465F4552524F525F4452E4
:1022E800565F5457495F4552525F414E41434B0038
:1022F8004E52465F4552524F525F4452565F5457B2
:10230800495F4552525F444E41434B004E52465F2F
:102318004552524F525F424C455F495053505F52AD
:10232800585F504B545F5452554E434154454400F6
:102338004E52465F4552524F525F424C455F49509C
:1023480053505F4348414E4E454C5F414C524541C6
:1023580044595F4558495354530000004E52465F54
:102368004552524F525F424C455F495053505F4C63
:10237800494E4B5F444953434F4E4E4543544544A1
:10238800000000004E52465F4552524F525F424C89
:10239800455F495053505F504545525F52454A4545
:1023A800435445440000000000000000C41F03001F
:1023B80001000000D01F030002000000F01F03000E
:1023C800030000001420030004000000282003007C
:1023D800050000003C200300060000005020030018
:1023E80007000000682003000800000080200300A8
:1023F80009000000982003000A000000B420030030
:102408000B000000CC2003000C000000E4200300B7
:102418000D000000F82003000E0000000C2103004E
:102428000F0000001C2103001000000030210300F1
:102438001100000048210300120000005821030089
:1024480013000000702103008000000084210300B5
:1024580081000000A821030082000000C4210300BD
:1024680083000000E0210300840000000022030034
:102478008500000024220300860000004C2203008F
:1024880090000000642203009100000084220300F1
:1024980092000000A422030000820000BC22030076
:1024A80001820000DC22030002820000F8220300FF
:1024B8000084000014230300018400003823030073
:1024C8000284000064230300038400008C230300BB
:1024D800636C6F636B000000433A5C4E6F72646913
:1024E800635F73656D695C6E5246355F53444B5F3D
:1024F80031352E332E305F353961633334355C69BD
:102508006E746567726174696F6E5C6E7266785C12
:102518006C65676163795C6E72665F6472765F632F
:102528006C6F636B2E630000433A5C4E6F72646994
:10253800635F73656D695C6E5246355F53444B5FEC
:1025480031352E332E305F353961633334355C696C
:102558006E746567726174696F6E5C6E7266785CC2
:102568006C65676163795C6E72665F6472765F75CD
:102578006172742E630000002E2E2F2E2E2F2E2E09
:102588002F2E2E2F2E2E2F2E2E2F696E74656772EA
:102598006174696F6E2F6E7266782F6E7266785FDF
:1025A800676C75652E680000434C4F434B00000074
:1025B800433A5C4E6F726469635F73656D695C6E04
:1025C8005246355F53444B5F31352E332E305F35DD
:1025D8003961633334355C6D6F64756C65735C6E3B
:1025E8007266785C647269766572735C7372635C38
:1025F8006E7266785F636C6F636B2E630000000019
:102608002E2E2F2E2E2F2E2E2F2E2E2F2E2E2F2EDD
:102618002E2F696E746567726174696F6E2F6E72A2
:1026280066782F6E7266785F676C75652E68000035
:102638002E2E2F2E2E2F2E2E2F2E2E2F2E2E2F2EAD
:102648002E2F6D6F64756C65732F6E7266782F68A8
:10265800616C2F6E72665F6770696F2E680000008C
:1026680000000050000300504750494F54450000F7
:10267800433A5C4E6F726469635F73656D695C6E43
:102688005246355F53444B5F31352E332E305F351C
:102698003961633334355C6D6F64756C65735C6E7A
:1026A8007266785C647269766572735C7372635C77
:1026B8006E7266785F6770696F74652E63000000DC
:1026C80050525300433A5C4E6F726469635F73659E
:1026D8006D695C6E5246355F53444B5F31352E331E
:1026E8002E305F353961633334355C6D6F64756CDA
:1026F80065735C6E7266785C647269766572735C29
:102708007372635C7072735C6E7266785F707273FA
:102718002E6300002E2E2F2E2E2F2E2E2F2E2E2FF4
:102728002E2E2F2E2E2F696E746567726174696F55
:102738006E2F6E7266782F6E7266785F676C75653D
:102748002E6800002E2E2F2E2E2F2E2E2F2E2E2FBF
:102758002E2E2F2E2E2F6D6F64756C65732F6E7253
:1027680066782F68616C2F6E72665F6770696F2E6E
:10277800680000005541525400000000433A5C4E86
:102788006F726469635F73656D695C6E5246355F2D
:1027980053444B5F31352E332E305F353961633307
:1027A80034355C6D6F64756C65735C6E7266785CED
:1027B800647269766572735C7372635C6E72667854
:1027C8005F756172742E6300E9C402002E2E2F2EED
:1027D8002E2F2E2E2F2E2E2F2E2E2F2E2E2F696E91
:1027E800746567726174696F6E2F6E7266782F6E8A
:1027F8007266785F676C75652E6800002E2E2F2E26
:102808002E2F2E2E2F2E2E2F2E2E2F2E2E2F6D6F5B
:1028180064756C65732F6E7266782F68616C2F6EA5
:1028280072665F6770696F2E6800000055415254E8
:1028380045000000433A5C4E6F726469635F7365DC
:102848006D695C6E5246355F53444B5F31352E33AC
:102858002E305F353961633334355C6D6F64756C68
:1028680065735C6E7266785C647269766572735CB7
:102878007372635C6E7266785F75617274652E63DD
:1028880000000000A9D00200433A5C4E6F726469F0
:10289800635F73656D695C6E5246355F53444B5F89
:1028A80031352E332E305F353961633334355C650D
:1028B80078616D706C65735C626C655F7065726978
:1028C80070686572616C5C626C655F6170705F7581
:1028D8006172745C6D61696E2E6300004C52616EAA
:1028E80067653831310000004661696C65642072A3
:1028F8006563656976696E67204E5553206D65730B
:10290800736167652E204572726F72203078257862
:102918002E200000436F6E6E6563746564000000CE
:10292800446973636F6E6E656374656400000000CC
:1029380044617461206C656E20697320736574202E
:10294800746F203078255828256429000800000075
:10295800060000000500000007000000000000005D
:1029680000E0D7014E524635323831312050657279
:102978006970686572616C20526F6C652053746170
:10298800727400005465726D696E616C000000001D
:10299800525454005345474745520000433A5C4E51
:1029A8006F726469635F73656D695C6E5246355F0B
:1029B80053444B5F31352E332E305F3539616333E5
:1029C80034355C636F6D706F6E656E74735C626CCA
:1029D800655C636F6D6D6F6E5C626C655F636F6E77
:1029E8006E5F73746174652E630000006E72665FBB
:1029F800626C655F676174740000000073645F62F5
:102A08006C655F6761705F646174615F6C656E6758
:102A180074685F757064617465282920287265710F
:102A28007565737429206F6E20636F6E6E656374AD
:102A3800696F6E20307825782072657475726E65BE
:102A4800642025732E000000546865207265717536
:102A580065737465642054582F5258207061636BF5
:102A68006574206C656E67746820697320746F6F75
:102A7800206C6F6E672062792025752F2575206F71
:102A880063746574732E00005468652072657175EF
:102A9800657374656420636F6D62696E6174696FD4
:102AA8006E206F6620545820616E64205258207042
:102AB80061636B6574206C656E67746873206973F5
:102AC80020746F6F206C6F6E6720627920257520E7
:102AD8006D6963726F7365636F6E64732E000000B7
:102AE80073645F626C655F67617474635F65786364
:102AF80068616E67655F6D74755F72657175657322
:102B08007428292072657475726E65642025732E89
:102B18000000000073645F626C655F6761747473C2
:102B28005F65786368616E67655F6D74755F726510
:102B3800706C7928292072657475726E6564202519
:102B4800732E0000626C655F6E7573009ECADC248C
:102B58000EE5A9E093F3A3B50000406E2E2E2F2EAC
:102B68002E2F2E2E2F2E2E2F2E2E2F2E2E2F636F02
:102B78006D706F6E656E74732F6C696272617269C5
:102B880065732F6578706572696D656E74616C5FC9
:102B980073656374696F6E5F766172732F6E7266A8
:102BA8005F73656374696F6E5F697465722E680020
:102BB8006E72665F73646800433A5C4E6F72646954
:102BC800635F73656D695C6E5246355F53444B5F56
:102BD80031352E332E305F353961633334355C63DC
:102BE8006F6D706F6E656E74735C736F6674646519
:102BF800766963655C636F6D6D6F6E5C6E72665F40
:102C08007364682E630000000100000714190300B4
:102C18001419030008000000141903001C1903000C
:102C2800080000001C1903002C190300080000000C
:102C38002E2E2F2E2E2F2E2E2F2E2E2F2E2E2F2EA7
:102C48002E2F636F6D706F6E656E74732F6C696273
:102C58007261726965732F6578706572696D656EEA
:102C680074616C5F73656374696F6E5F76617273AC
:102C78002F6E72665F73656374696F6E5F697465E2
:102C8800722E68006E72665F7364685F626C6500BE
:102C980073645F626C655F6366675F736574282938
:102CA8002072657475726E65642025732077686577
:102CB8006E20617474656D7074696E6720746F201E
:102CC80073657420424C455F434F4E4E5F43464701
:102CD8005F4741502E00000073645F626C655F635C
:102CE80066675F73657428292072657475726E65EE
:102CF80064202573207768656E20617474656D7033
:102D080074696E6720746F2073657420424C455F48
:102D18004741505F4346475F524F4C455F434F55CD
:102D28004E542E0073645F626C655F6366675F7301
:102D3800657428292072657475726E656420257320
:102D4800207768656E20617474656D7074696E674C
:102D580020746F2073657420424C455F434F4E4E7C
:102D68005F4346475F474154542E000073645F62D7
:102D78006C655F6366675F73657428292072657484
:102D880075726E6564202573207768656E2061749E
:102D980074656D7074696E6720746F207365742034
:102DA800424C455F434F4D4D4F4E5F4346475F563C
:102DB800535F555549442E0073645F626C655F63C9
:102DC80066675F73657428292072657475726E650D
:102DD80064202573207768656E20617474656D7052
:102DE80074696E6720746F2073657420424C455F68
:102DF80047415454535F4346475F415454525F54CC
:102E080041425F53495A452E0000000073645F62D7
:102E18006C655F6366675F736574282920726574E3
:102E280075726E6564202573207768656E206174FD
:102E380074656D7074696E6720746F207365742093
:102E4800424C455F47415454535F4346475F53459F
:102E580052564943455F4348414E4745442E00007A
:102E6800496E73756666696369656E742052414D73
:102E780020616C6C6F636174656420666F72207486
:102E8800686520536F66744465766963652E000033
:102E98004368616E6765207468652052414D2073F0
:102EA80074617274206C6F636174696F6E206672EE
:102EB8006F6D203078257820746F20307825782E33
:102EC800000000004D6178696D756D2052414D20FC
:102ED80073697A6520666F72206170706C696361CE
:102EE80074696F6E20697320307825782E00000091
:102EF80073645F626C655F656E61626C652829202A
:102F080072657475726E65642025732E000000006A
:102F1800433A5C4E6F726469635F73656D695C6E9A
:102F28005246355F53444B5F31352E332E305F3573
:102F38003961633334355C636F6D706F6E656E74C1
:102F4800735C736F66746465766963655C636F6DE3
:102F58006D6F6E5C6E72665F7364685F626C652E1F
:102F680063000000DC1803001419030008000000C7
:102F78002E2E2F2E2E2F2E2E2F2E2E2F2E2E2F2E64
:102F88002E2F636F6D706F6E656E74732F6C696230
:102F98007261726965732F6578706572696D656EA7
:102FA80074616C5F73656374696F6E5F7661727369
:102FB8002F6E72665F73656374696F6E5F6974659F
:102FC800722E68006E72665F7364685F736F630069
:102FD800433A5C4E6F726469635F73656D695C6EDA
:102FE8005246355F53444B5F31352E332E305F35B3
:102FF8003961633334355C636F6D706F6E656E7401
:10300800735C736F66746465766963655C636F6D22
:103018006D6F6E5C6E72665F7364685F736F632E4C
:1030280063000000D4180300DC1803000800000047
:1030380044300300743103004830030043000000AB
:10304800770F0300970F0300A30F0300AF0F0300D0
:10305800CF0F0300DB0F0300450F0300170F03001A
:1030680053756E004D6F6E005475650057656400AA
:10307800546875004672690053617400004A616EB5
:1030880000466562004D617200417072004D6179C1
:10309800004A756E004A756C00417567005365708B
:1030A800004F6374004E6F760044656300002E0085
:1030B8000053756E646179004D6F6E6461790054D8
:1030C800756573646179005765646E6573646179C9
:1030D8000054687572736461790046726964617935
:1030E80000536174757264617900004A616E75619C
:1030F8007279004665627275617279004D6172631A
:103108006800417072696C004D6179004A756E659E
:10311800004A756C79004175677573740053657062
:1031280074656D626572004F63746F626572004EFC
:103138006F76656D62657200446563656D62657280
:103148000000414D00504D0000256D2F25642F25AE
:10315800790025483A254D3A2553002561202562F6
:10316800202565202554202559000000B63003008D
:10317800B8300300B8300300B8300300B83003009B
:10318800B8300300B8300300B8300300B83003008B
:10319800B8300300FFFFFFFFFFFFFFFFFFFFFFFF48
:1031A800FFFF0000B930030068300300F33003006C
:1031B800853003004A310300513103005A310300BE
:1031C8006331030020202020202020202068282888
:1031D80028282020202020202020202020202020D7
:1031E800202020204810101010101010101010105F
:1031F800101010108484848484848484848410103F
:10320800101010101081818181818101010101015B
:103218000101010101010101010101010101011087
:103228001010101010828282828282020202020230
:103238000202020202020202020202020202021058
:10324800101010200007032004170201085710402F
:10325800803031323334353637383941424344458A
:103268004630313233343536373839616263646514
:0832780066286E756C6C2900DC
:1032800000000000FF00000000000000C41A03005E
:10329000CC1A0300D41A0300DC1A0300E41A03005A
:1032A000EC1A0300F41A0300FC1A0300041B0300C9
:1032B0000C1B0300141B03001C1B0300241B030036
:1032C000000000000020004000000000002000403E
:1032D000000000000090D003203400200100040012
:1032E00000000000000000000000000000000000DE
:1032F00000000000F02A002000000000FFFF140082
:103300004445564943455F3030303031C064000099
:103310000000000000000000FF0000004834002012
:103320001F000000683400201F0000000B00030095
:1033300091D902000C00030091D90200180003008B
:1033400091D902001900030091D90200383003001E
:1033500038300300383003003830030038300300C1
:0C336000DC3A0020E03A0020E43A0020B3
:040000032000637105
:00000001FF
